:040000005CEF00F0C1
:100008005D820F0112A913D00101652B8EA802D0C1
:1000180083A206D0899403AE02D0899201D0898246
:100028008EB883B201D089840F0112993DD012A1F4
:100038003BD00101642B8EB883B28992901C056E67
:100048008E1C066E038E89848EA0FED78EA802D0E1
:1000580083A202D0899401D0898406A822D00550B1
:100068007F0B096E0101E11902E1838205D0E0519D
:10007800091809E1838405D0839413D083A211D091
:10008800839483920ED00950076E086A085009E1DC
:100098000750040AF3E0100AF1E02B0AF2E0600AC4
:1000A800EBE089920F0112910E01CA995D9211003D
:1000B8004EEF4CF051C0D9FF52C0DAFFDE6ADD6A5C
:1000C80050C00AF0A6EC45F00AC08CF00BC08DF0C9
:1000D80000018DBF0B0CD8908C35D96E8D35DA6E3A
:1000E800480ED926010EDA22DECFA3F0DDCFA4F028
:1000F800A351A41101E10C0C51C0D9FF52C0DAFF81
:10010800A3C0DEFFA4C0DDFF5390A3C0D9FFA4C0E5
:10011800DAFFDF5012E020EE01F0A351D926A451F6
:10012800DA22DF50A2EC60F00001986F98B105D098
:100138005350D8A498A5000C0A0CA3C0D9FFA4C09A
:10014800DAFFDF6A20EE01F0A351D926A451DA22A2
:100158008CC0DFFF20EE01F0A351D926A451DA228A
:10016800DF50F0EC42F00001986F98B1030C535047
:1001780002E098B50A0CA3C048F0A4C049F04B6A45
:100188004A6A41EC46F048C0A1F049C0A2F0040E0A
:100198000001A119A21101E1010CA25103E1020E13
:1001A800A15D01E30D0C20EE2BF0A351D926A4513B
:1001B800DA22DECF94F0DECF95F0DECF96F0DECFF8
:1001C80097F03A0EA3250A6E000EA4210B6EAFEC31
:1001D8005EF0020E0B180A1001E00D0C450E00012E
:1001E800A3250A6E000EA4210B6EAFEC5EF00AC0C8
:1001F8009DF00BC09EF000019F6BA06B9D519E115E
:100208009F11A01110E1530EA3250A6E000EA42120
:100218000B6E1BEC53F00AC09DF00BC09EF00CC097
:100228009FF00DC0A0F0000120EE17F0A351D926D1
:10023800A451DA229DC0DEFF9EC0DEFF9FC0DEFF14
:10024800A0C0DEFF20EE3FF0A351D926A451DA2248
:1002580010EE02F0A351E126A451E222DFCFE7FF1E
:1002680020EE02F0A351D926A451DA22DE040AE0D6
:1002780020EE02F0A351D926A451DA22020EDE188C
:1002880001E00D0C9DC00AF09EC00BF09FC00CF061
:10029800A0C00DF020EE02F0A351D926A451DA2215
:1002A800DF500E6E0F6A106A116A77EC57F00AC0B9
:1002B8009DF00BC09EF00CC09FF00DC0A0F020EE8A
:1002C8003CF0A351D926A451DA22DF50746F756B24
:1002D80020EE09F0A351D926A451DA2274C0DEFF1A
:1002E80075C0DDFF20EE09F0A351D926A451DA220A
:1002F800DE50DE10D8B40D0C20EE09F0A351D9263B
:10030800A451DA22DECF74F0DDCF75F020EE09F0CB
:10031800A351D926A451DA22DECF76F0DDCF77F0CB
:10032800FF0E7625786FFF0E7721796F7451781557
:100338007A6F755179157B6F7A1101E00D0C400EBB
:10034800A3250A6E000EA4210B6EAFEC5EF000012F
:1003580020EE07F0A351D926A451DA220AC0DEFF05
:100368000BC0DDFF20EE07F0A351D926A451DA22F5
:10037800DF50746F0F0E741701E00D0C420EA325A9
:100388000A6E000EA4210B6EAFEC5EF00AC090F06E
:100398000BC091F00001926B936B905191119211E7
:1003A800931110E14F0EA3250A6E000EA4210B6EC7
:1003B8001BEC53F00AC090F00BC091F00CC092F007
:1003C8000DC093F03D0E0001A3250A6E000EA42176
:1003D8000B6EAFEC5EF00AC08EF00BC08FF0000120
:1003E8008E518F1101E10D0C20EE07F0A351D92693
:1003F800A451DA22DECF74F0DDCF75F0040E766FEB
:10040800D89075337433762FFBD78E517425776F58
:100418008F517521786F796BD8B0792B7A6B9D5194
:100428007725886F9E517821896F9F5179218A6F2E
:10043800A0517A218B6F8851905D895191598A51C9
:1004480092598B51935901E20D0C8851905D0A6EB7
:10045800895191590B6E8A5192590C6E8B5193594F
:100468000D6E20EE09F0A351D926A451DA22DECF71
:1004780074F0DDCF75F074C00EF075C00FF0106A1F
:10048800116AB4EC58F00AC099F00BC09AF00CC08D
:100498009BF00DC09CF0000199519A119B119C1181
:1004A80001E10D0CA16BA26BF60E995DFF0E9A5936
:1004B800FF0E9B590F0E9C5903E2A26B030EA16F0E
:1004C8009C519B1108E1F60E995DFF0E9A5903E2C3
:1004D800A26B020EA16F9C519B1108E1F60E995D6B
:1004E8000F0E9A5903E2A26B010EA16FA151A2113E
:1004F80001E10D0C020E9925746F000E9A21756F9B
:10050800000E9B21766F000E9C21776F20EE13F072
:10051800A351D926A451DA2274C0DEFF75C0DEFFCC
:1005280076C0DEFF77C0DEFF20EE1BF0A351D92690
:10053800A451DA2294C0DEFF95C0DEFF96C0DEFF2C
:1005480097C0DEFF8E519425746F8F519521756F7A
:10055800000E9621766F000E9721776F20EE1FF020
:10056800A351D926A451DA2274C0DEFF75C0DEFF7C
:1005780076C0DEFF77C0DEFF88519425746F8951FD
:100588009521756F8A519621766F8B519721776FD8
:1005980020EE27F0A351D926A451DA2274C0DEFF39
:1005A80075C0DEFF76C0DEFF77C0DEFF030EA1193F
:1005B800A2114DE1590EA3250A6E000EA4210B6E5F
:1005C800AFEC5EF00A500B1001E00D0C000120EEBC
:1005D80007F0A351D926A451DA22DE50DE1001E03B
:1005E8000D0C5B0EA3250A6E000EA4210B6E1BECEE
:1005F80053F0000120EE23F0A351D926A451DA22AA
:100608000AC0DEFF0BC0DEFF0CC0DEFF0DC0DEFF40
:1006180020EE13F0A351D926A451DA22DECF74F0CC
:10062800DECF75F0DECF76F0DECF77F0020ED89011
:100638007437753776377737E82EF9D774C084F072
:1006480075C085F076C086F077C087F0B8D020EE08
:1006580007F0A351D926A451DA22DE50DE1001E1B9
:100668000D0C20EE1FF0A351D926A451DA22DECFBB
:1006780074F0DECF75F0DECF76F0DECF77F09D51E7
:100688007425786F9E517521796F9F5176217A6F05
:10069800A05177217B6F20EE23F0A351D926A451D6
:1006A800DA2278C0DEFF79C0DEFF7AC0DEFF7BC0C9
:1006B800DEFF020EA119A2116BE020EE13F0A35188
:1006C800D926A451DA22DECF74F0DECF75F0DECF62
:1006D80076F0DECF77F0010E7415786F796B7A6B50
:1006E8007B6B20EE13F0A351D926A451DA22DECF7A
:1006F8007CF0DECF7DF0DECF7EF0DECF7FF0030E24
:100708007C03F3CF80F0F4CF81F0826B836B7D03A1
:10071800F3508127F4508223000E83237C03F35087
:100728008127F4508223000E8323030E7E03F350A7
:100738008227F4508323000E7D03F3508227F45060
:100748008323000E7C03F3508227F4508323030E87
:100758007F03F3508327000E7E03F3508327000E98
:100768007D03F3508327000E7C03F3508327D89032
:10077800833382338133803378518025846F795174
:100788008121856F7A518221866F7B51832116D012
:1007980020EE13F0A351D926A451DA22DECF74F04B
:1007A800DECF75F0DECF76F0DECF77F0D8907435F7
:1007B800846F7535856F7635866F7735876FFF0E51
:1007C8008425746F010E8521756F000E8621766F62
:1007D800000E8721776F0A0E05D0D89077337633CD
:1007E80075337433E82EF9D720EE17F0A351D926C4
:1007F800A451DA227451DE5C7551DE587651DE5808
:100808007751DE5801E20D0C20EE0FF0A351D926E6
:10081800A451DA22DE68DE68DE68DD68DD52DD526A
:1008280010EE0BF0A351E126A451E222DECFE6FF41
:10083800DECFE6FFDECFE6FFDECFE6FF20EE04F0F8
:10084800A351D926A451DA22800EDF6E030EA11916
:10085800A21101E090D05F0EA3250A6E000EA4211C
:100868000B6EAFEC5EF00A040B1001E084D0A3C05D
:1008780036F0A4C037F0010E00019425386E000E42
:100888009521396E000E96213A6E000E97213B6E27
:100898005EEC54F000096FE1000120EE04F0A35172
:1008A800D926A451DA22DF6A2D0EA3250A6E020E7C
:1008B800A4210B6EAFEC5EF0550E0A185CE1AA0E8F
:1008C8000B1859E12F0E0001A3250A6E000EA42172
:1008D8000B6E1BEC53F0520E0A184DE1520E0B181A
:1008E8004AE1610E0C1847E1410E0D1844E1130E60
:1008F8000001A3250A6E020EA4210B6E1BEC53F017
:10090800720E0A1838E1720E0B1835E1410E0C18F8
:1009180032E1610E0D182FE1170E0001A3250A6EB2
:10092800020EA4210B6E1BEC53F0000120EE0FF019
:10093800A351D926A451DA220AC0DEFF0BC0DEFF7C
:100948000CC0DEFF0DC0DEFF1B0EA3250A6E020ED3
:10095800A4210B6E1BEC53F0000120EE0BF0A35109
:10096800D926A451DA220AC0DEFF0BC0DEFF0CC074
:10097800DEFF0DC0DEFFA3C0D9FFA4C0DAFFA1C00F
:10098800DFFF0101464B472B000120EE05F0A35184
:10099800D926A451DA2246C1DEFF47C1DDFF000C8B
:1009A8000B6A0A6A5BEC60F00101F86F5B6B070E7B
:1009B8008C6E010EF76F626B04000F010D6B156BE7
:1009C8001D6B226B0F0E596F116B196B216B266B08
:1009D8002E6B0E6B166B1E6B236B2B6B88688968EE
:1009E8008A688A8E8890889283820382FAEC5EF005
:1009F80088948384888C839C889E838E8B6889687E
:100A0800FC0E00019D6FF80E9E6FA60E9F6FFF0EE5
:100A1800A06FB40EA16FFE0EA26F3F0EA36FFF0E64
:100A2800A46F4FEC60F08A98858894EC5EF0630EB2
:100A380000019D6FFB0E9E6FF8C19FF0A06B4FECFD
:100A480060F00101F82901E1F86B0F0EF817FEECD0
:100A580047F00101F86F7B0E00019D6FFB0E9E6F42
:100A6800F8C19FF0A06B4FEC60F00400190E010173
:100A7800C06F5A0EBF6FB10EE82EFED7BF2FFCD73E
:100A8800C02FFAD700D0D250F00B0109D26ED09EF9
:100A98000E01C691CF0ECF16CF82CF80C2890F012B
:100AA8001381138914890E01BA89F28EEFEC58F07C
:100AB80083928394040015EC50F015EC50F05A0E14
:100AC8000E6EFF0E0F6E77EC58F0A60E0E6EFF0E30
:100AD8000F6E77EC58F08FA22FD0290E0101C06F4E
:100AE800960EBF6F7F0EE82EFED7BF2FFCD7C02F04
:100AF800FAD7000E0A6E800E38EC5CF0270E0E6EE8
:100B0800FE0E0F6E77EC58F017D0690E00019D6F3E
:100B1800FE0E9E6F8FCF9FF0A06B4FEC60F0290EFA
:100B28000101C06F960EBF6F7F0EE82EFED7BF2F54
:100B3800FCD7C02FFAD704008FB2E7D78380040010
:100B4800AAEC49F0F30E00019D6FFC0E9E6F61C187
:100B58009FF0A06B4FEC60F0000E0A6EC00E38ECF0
:100B68005CF0660E1E6E010E1F6E7B0E206EFC0E74
:100B7800216E61C122F0236AC9EC5EF0660E0E6E2A
:100B8800010E0F6E77EC58F0190E0101C06F5A0E66
:100B9800BF6FB10EE82EFED7BF2FFCD7C02FFAD7F4
:100BA80000D02CEC35F001016151200FE16F61514B
:100BB800400FE06F6151600FDF6F839EF7050EE114
:100BC8005F510CE1540E00019D6FFD0E9E6F4FECBE
:100BD80060F0020E01015F6F220E5E6FF7510EE1A9
:100BE8005F510CE1440E00019D6FFD0E9E6F4FECAE
:100BF80060F0010E01015F6F040E5E6F5A5102E052
:100C080082EC40F0DEC193FF6CEC2DF053EC51F018
:100C1800000E0A6E800E38EC5CF050EC5FF0000EAF
:100C28000A6E800E38EC5CF00101F8510F0D2F0EA2
:100C3800F3240E6E090EF4200F6E77EC58F00101C4
:100C480062BF61EC44F00101C46BC96B000EC76F51
:100C5800010EC66FC7BF05D0C75166E1040EC65D59
:100C680063E20F0EC603F3CFBFF1F4CFC0F1C703A1
:100C7800F350C0271F0EBF250A6E0A0EC0210B6E47
:100C880011EC5DF00B5003E1030E0A5C49E3B10E71
:100C980000019D6FFD0E9E6F0F0E0101C603F3CF7D
:100CA800BFF1F4CFC0F1C703F350C0271F0EBF2513
:100CB80000019F6F0A0E0101C0210001A06F4FECD7
:100CC80060F0220E0101C603F3CFBFF1F4CFC0F1EB
:100CD800C703F350C027000EBF250001B96F030EEC
:100CE8000101C0210001BA6F0F0E0101C603F3CF45
:100CF800C1F1F4CFC2F1C703F350C2271F0EC125BB
:100D08000001BB6F0A0E0101C2210001BC6F030E76
:100D1800BD6FBDEC11F00101C56FC55166EC5BF00C
:100D28000101C64BC72B96D75C5101E18C905C053D
:100D380002E1070E8C6E020E5C1901E057D1020E1B
:100D48005C1901E053D10F01108B070E2D6F4ED1A6
:100D5800849284948EA889948BEC60F00A500B10CE
:100D680001E103D1C9C1C3F1C80E0A6E010E0B6EB1
:100D78001CEC60F00101C96FC8B9C99F62511CE041
:100D8800350EC91907E12A0E00019D6FF90E9E6FF5
:100D98004FEC60F0480E00019D6FFF0E9E6FC9C1B9
:100DA8009FF0A06B0101C8390F0B030B0001A16F65
:100DB800A26B4FEC60F004D06A0EE82EFED700D08C
:100DC8000101F75109E10D0E0101BF6F760EE82E02
:100DD800FED7BF2FFCD700000101C8A92FD0DF51D3
:100DE800C9192CE15F0EC31929E1620E00019D6F3C
:100DF800FF0E9E6F4FEC60F00382030E9D6FFF0E97
:100E08009E6F5FC19FF0A06B5EC1A1F0A26B4FEC1B
:100E180060F027EE2FF05FC1DFFF27EE30F05EC1F4
:100E2800DFFF8384020EA9EC56F08394039201013C
:100E3800636BB5EC60F00101C96BD8D0F75145E0A0
:100E4800C851100B4F6E000E506EC951FEEC39F0B0
:100E58004FC0CAF150C0CBF1080E0101CA19CB111D
:100E680001E10000070E0101CA19CB1102E1DAEC19
:100E78005AF0CA05CB1102E142EC55F0020E01010D
:100E8800CA19CB1102E1DAEC38F0030E0101CA19D4
:100E9800CB1104E1D0EC1EF00101C46F050ECA1994
:100EA800CB1104E1EDEC3BF00101C46F090ECA1946
:100EB800CB1102E10FEC52F00A0E0101CA19CB1155
:100EC80001E094D0C7EC4DF091D0C8C11FF0206A62
:100ED800C95130EC17F01FC0CAF120C0CBF1070E82
:100EE8000101CA19CB1102E176EC5AF0020ECA19B7
:100EF800CB1102E1D4EC59F0CA05CB1102E11FEC89
:100F080023F0030ECA19CB1102E183EC50F0040E52
:100F1800CA19CB1102E1E2EC5EF0050ECA19CB1139
:100F280002E1C0EC4AF0060E0101CA19CB1102E138
:100F3800ACEC60F0080ECA19CB1102E1FCEC3AF0F7
:100F4800090ECA19CB1102E1BBEC4EF00A0E0101E1
:100F5800CA19CB1102E1B1EC5DF00C0E0101CA19FE
:100F6800CB1144E1D0EC33F041D0FEEC47F0010165
:100F78005B6F5C513BE0F8515B1938E0838E000EE3
:100F88000A6EC00E38EC5CF050EC5FF0000E0A6E92
:100F9800C00E38EC5CF0F80E0E6EFE0E0F6E77EC9D
:100FA80058F05BC1F8F1000E526E030E536E26EC3A
:100FB8005EF02CEC35F001015A5102E082EC40F071
:100FC800420E00019D6FFA0E9E6FF8C19FF0A06B54
:100FD8005FC1A1F0A26B5EC1A3F0A46B4FEC60F0FF
:100FE8000101F75103E0F85137EC60F08FB22ED0D1
:100FF800050E0101C4192AE0ABD6690E00019D6FE8
:10100800FE0E9E6F8FCF9FF0A06B4FEC60F0290E05
:101018000101C06F960EBF6F7F0EE82EFED7BF2F5F
:10102800FCD7C02FFAD70400000E0A6EC00E38ECA9
:101038005CF050EC5FF0000E0A6EC00E38EC5CF00D
:101048006A0E0E6EFF0E0F6E77EC58F08FB2D5D782
:10105800090E0101C06F1E0EBF6FE40EE82EFED709
:10106800BF2FFCD7C02FFAD70000839483920001CA
:10107800A56BA66B2C0EA76FF90EA86FA96BD4EC05
:1010880055F05DD5466E456AF3D2090E461817E14C
:10109800595015E0456A8390456A010E586E5A50BA
:1010A8001E0D1B0EF324D96E020EF420DA6E200EEC
:1010B800DF6E030E0101576F446B456B83904650FA
:1010C80009E1595007E0456A0101456B0A0EB1D0A4
:1010D800839046D3020E461807E1595005E0456A49
:1010E8000101456B140EA5D01F0E466438D0300E92
:1010F800466035D0595033E04650E00F5A6E456A85
:101108000F0E5A1805E156C158F00101566BACD2C2
:101118005A50220D0A0EF324D96E030EF420DA6E0B
:10112800DE50DE10DE10DE1003E0030E5A649CD29F
:101138005A6A010E586E5A501E0D1B0EF324D96EB2
:10114800020EF420DA6E5A501E0D1B0EF324E16EC7
:10115800020EF420E26EE7501009DF6E85D23F0ED2
:10116800466428D0480E466025D0595023E05A508E
:101178001E0D000EF324D96E020EF420DA6E4650CE
:10118800C00FDF6E5A501E0D000EF324D96E020EEA
:10119800F420DA6EDF500CE05A501E0D1B0EF324BB
:1011A800D96E020EF420DA6E100EDF6E010E586E44
:1011B800456A5AD2480E461808E1595006E0456A71
:1011C800120E0101456FC00E34D0310E461807E1EA
:1011D800595005E00C0E0101456F1D0E2ED2340E3C
:1011E800461807E1595005E00101446B456B456A13
:1011F8006FD7350E461808E1595006E0456A0D0EBE
:101208000101456FAC0E15D0370E461808E159504C
:1012180006E083800E0E0101456F750E0ED20D0E8D
:10122800461809E1595007E0456A020E0101456F69
:10123800BC0E446F4DD7100E461807E1595005E013
:10124800030E0101456FE90EF8D1180E461807E1A3
:10125800595005E0070E0101456F090EEED13B0E0E
:10126800461807E1595005E00E0E0101456F7E0E44
:10127800E4D13E0E461801E073D2595001E170D214
:101288000F0E0101456F3D0ED8D15A501E0D010EAB
:10129800F324D96E020EF420DA6E46C0DFFF030E87
:1012A8000101456FEA0EC9D15A501E0D020EF324F2
:1012B800D96E020EF420DA6E46C0DFFF030E01017C
:1012C800456FEB0EBAD15A501E0D030EF324D96E9A
:1012D800020EF420DA6E46C0DFFF030E0101456FEF
:1012E800EC0EABD15A501E0D040EF324D96E020E2B
:1012F800F420DA6E46C0DFFF030E0101456FED0EE4
:101308009CD15A501E0D050EF324D96E020EF420FE
:10131800DA6E46C0DFFF030E0101456FEE0E8DD178
:101328005A501E0D060EF324D96E020EF420DA6E02
:1013380046C0DFFF5A501E0D050EF324D96E020E6B
:10134800F420DA6EDF50226E22C023F0246A256A68
:10135800266A25C026F024C025F023C024F0236A7D
:101368005A501E0D040EF324D96E020EF420DA6EC4
:10137800DF50276E27C028F0296A2A6A2B6A29C0FD
:101388002BF028C02AF0296A286A5A501E0D030E2D
:10139800F324D96E020EF420DA6EDF502C6E2CC0C6
:1013A8002DF02E6A2F6A306A2DC030F02F6A2E6A0F
:1013B8002D6A28502D24316E29502E20326E2A5045
:1013C8002F20336E2B503020346E23503124356E4D
:1013D80024503220366E25503320376E2650342064
:1013E800386E5A501E0D060EF324D96E020EF420E4
:1013F800DA6EDF503524396E000E36203A6E000E54
:1014080037203B6E000E38203C6E39C03DF03AC0A4
:101418003EF03BC03FF03CC040F0416A40BE4168EE
:1014280041C042F041C043F041C044F05A501E0D43
:10143800070EF324D96E020EF420DA6E3DC0DEFFEB
:101448003EC0DEFF3FC0DEFF40C0DEFF41C0DEFF22
:1014580042C0DEFF43C0DEFF44C0DEFF5A501E0D0F
:101468001C0EF324D96E020EF420DA6EDECF22F0C1
:10147800DDCF23F022C00AF023C00BF00C6A0D6AFE
:101488000E6A0F6A106A116A5A501E0D070EF3246D
:10149800D96E020EF420DA6EDECF24F0DECF25F00E
:1014A800DECF26F0DECF27F0DECF28F0DECF29F022
:1014B800DECF2AF0DECF2BF024C012F025C013F0C7
:1014C80026C014F027C015F028C016F029C017F060
:1014D8002AC018F02BC019F063EC56F00AC02CF0A3
:1014E8000BC02DF00CC02EF00DC02FF00EC030F048
:1014F8000FC031F010C032F011C033F05A501E0D39
:10150800070EF324D96E020EF420DA6E2CC0DEFF2B
:101518002DC0DEFF2EC0DEFF2FC0DEFF30C0DEFF95
:1015280031C0DEFF32C0DEFF33C0DEFF8390010131
:10153800446B456B15D15A501E0D1A0EF324D96E03
:10154800020EF420DA6E46C0DFFF070E0101456F78
:101558000A0E73D05A501E0D190EF324D96E020EBE
:10156800F420DA6E46C0DFFF070E0101456F0B0E4F
:1015780064D05A501E0D180EF324D96E020EF420B2
:10158800DA6E46C0DFFF070E0101456F0C0E55D01D
:101598005A501E0D170EF324D96E020EF420DA6E7F
:1015A80046C0DFFF61D00101446B456B586A90D596
:1015B80046C030F10F0E0101456F3E0E3ED046C0C9
:1015C80031F10F0E0101456F3F0E37D046C032F1A1
:1015D8000F0E0101456F400E30D046C033F10F0E9B
:1015E8000101456F410E29D046C034F10F0E0101AB
:1015F800456F420E22D046C035F10F0E0101456FEE
:10160800430E1BD046C036F10F0E0101456F440E44
:1016180014D046C037F128D00C0E0101456F1E0EBC
:101628000CD00C0E0101456F1C0E446F0A0E456E5E
:101638004FD50E0E0101456F760E446F91D0010112
:10164800446B456B090E456E83808AD046500CE08A
:101658005A501E0D1B0EF324D96E020EF420DA6EBA
:10166800080EDF6E010E586E0101446B456B30D5D4
:1016780044C122F045C123F0235013E0030A15E0CA
:10168800040A27E00B0A33E0010A37E0030A3BE0CB
:10169800010A42E01D0A5AE00E0A5DE03B0A5EE0DC
:1016A8005FD0225001E1F1D45BD02250E90A01E178
:1016B800ECD5030A01E1F8D5010A01E104D6070ACD
:1016C80001E110D6010A01E11CD6030A01E128D67E
:1016D80047D02250090A01E12ED7030A01E13AD77F
:1016E800010A01E146D7070A01E152D739D0225051
:1016F8001D0A92E0030A95E033D02250480A01E11E
:1017080016D7E40A2DD02250750A93E0030A97E011
:10171800080A01E148D724D022503D0A01E148D700
:10172800030A01E14CD7010A01E150D77F0A01E120
:1017380054D7010A01E158D7030A01E15CD7010A2D
:1017480001E160D7070A01E164D70AD02250C00A34
:1017580001E17CD705D022502A0A02D022500F0A74
:10176800455012008DC0A3F08EC0A4F09151D96EDF
:10177800DA6ADE6ADD6A8BC00BF08CC00CF0B30E3F
:101788000D6EC5EC52F00001A26FA2510AE120EEE5
:101798000FF08B51D9268C51DA22DF50A26FA2515B
:1017A80002E0A251120020EE0EF08B51D9268C5186
:1017B800DA22DFA2070C20EE10F08B51D9268C51CB
:1017C800DA2210EE10F08B51E1268C51E222E6CF9E
:1017D80096F0E6CF97F0E6CF98F0E6CF99F08F51E4
:1017E80096259A6F905197219B6F000E98219C6FB8
:1017F800000E99219D6FDE509A5DDE509B59DE5098
:101808009C59DE509D5901E3D9D220EE10F08B513E
:10181800D9268C51DA22DECF92F0DDCF93F0921DDB
:101828008F6F931D906FCAD220EE10F08B51D9267E
:101838008C51DA22FF0EDE14926F010EDE14936FC4
:10184800000EDE14946F000EDE14956F9251931102
:101858009411951101E0FDD120EE10F08B51D9269D
:101868008C51DA22DECF92F0DECF93F0DECF94F007
:10187800DECF95F00A0E05D0D89095339433933384
:101888009233E82EF9D720EE09F0B351D926B45196
:10189800DA22DECF96F0DDCF97F0FF0E9625986F0F
:1018A800FF0E9721996F92519815A56F935199152D
:1018B800A66FA51101E091D020EE10F08B51D9262A
:1018C8008C51DA22DE50DE10DE10DE101EE120EE32
:1018D80006F08B51D9268C51DA22DECFADF0DECF5F
:1018E800AEF0DECFAFF0DECFB0F0AD51AE11AF113C
:1018F800B01127E18BC06EF08CC06FF0706B716B0C
:10190800726B736B3FEC25F014D08BC06EF08CC0FB
:101918006FF020EE14F08B51D9268C51DA22DECFED
:1019280070F0DECF71F0DECF72F0DECF73F03FECF7
:1019380025F06EC0ADF06FC0AEF070C0AFF071C0F2
:10194800B0F0AD51AE11AF11B01101E13BD2AD0510
:10195800AE11AF11B01109E120EE0FF08B51D9266D
:101968008C51DA22020EDF6E020CAD290FE1AE298E
:101978000DE1AF290BE1B02909E120EE0FF08B5101
:10198800D9268C51DA22010EDF6E010C20EE14F0FC
:101998008B51D9268C51DA22ADC0DEFFAEC0DEFFF6
:1019A800AFC0DEFFB0C0DEFF20EE06F08B51D926B7
:1019B8008C51DA22DE50DE10DE10DE100EE120EE51
:1019C80006F08B51D9268C51DA22ADC0DEFFAEC0AD
:1019D800DEFFAFC0DEFFB0C0DEFF20EE18F08B5197
:1019E800D9268C51DA2210EE2BF0B351E126B451EE
:1019F800E222DE50E61812E1DE50E6180FE1DE5072
:101A0800E6180CE1DE50E61809E1B3C023F0B4C0D3
:101A180024F0AEEC43F0000901E051D1B3C00AF064
:101A2800B4C00BF0000120EE14F08B51D9268C5174
:101A3800DA22DECF0CF0DECF0DF0DECF0EF0DECFF7
:101A48000FF036EC4AF00AC0A9F00BC0AAF00CC09F
:101A5800ABF00DC0ACF00001A951AA11AB11AC114B
:101A680001E17AD7A551A927A651AA23000EAB23D5
:101A7800AC238FC092F090C093F0090E946FD89069
:101A880093339233942FFBD792C0A7F093C0A8F05A
:101A9800A751A81101E1A2D0A751A525926FA8517D
:101AA800A621936F20EE09F0B351D926B451DA225A
:101AB8009251DE5C9351DE5810E220EE09F0B351EA
:101AC800D926B451DA22DECF92F0DDCF93F0A551BA
:101AD800925DA76FA6519359A86FA3C019F0A4C02F
:101AE8001AF0A9C01BF0AAC01CF0ABC01DF0ACC016
:101AF8001EF0A7C01FF0A8C020F020EE01F0B351DF
:101B0800D926B451DA22DF5032EC4FF0000901E057
:101B1800D6D00001A751926FA851936F946B956B23
:101B280020EE2BF0B351D926B451DA22DECF96F04D
:101B3800DECF97F0DECF98F0DECF99F0A951965D11
:101B48009A6FAA5197599B6FAB5198599C6FAC519A
:101B580099599D6F92519A5D93519B5994519C59F3
:101B680095519D592CE22F0EB3250A6E000EB42113
:101B78000B6E20EE2BF0B351D926B451DA22DECF0A
:101B880092F0DDCF93F0A951925FAA51935B090EB1
:101B9800D89092379337E82EFBD79251A3250C6E35
:101BA8009351A4210D6E020E0F6E0E6AF0EC5CF0DC
:101BB80020EE03F0B351D926B451DA22DF6AA7C068
:101BC80092F0A8C093F0090ED89092379337E82E78
:101BD800FBD792C0B1F093C0B2F0A1D020EE0AF0CA
:101BE8008B51D9268C51DA2210EE10F08B51E12658
:101BF8008C51E222DE50E65CDE50E658DE50E658B4
:101C0800DE50E65818E3B3C023F0B4C024F0AEECBD
:101C180043F0000901E053D0000120EE2BF0B3514E
:101C2800D926B451DA22A9C0DEFFAAC0DEFFABC0B4
:101C3800DEFFACC0DEFF20EE18F08B51D9268C51A8
:101C4800DA22A9C0DEFFAAC0DEFFABC0DEFFACC04F
:101C5800DEFF20EE10F08B51D9268C51DA22DECF30
:101C680092F0DDCF93F09251946F010E9315956F1A
:101C780094510008B16F9551D8A0E82A0208B26FB4
:101C8800B1518F5DB251905904E28FC0B1F090C04C
:101C9800B2F0B3C036F0B4C037F020EE18F08B5174
:101CA800D9268C51DA22DECF38F0DECF39F0DECFFC
:101CB8003AF0DECF3BF05EEC54F0000902E00001A0
:101CC8005CD6000120EE10F08B51D9268C51DA2217
:101CD800DECF92F0DDCF93F09251946F010E931501
:101CE800956F9451B325966F9551B421976F2F0E28
:101CF80096250A6E000E97210B6EA3C00CF0A4C0A7
:101D08000DF0B1C00EF0B2C00FF0F0EC5CF020EEB8
:101D180003F0B351D926B451DA22010EDF6EB15166
:101D28008F5FB251905B9151D96EDA6AB151DE265C
:101D3800B251DD22B151A327B251A42320EE10F0F5
:101D48008B51D9268C51DA22B151DE26B251DE22CE
:101D5800000EDE22DE2220EE10F08B51D9268C51A7
:101D6800DA2210EE0AF08B51E1268C51E222DE5085
:101D7800E65CDE50E658DE50E658DE50E65820EEC7
:101D88000AF0D8A020EE10F08B51D9268C51DA2217
:101D9800DECF9EF0DECF9FF0DECFA0F0DECFA1F049
:101DA80020EE0AF08B51D9268C51DA229EC0DEFF34
:101DB8009FC0DEFFA0C0DEFFA1C0DEFF8F519011E3
:101DC80001E032D520EE0EF08B51D9268C51DA2263
:101DD800000EDB8C000C8BC00BF08CC00CF0A90E35
:101DE8000D6EC5EC52F00001AB6FAB5108E120EE6F
:101DF8000FF08B51D9268C51DA22DF50AB6FAB51E3
:101E080002E0AB51120020EE0AF08B51D9268C511A
:101E1800DA228D51DE5C8E51DE588F51DE5890519A
:101E2800DE5816E220EE0EF08B51D9268C51DA22BC
:101E3800DFB20ED020EE0AF08B51D9268C51DA226F
:101E4800DECF8DF0DECF8EF0DECF8FF0DECF90F0DC
:101E580020EE10F08B51D9268C51DA22DECFA1F07A
:101E6800DECFA2F0DECFA3F0DECFA4F0A56BA66B89
:101E7800A76BA86B20EE10F08B51D9268C51DA2273
:101E8800A5C0DEFFA6C0DEFFA7C0DEFFA8C0DEFF3C
:101E98008D518E118F11901101E100D220EE09F0C1
:101EA800A951D926AA51DA22DECF91F0DDCF92F0DE
:101EB8009151936F9251946F956B966B090ED890D0
:101EC8009337943795379637E82EF9D793C0ACF007
:101ED80094C0ADF095C0AEF096C0AFF0A151A2117C
:101EE800A311A41101E196D0FF0E8D250A6EFF0EF5
:101EF8008E210B6EFF0E8F210C6EFF0E90210D6E42
:101F0800ACC00EF0ADC00FF0AEC010F0AFC011F015
:101F1800B4EC58F00AC091F00BC092F00CC093F0EA
:101F28000DC094F0FF0E0001A1250A6EFF0EA2213C
:101F38000B6EFF0EA3210C6EFF0EA4210D6EACC01C
:101F48000EF0ADC00FF0AEC010F0AFC011F0B4ECA1
:101F580058F00A500001915D0B5092590C5093595A
:101F68000D50945957E3FF0EAC25916FFF0EAD212C
:101F7800926FFF0EAE21936FFF0EAF21946F911DEC
:101F8800956F921D966F931D976F941D986FFF0E16
:101F9800A125996FFF0EA2219A6FFF0EA3219B6FB7
:101FA800FF0EA4219C6F955199159D6F96519A1516
:101FB8009E6F97519B159F6F98519C15A06F20EEAF
:101FC80010F08B51D9268C51DA229DC0DEFF9EC0BD
:101FD800DEFF9FC0DEFFA0C0DEFF20EE10F08B51B9
:101FE800D9268C51DA22DE508D5FDE508E5BDE50B2
:101FF8008F5BDD50905B20EE14F08B51D9268C510D
:10200800DA22DECFB0F0DECFB1F0DECFB2F0DECF35
:10201800B3F060D020EE06F08B51D9268C51DA222D
:10202800DECFB0F0DECFB1F0DECFB2F0DECFB3F06E
:10203800B051B111B211B3113FE18BC06EF08CC039
:102048006FF0706B716B726B736B3FEC25F06EC049
:10205800B0F06FC0B1F070C0B2F071C0B3F0B005AD
:10206800B111B211B31109E120EE0FF08B51D9264D
:102078008C51DA22020EDF6E020CB0290FE1B12971
:102088000DE1B2290BE1B32909E120EE0FF08B51E4
:10209800D9268C51DA22010EDF6E010C20EE06F0F3
:1020A8008B51D9268C51DA22B0C0DEFFB1C0DEFFD9
:1020B800B2C0DEFFB3C0DEFF20EE14F08B51D9268C
:1020C8008C51DA22B0C0DEFFB1C0DEFFB2C0DEFF45
:1020D800B3C0DEFFB051B111B211B31101E085D028
:1020E800DDD0AC518D5FAD518E5BAE518F5BAF5182
:1020F800905B20EE10F08B51D9268C51DA22AC512E
:10210800DE26AD51DE22AE51DE22AF51DE2220EEB8
:102118000EF08B51D9268C51DA22DFA220D08BC049
:102128006EF08CC06FF0B0C070F0B1C071F0B2C08A
:1021380072F0B3C073F03FEC25F06EC0B0F06FC022
:10214800B1F070C0B2F071C0B3F0B051B111B211BA
:10215800B3111BE18D6B8E6B8F6B906B50D08BC066
:1021680041F08CC042F0B0C043F0B1C044F0B2C0FE
:1021780045F0B3C046F026EC2FF041C0B0F042C0A5
:10218800B1F043C0B2F044C0B3F00001B02907E198
:10219800B12905E1B22903E1B32901E176D7B351A9
:1021A800B211B11104E1020EB05D01E25DD720EE7B
:1021B80013F0A951D926AA51DA22DE50B05DDE50BB
:1021C800B159DE50B259DE50B35901E34DD720EE74
:1021D80014F08B51D9268C51DA22B0C0DEFFB1C081
:1021E800DEFFB2C0DEFFB3C0DEFF8D51AC5D8E51A5
:1021F800AD598F51AE599051AF5901E272D720EEC7
:1022080010F08B51D9268C51DA228D51DE268E5151
:10221800DE228F51DE229051DE228D51916F010E08
:102228008E15926F936B946B91119311941136E004
:10223800A9C00AF0AAC00BF0B0C00CF0B1C00DF0F4
:10224800B2C00EF0B3C00FF036EC4AF00AC0A5F0E9
:102258000BC0A6F00CC0A7F00DC0A8F00001A55156
:10226800A611A711A81101E1FFD68DC091F08EC06B
:1022780092F08FC093F090C094F00A0E05D0D890D9
:102288009433933392339133E82EF9D79151A5279C
:102298009251A6239351A7239451A82320EE10F01E
:1022A8008B51D9268C51DA2210EE0AF08B51E12697
:1022B8008C51E222DE50E65CDE50E658DE50E658ED
:1022C800DE50E6581CE220EE10F08B51D9268C51D6
:1022D800DA2210EE0AF08B51E1268C51E222DECF91
:1022E800E6FFDECFE6FFDECFE6FFDECFE6FF20EE3D
:1022F8000EF08B51D9268C51DA22000EDB8C20EEA1
:1023080010F08B51D9268C51DA22FF0EDE14916F12
:10231800010EDE14926F000EDE14936F000EDE14B1
:10232800946F915192119311941101E16AD520EEA5
:1023380018F08B51D9268C51DA22A551DE180AE102
:10234800A651DE1807E1A751DE1804E1A851DE18EE
:1023580001E157D520EE18F08B51D9268C51DA229D
:10236800A5C0DEFFA6C0DEFFA7C0DEFFA8C0DEFF57
:1023780048D5B951BA1101E1090C3F0EBD17BB0E82
:10238800506E8E0E516E010E526EBDC053F05EEC53
:1023980000F00101906F905101E0A8D28EC191F137
:1023A8008FC192F1910E0001AB6F010EAC6FBBC0F3
:1023B800ADF0BCC0AEF026EC42F00101906F905138
:1023C80004E1B8AF02D0060E906FBDC0BEF01C0E7F
:1023D8000001BE1701E1D1D0010190510FE0040EB8
:1023E800901909E1910E0001AE6F010EAF6FB1ECCB
:1023F80051F00101906F0001BD870DD095C1BEF06D
:10240800110E0001BE1702E0070E03D0BDA503D0D0
:10241800080E0101906F0101905101E0BDD000014B
:10242800BDA7BAD08EC111F08FC112F0ABC113F0A5
:10243800ACC114F029EC59F011C07EF112C07FF143
:1024480013C080F114C081F10E0E0101AB250A6E94
:10245800000EAC210B6E0C6A0D6A210E0E6E500E2A
:102468000F6E40EC5AF0010120EE0BF0AB51D9266B
:10247800AC51DA22200EDF6E8EC10EF08FC10FF044
:10248800ABC110F0ACC111F0126A136A146A156A74
:1024980072EC5DF01C0E0101AB250A6E000EAC213A
:1024A8000B6E0C6A0D6A0E6A0F6A40EC5AF0010155
:1024B80020EE03F08E51D9268F51DA22010EDF6EFD
:1024C8007E517F118011811167E020EE2BF08E5133
:1024D800D9268F51DA22DECF82F1DECF83F1DECF2B
:1024E80084F1DECF85F1910E00016E6F010E6F6FE2
:1024F8007EC170F07FC171F080C172F081C173F04C
:10250800746B756B766B776B5BEC41F00101906FC8
:10251800905142E18EC136F08FC137F082C138F058
:1025280083C139F084C13AF085C13BF05EEC54F0C8
:102538000101906FFF0E7E250001BE6FFF0E0101A5
:102548007F210001BF6FFF0E010180210001C06FD4
:10255800FF0E010181210001C16F010120EE0BF086
:102568008E51D9268F51DA22BEC0DEFFBFC0DEFFF2
:10257800C0C0DEFFC1C0DEFF0FD0010190510CE1E9
:1025880095A902D0040E07D00001BDA305D0010112
:1025980095A102D0070E906F0101905123E100012F
:1025A800BDB7BD8D010120EE2BF08E51D9268F517C
:1025B800DA22000110EE1CF0B951E126BA51E222EC
:1025C800DECFE6FFDECFE6FFDECFE6FFDECFE6FFBB
:1025D80020EE20F0B951D926BA51DA22ABC1DEFF7C
:1025E800ACC1DDFF0101905101E080D18EC111F035
:1025F8008FC112F0ABC113F0ACC114F029EC59F043
:10260800000120EE06F0B951D926BA51DA2211C0DC
:10261800DEFF12C0DEFF13C0DEFF14C0DEFF1C0E9B
:102628000101AB250A6E000EAC210B6E1BEC53F0BA
:10263800000120EE0AF0B951D926BA51DA220AC0AF
:10264800DEFF0BC0DEFF0CC0DEFF0DC0DEFFB9C031
:10265800D9FFBAC0DAFF8EC1DEFF8FC1DDFF0101ED
:1026680020EE05F08E51D9268F51DA22000110EEA6
:1026780002F0B951E126BA51E222DECFE6FFDDCF02
:10268800E5FF20EE0EF0B951D926BA51DA22BDC0C5
:10269800DFFF20EE0FF0B951D926BA51DA22DF6AEE
:1026A80020EE18F0B951D926BA51DA22DE6ADE6A6C
:1026B800DE6ADD6A20EE10F0B951D926BA51DA2265
:1026C800DE6ADE6ADE6ADD6ABDAB10D120EE0AF092
:1026D800B951D926BA51DA22DE50DE10DE10DE10EA
:1026E80001E104D120EE0AF0B951D926BA51DA2213
:1026F80010EE10F0B951E126BA51E222DECFE6FF22
:10270800DECFE6FFDECFE6FFDECFE6FF010120EEFB
:1027180009F08E51D9268F51DA22DECFBEF0DDCFF7
:10272800BFF00001BE51C06FBF51C16FC26BC36B18
:10273800090ED890C037C137C237C337E82EF9D74A
:10274800C0C07AF1C1C07BF1C2C07CF1C3C07DF1C9
:1027580020EE06F0B951D926BA51DA22DECF8AF135
:10276800DECF8BF1DECF8CF1DECF8DF120EE0AF0DB
:10277800B951D926BA51DA22DECF86F1DECF87F1F8
:10278800DECF88F1DECF89F132D0B9C041F0BAC0CE
:1027980042F08AC143F08BC144F08CC145F08DC131
:1027A80046F026EC2FF041C08AF142C08BF143C0BD
:1027B8008CF144C08DF101018D518C118B1105E113
:1027C800020E8A5D02E2020E906F8A2908E18B29C7
:1027D80006E18C2904E18D2902E1010E906F7A51FE
:1027E800865F7B51875B7C51885B7D51895B0101EA
:1027F800905109E186517A5D87517B5988517C59FE
:1028080089517D59C2E3000120EE14F0B951D9264F
:10281800BA51DA228AC1DEFF8BC1DEFF8CC1DEFF2E
:102828008DC1DEFF0101905161E186510001BE6F4B
:10283800010E010187150001BF6FC06BC16BBE118E
:10284800C011C11153E08EC10AF08FC10BF08AC1CB
:102858000CF08BC10DF08CC10EF08DC10FF036EC71
:102868004AF00AC082F10BC083F10CC084F10DC09C
:1028780085F10101825183118411851103E1020E52
:10288800906F34D086C1BEF087C1BFF088C1C0F058
:1028980089C1C1F00A0E06D00001D890C133C033F7
:1028A800BF33BE33E82EF8D7010182510001BE259F
:1028B800C26F010183510001BF21C36F010184511F
:1028C8000001C021C46F010185510001C121C56FFC
:1028D80020EE18F0B951D926BA51DA22C2C0DEFF6B
:1028E800C3C0DEFFC4C0DEFFC5C0DEFF01019051DA
:1028F80006E0B9C0D9FFBAC0DAFFDE6ADD6A9051D6
:10290800120019C0F6FF1AC0F7FFF86A0800F5CFE1
:102918009CF0194A1A2A00019C5101E11200250E67
:102928009C190AE017C00BF018C00CF09CC00DF001
:102938000E6AFDEC5FF0E5D7946B956B926B936B29
:10294800200E836F9669976919C0F6FF1AC0F7FFC2
:10295800F86A0800F5CF9CF0194A1A2A300E9C191B
:102968000DE1300E836F19C0F6FF1AC0F7FFF86A41
:102978000800F5CF9CF0194A1A2A07D02D0E9C1989
:1029880004E1936B020E926FEED72A0E9C1945E173
:102998001B50D96EDA6A020EDF26DF5CD96EDA6A5E
:1029A800DECF8AF0DECF8BF08BAF0BD08A510008D8
:1029B8008A6F8B51D8A0E82A00088B6F936B020EA0
:1029C800926F8AC094F08BC095F019C0F6FF1AC0B8
:1029D800F7FFF86A0800F5CF9CF0194A1A2A23D0A5
:1029E8000A0E9403F3CF1CF0F4CF1DF09503F350B7
:1029F8001D269C511C26000E1D22D00E1C24946FEF
:102A0800FF0E1D20956F19C0F6FF1AC0F7FFF86A70
:102A18000800F5CF9CF0194A1A2A2F0E9C6503D09E
:102A2800390E9C65DDD72E0E9C194AE119C0F6FFB8
:102A38001AC0F7FFF86A0800F5CF9CF0194A1A2A5D
:102A48002A0E9C1917E11B50D96EDA6A020EDF268E
:102A5800DF5CD96EDA6ADECF96F0DECF97F019C068
:102A6800F6FF1AC0F7FFF86A0800F5CF9CF0194A7C
:102A78001A2A26D0966B976B1DD00A0E9603F3CFB1
:102A88001CF0F4CF1DF09703F3501D269C511C2613
:102A9800000E1D22D00E1C24966FFF0E1D20976F6E
:102AA80019C0F6FF1AC0F7FFF86A0800F5CF9CF0C6
:102AB800194A1A2A2F0E9C6503D0390E9C65DDD75A
:102AC8006C0E9C190BE1928519C0F6FF1AC0F7FF2E
:102AD800F86A0800F5CF9CF0194A1A2A9C5101E0BF
:102AE800ADD01200856B020E08D0856B080E05D09C
:102AF800856B0A0E02D0856B100E846FBFD017C08D
:102B08000BF018C00CF01B50D96EDA6ADF50DF2AC0
:102B1800DF2AD96EDA6ADF500D6E0E6AFDEC5FF0BF
:102B2800F0D61B50D96EDA6A020EDF26DF5CD96E4A
:102B3800DA6ADECF90F0DECF91F09051911104E186
:102B48002C0E906FF90E916F90C00AF091C00BF0A7
:102B580011EC5DF00AC098F00BC099F0000197BF26
:102B680016D09851965D9951975911E296C098F0F0
:102B780097C099F00CD017C00BF018C00CF083C0A8
:102B88000DF00E6AFDEC5FF00001984B992B92B3A3
:102B980022D09451985D955199591DE2ECD717C0F0
:102BA8000BF018C00CF090C0F6FF91C0F7FF000EB4
:102BB800F86E0E0EF76403D00800F55005D0F6CF76
:102BC800E9FFF7CFEAFFEF500D6E0E6AFDEC5FF0FC
:102BD8000001904B912B90C0F6FF91C0F7FF000EBB
:102BE800F86E0E0EF76403D00800F55005D0F6CF46
:102BF800E9FFF7CFEAFFEF50000912E0000196075E
:102C0800D8A097079629CBE197290AE0C8D717C01B
:102C18000BF018C00CF00E6A200E0D6EFDEC5FF084
:102C2800000198511C6E99511D6E984B992B945127
:102C38001C5C95511D5801E364D6E9D79C511C6E64
:102C48001D6A1D5001E06ED61C50580A01E153D789
:102C58003A0A01E147D7010A01E151D7070A01E120
:102C680047D70B0A01E141D71C0A01E15AD7060AE6
:102C780001E13ED70D0A01E13ED754D692A511D005
:102C88001B50D96EDA6A040EDF26DF5CD96EDA6A69
:102C9800DECF8CF0DECF8DF0DECF8EF0DECF8FF082
:102CA80027D0640E9C1913E01B50D96EDA6ADF50E6
:102CB800DF2ADF2AD96EDA6ADECF1CF0DDCF1DF0FD
:102CC8001CC08CF01DC08DF08E6B8F6B11D01B500B
:102CD800D96EDA6ADF50DF2ADF2AD96EDA6ADECFE8
:102CE8008CF0DDCF8DF0000E8DBFFF0E8E6F8F6FD5
:102CF800640E9C190CE18FAF0AD08C6D8D1FD8B073
:102D08008D2B8E1FD8B08E2B000E8F5792819A6B09
:102D18009B6B8CC086F08DC087F08EC088F08FC00A
:102D280089F086C00AF087C00BF088C00CF089C013
:102D38000DF084C00EF085C00FF0106A116AA9EC7E
:102D48005AF00A500001826F86C00AF087C00BF063
:102D580088C00CF089C00DF084C00EF085C00FF05B
:102D6800106A116AB4EC58F00AC086F00BC087F0FC
:102D78000CC088F00DC089F0090E000182650BD0E7
:102D8800780E9C1903E0816B070E02D0816B270E29
:102D9800806F805182279A51600FD96EDA6A82510A
:102DA800300FDF6E9A4B9B2B865187118811891142
:102DB80005E09B5103E1200E9A5DB3E392A108D090
:102DC8009A51600FD96EDA6A2D0EDF6E9A4B9B2BE3
:102DD8009AC098F09BC099F00CD017C00BF018C09F
:102DE8000CF083C00DF00E6AFDEC5FF00001984B0B
:102DF800992B92B305D09451985D95519959EDE36B
:102E080017C00BF018C00CF09A07D8A09B079A516E
:102E1800600FD96EDA6ADF500D6E0E6AFDEC5FF056
:102E280000019A519B110AE0EBD717C00BF018C0AC
:102E38000CF00E6A200E0D6EFDEC5FF0000198514B
:102E48001C6E99511D6E984B992B94511C5C955191
:102E58001D5801E356D5E9D7256E1F50100B236E78
:102E6800205002E053EC51F0246A235001E129D2AA
:102E7800259E040E251803E10001FE5103E1140EFE
:102E8800251807E10101406B416B206A070E1F6E90
:102E9800070C3F0E251808E10001FE6B0101406B8D
:102EA800416B1F6A206A12005F0E251807E10101B5
:102EB800546B406B416B1F6A206A12003F0E2564F9
:102EC8000BD05F0E256008D00101E051251804E001
:102ED800546B1F6A206A12000101E05125180AE1AB
:102EE800010E546F0001FE6B0101406B416B1F6ABC
:102EF800206A1200E151251801E0E3D1010E00011A
:102F0800FE6FF2D7600E25180CE10101545109E05B
:102F18005251080ED8B4030E246E0101406B416B68
:102F280038D2600E25180AE10001FE5107E00101C0
:102F3800525102E0090EF0D7050EEED7680E25189B
:102F48000AE10001FE5107E01A0E0101416F900EDF
:102F580062D183801ED2680E251805E10101545103
:102F680002E0020ED9D76A0E251808E10001FE51C9
:102F780005E01A0E0101416FF40E4DD16C0E2518B3
:102F880008E10001FE5105E01A0E0101416F2C0E07
:102F980042D1700E251808E10101545105E0040ED4
:102FA800246E406B416BD5D7700E251801E0F1D126
:102FB8000001FE5101E1EDD11B0E0101416F620ECE
:102FC8002AD1838025500CE11FAA05D0246A01016B
:102FD800406B416B83901A0E0101416FAF0E406F39
:102FE800020E251805E11A0E0101416F920E406F7D
:102FF800050E251805E11A0E0101416FAE0E406F4E
:10300800070E251805E11A0E0101416FB80E406F31
:10301800080E251805E11A0E0101416FCC0E406F0C
:10302800030E251802E025280CE18380680E216E26
:10303800E40EE82EFED7212EFCD700D0246A839018
:103048006CD7140E251805E11A0E0101416F9E0E6A
:10305800406F160E251801E09CD11A0E0101416F30
:10306800A40ECAD0050E251805E11A0E0101416FFC
:10307800F50E406F080E251801E08BD11A0E0101DC
:10308800416FCC0E406F010E526F83D125C05AF0AC
:103098001A0E0101416F950EAFD02550226E216A9C
:1030A8005A500C0D000EF324D96E010EF420DA6E7E
:1030B80021C0DEFF22C0DDFF1A0E0101416F960E0E
:1030C8009BD02550216E226A5A500C0D000EF32415
:1030D800D96E010EF420DA6E21C0DEFF22C0DDFFBA
:1030E8001A0E0101416F970E87D05A500C0D020E2F
:1030F800F324D96E010EF420DA6E25C0DFFF1A0E14
:103108000101416F980E78D05A500C0D030EF3242C
:10311800D96E010EF420DA6E25C0DFFF0101406B85
:10312800416B010E37D01A0E0101416FB90E73D0F1
:103138001A0E0101416FBA0E5FD01A0E0101416FDC
:10314800BB0E406F350E00019D6FFE0E9E6F4FEC5B
:1031580060F00101536B406B416B55D00101406B2E
:10316800416B350E00019D6FFE0E9E6F4FEC60F0B7
:103178004AD00E0E00019D6FFF0E9E6F4FEC60F05F
:103188000101406B416B010E506F3DD00101406B56
:10319800416B060E246EFDD025C05AF00101406B2C
:1031A800416B246A30D00101526B1A0E416FF70E41
:1031B800406F29D01A0E0101416FF70E1DD0839080
:1031C800270E0101416F0F0E17D0180E251801E0C8
:1031D800E0D01A0E0101416F2D0E0ED01A0E01011A
:1031E800416F2E0E09D01A0E0101416F2F0E04D027
:1031F8001A0E0101416F300E406FCBD00101406BB8
:10320800416B0A0E246E8390C4D0040E246E270EE0
:103218000101416F0F0E406F9CD68380010104D0DD
:103228008390010E0101526F406B416B246AB1D04B
:103238008390010E0101526F406B416B246A5A5012
:103248000C0D000EF324D96E010EF420DA6EDE6A3E
:10325800DD6A5A500C0D020EF324D96E010EF420CB
:10326800DA6E2544E846030BDF6E5A500C0D030E48
:10327800F324D96E010EF420DA6E25503F0BDF6E71
:103288009E0E00019D6FFC0E9E6F25C09FF0A06BE7
:103298005A500C0D020EF324D96E010EF420DA6E8A
:1032A800DF50A16FA26B5A500C0D030EF324D96E98
:1032B800010EF420DA6EDF50A36FA46B4FEC60F0C0
:1032C80068D040C121F041C122F0225007E01A0A1B
:1032D80009E0010A54E03C0A5AE05BD0215001E1C0
:1032E80011D657D021502C0A01E16FD7010A01E10C
:1032F80075D7030A01E177D7010A01E179D71F0AD7
:1033080001E17CD7A00A01E15CD6020A01E1BED640
:10331800070A01E1C2D6030A01E1D3D6010A01E195
:10332800E4D60F0A01E1F0D6060A01E122D73A0AEB
:1033380001E12CD70A0A01E173D7010A01E178D724
:10334800170A01E1F0D6010A01E1F2D6030A01E108
:10335800F4D6010A01E102D7790A01E102D60E0A80
:1033680001E11AD7380A01E17DD6010A01E11BD72C
:10337800030A01E11FD7010A01E121D70AD0215030
:10338800580A01E142D73A0A01E147D702D0215051
:103398000F0A24C01FF0206A120051C081F052C0E9
:1033A80082F055C0D9FF56C0DAFFDE6ADD6A4FC029
:1033B8000BF050C00CF08D0E0D6EC5EC52F00001F4
:1033C8007C6F7C510AE120EE0FF04F50D926505007
:1033D800DA22DF507C6F7C5102E07C51120020EE33
:1033E8000EF04F50D9265050DA22DFA0070C20EEFD
:1033F80010F04F50D9265050DA22DECF6CF0DECFD5
:103408006DF0DECF6EF0DECF6FF020EE0AF04F5099
:10341800D9265050DA22DECF70F0DECF71F0DECF41
:1034280072F0DECF73F06C51705D786F6D51715929
:10343800796F6E5172597A6F6F5173597B6F535010
:103448006C6F54506D6F6E6B6F6B6C51785D6D5116
:1034580079596E517A596F517B5901E31AD278C064
:1034680053F079C054F015D220EE10F04F50D92601
:103478005050DA22FF0EDE146C6F010EDE146D6FF1
:10348800000EDE146E6F000EDE146F6F6C516D113E
:103498006E116F1101E083D120EE10F04F50D92644
:1034A8005050DA22DECF6CF0DECF6DF0DECF6EF05A
:1034B800DECF6FF00A0E05D0D8906F336E336D33C0
:1034C8006C33E82EF9D720EE09F08D51D9268E51AC
:1034D800DA22DECF70F0DDCF71F0FF0E7025726F4B
:1034E800FF0E7121736F6C517215836F6D517315D7
:1034F800846F831166E120EE10F04F50D9265050AA
:10350800DA22DE50DE10DE10DE100FE120EE06F0CB
:103518004F50D9265050DA22DECF7DF0DECF7EF034
:10352800DECF7FF0DECF80F01CD04FC041F050C01E
:1035380042F020EE14F04F50D9265050DA22DECF58
:1035480043F0DECF44F0DECF45F0DECF46F026EC88
:103558002FF041C07DF042C07EF043C07FF044C0F0
:1035680080F0000180517F117E110CE1020E7D5D1B
:1035780009E220EE0FF04F50D9265050DA22020E01
:10358800DF6E020C7D290FE17E290DE17F290BE119
:10359800802909E120EE0FF04F50D9265050DA2249
:1035A800010EDF6E010C20EE14F04F50D92650505A
:1035B800DA227DC0DEFF7EC0DEFF7FC0DEFF80C076
:1035C800DEFF8DC00AF08EC00BF020EE14F04F50D5
:1035D800D9265050DA22DECF0CF0DECF0DF0DECF48
:1035E8000EF0DECF0FF036EC4AF00AC085F00BC0C3
:1035F80086F00CC087F00DC088F000018551861157
:103608008711881101E1B5D7835185278451862315
:10361800000E8723882353C06CF054C06DF0090E48
:103628006E6FD8906D336C336E2FFBD76CC089F0FA
:103638006DC08AF089518A1101E1A3D0895183258F
:103648006C6F8A5184216D6F20EE09F08D51D92657
:103658008E51DA226C51DE5C6D51DE5810E220EE9C
:1036680009F08D51D9268E51DA22DECF6CF0DDCFEC
:103678006DF083516C5D896F84516D598A6F81C07B
:1036880019F082C01AF085C01BF086C01CF087C0F4
:103698001DF088C01EF089C01FF08AC020F020EEFF
:1036A80001F08D51D9268E51DA22DF506FEC53F09C
:1036B800000901E06FD7000120EE03F08D51D926F3
:1036C8008E51DA22DF504EE089516C6F8A516D6F4E
:1036D8006E6B6F6B20EE2BF08D51D9268E51DA224E
:1036E800DECF70F0DECF71F0DECF72F0DECF73F098
:1036F8008551705D746F86517159756F8751725914
:10370800766F88517359776F6C51745D6D51755927
:103718006E5176596F51775925E220EE2BF08D5175
:10372800D9268E51DA22DECF6CF0DDCF6DF08551CF
:103738006C5F86516D5B090ED8906C376D37E82E3B
:10374800FBD76C5181250A6E6D5182210B6E2F0EAD
:103758008D250C6E000E8E210D6E020E0F6E0E6AF8
:10376800F0EC5CF089C06CF08AC06DF0090ED8905E
:103778006C376D37E82EFBD76CC08BF06DC08CF0C2
:103788006BD020EE18F04F50D9265050DA2285C061
:10379800DEFF86C0DEFF87C0DEFF88C0DEFF20EECA
:1037A80010F04F50D9265050DA22DECF6CF0DDCF22
:1037B8006DF06C516E6F010E6D156F6F6E510008D4
:1037C8008B6F6F51D8A0E82A02088C6F8B51535C1D
:1037D8008C51545804E253C08BF054C08CF08DC007
:1037E80036F08EC037F020EE18F04F50D9265050E2
:1037F800DA22DECF38F0DECF39F0DECF3AF0DECF96
:103808003BF05EEC54F0000901E0C4D681C00AF038
:1038180082C00BF020EE10F04F50D9265050DA221B
:10382800DECF6CF0DDCF6DF000016C516E6F010ED4
:103838006D156F6F6E518D25706F6F518E21716F81
:103848002F0E70250C6E000E71210D6E8BC00EF0C0
:103858008CC00FF0F0EC5CF08B51535E8C51545AD5
:1038680055C0D9FF56C0DAFF8B51DE268C51DD22B8
:103878008B5181278C51822320EE10F04F50D9268E
:103888005050DA228B51DE268C51DE22000EDE22C9
:10389800DE225350541001E0E7D5000C690EF66E95
:1038A800F80EF76E000EF86E0900F5CFE6F00A0084
:1038B800F5CFE7F00001EA6BED6B0101ED6BDE512E
:1038C800ECEC5FF0CD6ACE6A0FD1EE6B2F0E136E63
:1038D800070E146EE60E156E8BEC55F013C0EBF068
:1038E80014C0ECF0EBC0D9FFECC0DAFF3B0EDE18D9
:1038F80001E0F5D0F9D0EE5113E1EBC00EF0ECC0C9
:103908000FF09CEC59F00001ED6F800EED6503D0CF
:10391800ED51800FEA6F030EEA65D5D0EA6BD3D07C
:10392800EE0511E10101F8510001ED1903E07F0EE8
:10393800ED1909E1EBC00EF0ECC00FF09CEC59F06A
:1039480001015F6FC0D0020EEE1911E10101F851BB
:103958000001ED1903E07F0EED1909E1EBC00EF04F
:10396800ECC00FF09CEC59F001015E6FACD0020E78
:10397800EE652CD0080EEE6129D00101F851000146
:10398800ED190CE07F0EED1909E0810EED1906E046
:10399800820EED1903E0830EED1918E1EA51050DC9
:1039A800AC0EF324E86F020EF420E96FEBC00EF0C2
:1039B800ECC00FF09CEC59F00001C36FEE51E82504
:1039C800C46F000EE921C56FFD0E5DD0070EEE65D0
:1039D8002CD01B0EEE6129D00101F8510001ED1920
:1039E8000CE07F0EED1909E0810EED1906E0820E5C
:1039F800ED1903E0830EED1918E1EA51130DAA0E33
:103A0800F324E86F030EF420E96FEBC00EF0ECC06E
:103A18000FF09CEC59F00001C36FEE51E825C46F1C
:103A2800000EE921C56FF80E2ED01A0EEE6533D0C0
:103A3800280EEE6130D00101F8510001ED190CE0BB
:103A48007F0EED1909E0810EED1906E0820EED19E1
:103A580003E0830EED191FE1EA510D0D780EF324F2
:103A6800E86F020EF420E96FEBC00EF0ECC00FF027
:103A78009CEC59F00001C36FEE51E825C46F000EAD
:103A8800E921C56FE50EC425D96EFF0EC521DA6E92
:103A9800C3C0DFFF18D0280EEE1915E10101F85157
:103AA8000001ED1903E07F0EED190DE1ED0E0A6E30
:103AB800010E0B6EEBC00CF0ECC00DF00F6A080E97
:103AC8000E6E91EC5BF00001EE2B136A146AE60EA1
:103AD800156E8BEC55F013C0EBF014C0ECF0000140
:103AE800EB51EC1101E007D72F0E00018F6F070E85
:103AF800906F926B910E916F000E936F030E946FFF
:103B0800ACEC54F08F51901101E0DFD6EE6BEE5122
:103B18000D0D820EF324D96E020EF420DA6EDF50FA
:103B2800C36FC3C0C4F0C56BC66BC76BC6C0C7F054
:103B3800C5C0C6F0C4C0C5F0C46BEE510D0D810EF2
:103B4800F324D96E020EF420DA6EDF50C86FC8C0B5
:103B5800C9F0CA6BCB6BCC6BCAC0CCF0C9C0CBF078
:103B6800CA6BC96BEE510D0D800EF324D96E020E8F
:103B7800F420DA6EDF50CD6FCDC0CEF0CF6BD06BB6
:103B8800D16BCEC0D1F0D06BCF6BCE6BC951CE25E7
:103B9800D26FCA51CF21D36FCB51D021D46FCC5122
:103BA800D121D56FC451D225D66FC551D321D76F36
:103BB800C651D421D86FC751D521D96FEE510D0DFB
:103BC800830EF324D96E020EF420DA6EDF50D62568
:103BD800DA6F000ED721DB6F000ED821DC6F000EE4
:103BE800D921DD6FDAC0DEF0DBC0DFF0DCC0E0F049
:103BF800DDC0E1F0E26BE1BFE269E2C0E3F0E2C000
:103C0800E4F0E2C0E5F0EE511E0D0F0EF324D96E7C
:103C1800020EF420DA6EDEC0DEFFDFC0DEFFE0C099
:103C2800DEFFE1C0DEFFE2C0DEFFE3C0DEFFE4C08E
:103C3800DEFFE5C0DEFFEE51130DAE0EF324D96EA4
:103C4800030EF420DA6EDF50C46FC36BEE51130D10
:103C5800AF0EF324D96E030EF420DA6EDF50C325BD
:103C6800C56F000EC421C66FEE511E0D1C0EF32445
:103C7800D96E020EF420DA6EC5C0DEFFC6C0DDFFC5
:103C8800EE511E0D1C0EF324D96E020EF420DA6ECE
:103C9800DECFC3F0DDCFC4F0C3C00AF0C4C00BF060
:103CA8000C6A0D6A0E6A0F6A106A116AEE511E0DCF
:103CB8000F0EF324D96E020EF420DA6EDECFC5F0B3
:103CC800DECFC6F0DECFC7F0DECFC8F0DECFC9F05A
:103CD800DECFCAF0DECFCBF0DECFCCF0C5C012F01D
:103CE800C6C013F0C7C014F0C8C015F0C9C016F09C
:103CF800CAC017F0CBC018F0CCC019F063EC56F06E
:103D08000AC0CDF00BC0CEF00CC0CFF00DC0D0F083
:103D18000EC0D1F00FC0D2F010C0D3F011C0D4F053
:103D28000001EE511E0D0F0EF324D96E020EF42081
:103D3800DA6ECDC0DEFFCEC0DEFFCFC0DEFFD0C062
:103D4800DEFFD1C0DEFFD2C0DEFFD3C0DEFFD4C0AD
:103D5800DEFF600E9D6FFA0E9E6FEEC09FF0A06BA7
:103D6800EE511E0D1C0EF324D96E020EF420DA6EED
:103D7800DECFA1F0DDCFA2F04FEC60F0EE2B030E0A
:103D8800EE65C5D6E70E9D6FFA0E9E6FED0E9F6F1E
:103D9800010EA06F4FEF60F0838E8380020E93ECCC
:103DA80060F0DDEC3CF00101846F845118E05A505A
:103DB8001E0D1B0EF324D96E020EF420DA6E5A5033
:103DC8001E0D1B0EF324E16E020EF420E26EE75086
:103DD8000409DF6EA0EC5FF00101845112005A5112
:103DE80050E0385139113A113B114BE05A5049E132
:103DF8005A501E0D070EF324D96E020EF420DA6E07
:103E080038C1E6F039C1E7F03AC1E8F00001E56BE6
:103E1800000EE525E96F010EE621EA6F000EE721A5
:103E2800EB6F000EE821EC6FED6BEE6BEF6BF06B58
:103E3800DE50E91926E1DE50EA1923E1DE50EB19DC
:103E480020E1DE50EC191DE1DE50ED191AE1DE50DB
:103E5800EE1917E1DE50EF1914E1DE50F01911E107
:103E68002F0E296E070E2A6E01015A5142EC4EF0B0
:103E78000392000EA9EC56F00392586A83905850AA
:103E880012005A501E0D170EF324D96E020EF4209C
:103E9800DA6EDE50DE10DE10DE101EE05A501E0D07
:103EA800170EF324D96E020EF420DA6EDE50DE10FF
:103EB800DE1002E1DE0410E05A501E0D170EF32446
:103EC800D96E020EF420DA6EDE280DE1DE280BE151
:103ED800DE2809E1DE2807E101017A697B697C694E
:103EE8007D69856B2FD05A501E0D170EF324D96E9D
:103EF800020EF420DA6EDECFDDF0DECFDEF0DECFAC
:103F0800DFF0DECFE0F0DEC0DDF0DFC0DEF0E0C0E5
:103F1800DFF00001E06BDDC07AF1DEC07BF1DFC0CD
:103F28007CF1E0C07DF15A501E0D170EF324D96EB6
:103F3800020EF420DA6EDECFDDF0DDCFDEF0DD51EB
:103F48000101856F866B0392806B816B826B836B3B
:103F58007E6B7F6BCAD08EA88EAA09D0D70E9D6FB4
:103F6800FE0E9E6F4FEC60F0B9D08394B9D07EC13D
:103F7800DDF07FC1DEF0000EDEBFFF0EDF6FE06F09
:103F8800FF0E01017A250001E16FFF0E01017B217F
:103F98000001E26FFF0E01017C210001E36FFF0EBB
:103FA80001017D210001E46FDD51E1190EE1DE51CF
:103FB800E2190BE1DF51E31908E1E051E41905E1E9
:103FC80001018551861101E103825A50220D000E2C
:103FD800F3244F6E030EF420506E2F0E516E070E11
:103FE800526E010E546E536A870E556E010E566E50
:103FF800D1EC19F00101896F895101E0D8D68751B8
:10400800881101E1D4D68EA88EAA08D0E20E00014C
:104018009D6FFE0E9E6F4FEC60F060D08751A9EC4B
:1040280056F08EB808D0E20E00019D6FFE0E9E6F0E
:104038004FEC60F053D001018751802788518123CC
:10404800000E822383235A501E0D070EF324D96EC7
:10405800020EF420DA6E000EDE240001DD6F010E80
:10406800DE20DE6F000EDE20DF6F000EDE20E06F48
:10407800000EDE20E16F000EDE20E26F000EDE2073
:10408800E36F000EDE20E46F5A501E0D070EF32476
:10409800D96E020EF420DA6EDDC0DEFFDEC0DEFF70
:1040A800DFC0DEFFE0C0DEFFE1C0DEFFE2C0DEFF12
:1040B800E3C0DEFFE4C0DEFF8EA88EAA07D0ED0EB7
:1040C8009D6FFE0E9E6F4FEC60F008D08EBC0AD03C
:1040D800220E9D6FFF0E9E6F4FEC60F0586A45D719
:1040E800839086D001017E4B7F2B7EC1DDF07FC19E
:1040F800DEF0000E0001DEBFFF0EDF6FE06F010192
:104108007A510001DD5D01017B510001DE59010199
:104118007C510001DF5901017D510001E05901E2A4
:104128001AD701018551861160E05A50220D000E00
:10413800F3244F6E030EF420506E2F0E516E070EAF
:10414800526E85C153F086C154F0870E556E010E2C
:10415800566ED1EC19F00101896F895101E027D61B
:1041680003828551A9EC56F00101875180278851B7
:104178008123000E822383235A501E0D070EF32439
:10418800D96E020EF420DA6E000EDE240001DD6F17
:10419800010EDE20DE6F000EDE20DF6F000EDE2057
:1041A800E06F000EDE20E16F000EDE20E26F000EF1
:1041B800DE20E36F000EDE20E46F5A501E0D070E5E
:1041C800F324D96E020EF420DA6EDDC0DEFFDEC005
:1041D800DEFFDFC0DEFFE0C0DEFFE1C0DEFFE2C0E1
:1041E800DEFFE3C0DEFFE4C0DEFF0392586A78D743
:1041F800839E45D65A500C0D030EF324D96E010E3A
:10420800F420DA6EDF2A5A500C0D030EF324D96E0F
:10421800010EF420DA6EDF500001C36FC46B5A50F0
:104228000C0D0B0EF324D96E010EF420DA6EDF505C
:10423800C56FFF0EC525C66FC76BFF0EC723C351D9
:10424800C65DC751800AC86FC451800AC8594AE27E
:104258005A500C0D030EF324D96E010EF420DA6EB9
:10426800DF6A5A500C0D020EF324D96E010EF420A9
:10427800DA6EDF2A5A500C0D020EF324D96E010EA5
:10428800F420DA6EDF50C36FC46B5A500C0D0A0E5F
:10429800F324D96E010EF420DA6EDF50C56FFF0EDD
:1042A800C525C66FC76BFF0EC723C351C65DC7516F
:1042B800800AC86FC451800AC85914E25A500C0DBC
:1042C800020EF324D96E010EF420DA6EDF6A5A501A
:1042D8000C0D000EF324D96E010EF420DA6EDE2ADE
:1042E800000EDD225A500C0D0B0EF324D96E010E70
:1042F800F420DA6EDF50C36FC3C0C4F0C56BC66B61
:10430800C76B5A500C0D000EF324D96E010EF42021
:10431800DA6EDECFC8F0DDCFC9F0C8C0CAF0C9C0B8
:10432800CBF0000ECBBFFF0ECC6FCD6FCA51C403CC
:10433800F3CFCEF0F4CFCFF0D06BD16BC503F350F1
:10434800CF27F450D023000ED123CB51C403F35010
:10435800CF27F450D023000ED123CA51C603F350FF
:10436800D027F450D123CB51C503F350D027F450B4
:10437800D123CC51C403F350D027F450D123C751D3
:10438800CA03F350D127CB51C603F350D127CC51E0
:10439800C503F350D127CD51C403F350D1275A5048
:1043A8000C0D040EF324D96E010EF420DA6ECEC083
:1043B800DEFFCFC0DEFFD0C0DEFFD1C0DEFF5A5027
:1043C8000C0D0A0EF324D96E010EF420DA6EDF50BC
:1043D800C36FC3C0C4F0C56BC66BC76B5A500C0D16
:1043E800040EF324D96E010EF420DA6EDECFC8F085
:1043F800DECFC9F0DECFCAF0DECFCBF0CAC0CBF03B
:10440800C9C0CAF0C8C0C9F0C86BC851C403F3CF4B
:10441800CCF0F4CFCDF0CE6BCF6BC503F350CD27E6
:10442800F450CE23000ECF23C951C403F350CD2737
:10443800F450CE23000ECF23C851C603F350CE2725
:10444800F450CF23C951C503F350CE27F450CF23DE
:10445800CA51C403F350CE27F450CF23C751C80321
:10446800F350CF27C951C603F350CF27CA51C5030C
:10447800F350CF27CB51C403F350CF275A500C0D1C
:10448800040EF324D96E010EF420DA6ECCC0DEFFE0
:10449800CDC0DEFFCEC0DEFFCFC0DEFF5A500C0D10
:1044A8000B0EF324D96E010EF420DA6EDF50C36FC1
:1044B800C3C0C4F0C56BC66BC76B5A500C0D020E57
:1044C800F324D96E010EF420DA6EDF50C86FC8C02D
:1044D800C9F0CA6BCB6BCC6BCBC0CCF0CAC0CBF0ED
:1044E800C9C0CAF0C96BC951C403F3CFCDF0F4CF2A
:1044F800CEF0CF6BD06BC503F350CE27F450CF234B
:10450800000ED023CA51C403F350CE27F450CF2352
:10451800000ED023C951C603F350CF27F450D0233F
:10452800CA51C503F350CF27F450D023CB51C4034D
:10453800F350CF27F450D023C751C903F350D027E5
:10454800CA51C603F350D027CB51C503F350D02727
:10455800CC51C403F350D0275A500C0D040EF32449
:10456800D96E010EF420DA6ECD51DE26CE51DE2250
:10457800CF51DE22D051DE225A500C0D030EF32407
:10458800D96E010EF420DA6EDF50C36FC3C0C4F0D9
:10459800C56BC66BC76BC6C0C7F0C5C0C6F0C4C084
:1045A800C5F0C46B5A500C0D040EF324D96E010EDD
:1045B800F420DA6EC451DE26C551DE22C651DE2251
:1045C800C751DE225A50220D000EF3248B6F030EC2
:1045D800F4208C6F5A500C0D040EF324D96E010E82
:1045E800F420DA6EDECF8DF0DECF8EF0DECF8FF0E6
:1045F800DECF90F0EFEC0EF0546E545019E0330E0D
:104608009D6FFB0E9E6F5A500C0D040EF324D96E4D
:10461800010EF420DA6EDECF9FF0DECFA0F0DECF01
:10462800A1F0DECFA2F054C0A3F0A46B4FEC60F071
:104638000101536B12005A500C0D000EF324D96E71
:10464800010EF420DA6E5A500C0D080EF324E16EB8
:10465800010EF420E26EE6CFC5F0E5CFC6F0FF0EFE
:104668000001C525C76FFF0EC621C86FDE50C75DA4
:10467800C851800AC96FDE50800AC95948E35A50A8
:104688000C0D020EF324D96E010EF420DA6EDF5001
:10469800C36FC46B5A500C0D0A0EF324D96E010E69
:1046A800F420DA6EDF50C56FFF0EC525C66FC76BE5
:1046B800FF0EC723C351C65DC751800AC86FC451D6
:1046C800800AC85924E35A500C0D030EF324D96EFE
:1046D800010EF420DA6EDF50C36FC46B5A500C0D14
:1046E8000B0EF324D96E010EF420DA6EDF50C56F7D
:1046F800FF0EC525C66FC76BFF0EC723C351C65D26
:10470800C751800AC86FC451800AC85961E21F0E98
:104718000101516F010E536F8390530E00019D6F7D
:10472800F90E9E6F5A500C0D000EF324D96E010E2F
:10473800F420DA6EDECF9FF0DDCFA0F05A500C0DDA
:10474800080EF324D96E010EF420DA6EDECFC3F022
:10475800DDCFC4F0FF0EC325A16FFF0EC421A26FE9
:104768005A500C0D020EF324D96E010EF420DA6EA5
:10477800DF50A36FA46B5A500C0D0A0EF324D96EA8
:10478800010EF420DA6EDF50C56FFF0EC525A56F48
:10479800A66BFF0EA6235A500C0D030EF324D96EF8
:1047A800010EF420DA6EDF50A76FA86B5A500C0D7B
:1047B8000B0EF324D96E010EF420DA6EDF50C66FAB
:1047C800FF0EC625A96FAA6BFF0EAA234FEC60F057
:1047D8005A500C0D0B0EF324D96E010EF420DA6E2C
:1047E800DF50C36FC3C0C4F0C56BC66BC76B5A50EC
:1047F8000C0D000EF324D96E010EF420DA6EDECF14
:10480800C8F0DDCFC9F0C8C0CAF0C9C0CBF0000EEF
:10481800CBBFFF0ECC6FCD6FCA51C403F3CFCEF020
:10482800F4CFCFF0D06BD16BC503F350CF27F45042
:10483800D023000ED123CB51C403F350CF27F4501B
:10484800D023000ED123CA51C603F350D027F45009
:10485800D123CB51C503F350D027F450D123CC51E9
:10486800C403F350D027F450D123C751CA03F350DF
:10487800D127CB51C603F350D127CC51C503F350F0
:10488800D127CD51C403F350D127CEC0D3F0CFC028
:10489800D4F0D0C0D5F0D1C0D6F0D3C00AF0D4C07F
:1048A8000BF0D5C00CF0D6C00DF05A500C0D0A0E06
:1048B800F324D96E010EF420DA6EDF50C36FC3C043
:1048C800C4F0C56BC66BC76BC6C0C7F0C5C0C6F021
:1048D800C4C0C5F0C46BC4C00EF0C5C00FF0C6C0DC
:1048E80010F0C7C011F077EC57F00AC0D3F00BC036
:1048F800D4F00CC0D5F00DC0D6F05A500C0D0B0EEC
:10490800F324D96E010EF420DA6EDF50C36FC3C0F2
:10491800C4F0C56BC66BC76B5A500C0D020EF3245E
:10492800D96E010EF420DA6EDF50C86FC8C0C9F026
:10493800CA6BCB6BCC6BCBC0CCF0CAC0CBF0C9C0B8
:10494800CAF0C96BC951C403F3CFCDF0F4CFCEF090
:10495800CF6BD06BC503F350CE27F450CF23000E96
:10496800D023CA51C403F350CE27F450CF23000EEE
:10497800D023C951C603F350CF27F450D023CA51CE
:10498800C503F350CF27F450D023CB51C403F350C1
:10499800CF27F450D023C751C903F350D027CA51A9
:1049A800C603F350D027CB51C503F350D027CC51C1
:1049B800C403F350D027CD51D327CE51D423CF51A0
:1049C800D523D051D6235A500C0D030EF324D96E9B
:1049D800010EF420DA6EDF50C36FC3C0C4F0C56B9C
:1049E800C66BC76BC6C0C7F0C5C0C6F0C4C0C5F0AB
:1049F800C46BC451D327C551D423C651D523C7513D
:104A0800D6235A50220D000EF3248B6F030EF42088
:104A18008C6FD3C08DF0D4C08EF0D5C08FF0D6C0C7
:104A280090F0EFEC0EF0D26FD25111E0330E9D6F83
:104A3800FB0E9E6FD3C09FF0D4C0A0F0D5C0A1F0EC
:104A4800D6C0A2F0D2C0A3F0A46B4FEC60F05A50CD
:104A58000C0D040EF324D96E010EF420DA6ED3C0C7
:104A6800DEFFD4C0DEFFD5C0DEFFD6C0DEFF010109
:104A7800536B839012006EC0D9FF6FC0DAFFDECF90
:104A880085F0DDCF86F0705171117211731128E134
:104A980020EE0BF08551D9268651DA22DECF7DF043
:104AA800DECF7EF0DECF7FF0DECF80F07D517E114D
:104AB8007F1180110FE020EE13F08551D926865121
:104AC800DA22DE507D5DDE507E59DE507F59DE50A1
:104AD800805952E3010E7D6F7E6B7F6B806B4CD0EB
:104AE8006EC041F06FC042F070C043F071C044F036
:104AF80072C045F073C046F026EC2FF041C087F035
:104B080042C088F043C089F044C08AF000018A514D
:104B18008911881109E1020E875D06E2010E6E6FA8
:104B28006F6B706B716B000C87290FE188290DE1A1
:104B380089290BE18A2909E187C06EF088C06FF0E6
:104B480089C070F08AC071F0120020EE13F0855110
:104B5800D9268651DA22DE50875DDE508859DE502C
:104B68008959DE508A59E8E370C07DF071C07EF043
:104B780072C07FF073C080F020EE0FF08551D92607
:104B88008651DA22DE50DE10DE10DE1005E16E6B93
:104B98006F6B706B716B1200816B826B836B846BB4
:104BA80070517D1909E171517E1906E172517F1921
:104BB8007DE173518019D8A479D07D29816F000EC9
:104BC8007E21826F000E7F21836F000E8021846F0B
:104BD80020EE13F08551D9268651DA22DE50815D08
:104BE800DE508259DE508359DE50845905E3020EA7
:104BF800816F826B836B846B6EC041F06FC042F033
:104C080081C043F082C044F083C045F084C046F0C0
:104C180026EC2FF041C087F042C088F043C089F0ED
:104C280044C08AF000018705881189118A1184E03F
:104C3800872907E1882905E1892903E18A2901E112
:104C48007BD78751881189118A1130E020EE0BF04B
:104C58008551D9268651DA22DECF87F0DECF88F05B
:104C6800DECF89F0DECF8AF08A518911881103E1FD
:104C7800020E875D17E320EE13F08551D926865181
:104C8800DA22DE50875DDE508859DE508959DE50C1
:104C98008A5908E287C07DF088C07EF089C07FF01D
:104CA8008AC080F0816B826B836B846B8151821127
:104CB8008311841162E17DC081F07EC082F07FC0E3
:104CC80083F080C084F0812B000E82238323842309
:104CD80020EE13F08551D9268651DA22DE50815D07
:104CE800DE508259DE508359DE5084590DE3020E9E
:104CF800816F826B836B846B80517F117E1104E11D
:104D0800020E7D5D01E243D76EC041F06FC042F0F4
:104D180081C043F082C044F083C045F084C046F0AF
:104D280026EC2FF041C087F042C088F043C089F0DC
:104D380044C08AF000018751881189118A111DE049
:104D48008705881189118A1101E1F6D6872907E1BB
:104D5800882905E1892903E18A2901E1EDD67D51F8
:104D68008119B1E17E518219AEE17F518319ABE11E
:104D78008051841901E10BD7A6D785C041F086C0C0
:104D880042F081C043F082C044F083C045F084C043
:104D980046F04768486849684A686DEC2BF000019E
:104DA8007C6F7C511DE1705171117211731118E003
:104DB80085C041F086C042F070C043F071C044F035
:104DC80072C045F073C046F081C047F082C048F019
:104DD80083C049F084C04AF06DEC2BF000017C6F71
:104DE8007C5143E120EE0BF08551D9268651DA2219
:104DF80081C0DEFF82C0DEFF83C0DEFF84C0DEFF2D
:104E080020EE0FF08551D9268651DA2210EE13F0E4
:104E18008551E1268651E222FE0EE624786FFF0EC8
:104E2800E620796FFF0EE6207A6FFF0EE6207B6F93
:104E3800DE50785DDE507959DE507A59DE507B5964
:104E48000BE320EE0FF08551D9268651DA22DE06D3
:104E5800000EDE5ADE5ADE5A20EE04F08551D926BD
:104E68008651DA22000EDB800DD07C0507E0010EAA
:104E7800816F000E826B836B846B04D081698269B9
:104E88008369846981C06EF082C06FF083C070F05E
:104E980084C071F01200000E4F6E030E506E2F0E7C
:104EA800516E070E526E020E546E536AF40E556E12
:104EB800566AD1EC19F00101606F740E00019D6F04
:104EC800FD0E9E6FF4C09FF0F5C0A0F04FEC60F0AF
:104ED800F66BF76BF26BF36BF86BF96BF851D40F59
:104EE800D96EDA6ADF6AF851E30FD96EDA6ADF6AD7
:104EF800F84BF92BF9BFF2D7F95103E10F0EF85D22
:104F0800EDE3FA6BFB6B54D12F0EFA25D96E070E21
:104F1800FB21DA6E0D0EDE1801E00FD19A0E0A6E33
:104F2800FF0E0B6ED40E0C6EF7EC54F00A500B10FB
:104F380007E1E30E0A6E6AEC52F00A500101F76FBE
:104F4800940E0A6EFF0E0B6ED40E0C6EF7EC54F036
:104F58000A500B1007E1E30E0A6E6AEC52F00A5091
:104F68000101626F790E0A6EFF0E0B6ED40E0C6E85
:104F7800F7EC54F00A500B1007E1E30E0A6E6AECE6
:104F880052F00A5001015C6FD70E0A6EFF0E0B6ECD
:104F9800D40E0C6EF7EC54F00A500B1007E1E30E38
:104FA8000A6E6AEC52F00A5001015A6FDF0E0A6E5F
:104FB800FF0E0B6ED40E0C6EF7EC54F00A500B106B
:104FC80007E1E30E0A6E6AEC52F00A500101DE6F47
:104FD800DB0E0A6EFF0E0B6ED40E0C6EF7EC54F05F
:104FE8000A500B1008E1E30E0A6E6AEC52F00AC090
:104FF8004CF10BC04DF1AB0E0A6EFF0E0B6ED40ECA
:105008000C6EF7EC54F00A500B1007E1E30E0A6E31
:105018006AEC52F00A500101616F0001FC6BFD6BF4
:10502800C50E1E6E1F6A800E206EFF0E216EFCC01C
:1050380022F0FDC023F0C9EC5EF0C50E0A6E0B6AC3
:10504800D40E0C6EF7EC54F00A500B1018E10F0E4A
:105058000001FC03F3CFC3F0F4CFC4F0FD03F35019
:10506800C4272F0EC3250A6E090EC4210B6EE30E4A
:105078000C6E0D6A0F6A0F0E0E6E91EC5BF000015C
:10508800FC4BFD2BFDBFCCD7FD5103E1100EFC5DA1
:10509800C7E3FD6B010EFC6FC50E1E6E1F6A870EFF
:1050A800206EFF0E216EFCC022F0FDC023F0C9EC7B
:1050B8005EF0C50E0A6E0B6AD40E0C6EF7EC54F057
:1050C8000A500B1018E10F0E0001FC03F3CFC3F0D8
:1050D800F4CFC4F0FD03F350C4271F0EC3250A6E96
:1050E8000A0EC4210B6EE30E0C6E0D6A0F6A0F0ECA
:1050F8000E6E91EC5BF00001FC4BFD2BFDBFCCD795
:10510800FD5103E1040EFC5DC7E3F86BF96BF85140
:10511800D40FD96EDA6ADF6AF851E30FD96EDA6A0A
:10512800DF6AF84BF92BF9BFF2D7F95103E10F0EFB
:10513800F85DEDE3F26BF36B15D02F0EFA25D96EFF
:10514800070EFB21DA6E0A0EDE1830E02F0EFA2564
:10515800D96E070EFB21DA6E200EDE1806E1F36B1E
:10516800010EF26FF66BF76B21D0F251F31109E0E3
:105178002F0EFA25D96E070EFB21DA6EF651E30FD2
:1051880008D02F0EFA25D96E070EFB21DA6EF651DC
:10519800D40FE16EE26ADFCFE7FFF7BF05D0F75122
:1051A80005E10F0EF65D02E2F64BF72BFA4BFB2BEF
:1051B800F451FA5DF551FB5901E2A6D6640E9D6FD4
:1051C800FD0E9E6F5CC19FF0A06B4FEC60F0DE0E91
:1051D8009D6FFD0E9E6FF7C19FF0A06B4FEC60F0C6
:1051E800C00E9D6FFD0E9E6F62C19FF0A06B4FECCD
:1051F80060F0CF0E9D6FFD0E9E6FDEC19FF0A06B1D
:105208004FEC60F0430E9D6FFC0E9E6F4CC19FF0FB
:105218004DC1A0F04FEC60F0FC6BFD6BD10E9D6FA3
:10522800FC0E9E6FFCC09FF0FDC0A0F00F0EFC03AB
:10523800F3CFC3F0F4CFC4F0FD03F350C4272F0E0F
:10524800C325A16F090EC421A26F4FEC60F0FC4B7F
:10525800FD2BFDBFE3D7FD5103E1100EFC5DDEE33E
:10526800FB6B010EFA6FE20E9D6FFC0E9E6FFAC08B
:105278009FF0FBC0A0F00F0EFA03F3CFC3F0F4CFFA
:10528800C4F0FB03F350C4271F0EC325A16F0A0EF9
:10529800C421A26F4FEC60F0FA4BFB2BFBBFE3D7A6
:1052A800FB5103E1040EFA5DDEE32A0E9D6FF90E51
:1052B8009E6F4FEF60F0276E1AC03EF01BC03FF0A4
:1052C800275001E0040C010E3C6E5CB0030CE4D1E5
:1052D80043EC60F0000901E1F8D13C6AF6D1136AA9
:1052E800146A156A166A090E42EC5EF0000901E0BC
:1052F800ECD1280E0A6E0B6A0D6A100E0C6E0AECC1
:105308005BF0000901E1E1D12844E846030BE80617
:1053180047E12FC01CF03F0E1C161CC01DF01E6A72
:105328001F6A206A1EC020F01DC01FF01E6A1D6A79
:105338003050226E3150216E21501D24236E225090
:105348001E20246E000E1F20256E000E2020266EC3
:105358002328386E000E2420396E000E25203A6E60
:10536800000E26203B6E38C01CF039C01DF03AC034
:105378001EF03BC01FF00A0ED8901C361D361E3694
:105388001F36E82EF9D71AC0D9FF1BC0DAFF1CC098
:10539800DEFF1DC0DEFF1EC0DEFF1FC0DEFF9DD783
:1053A8001C6A32AE01D01C2A010E1C162DC01DF03D
:1053B8000F0E1D163150030B020DF3501D241C2433
:1053C800020F3D6E2E50030B1C6E1D6A0A0ED890FC
:1053D8001C361D36E82EFBD72F501E6E1F6AD8903C
:1053E8001E361F36D8901E361F363044E846030B4B
:1053F8001E24206E000E1F20216E1C502024226EB9
:105408001D502120236E222A000E232222C038F0AC
:1054180023C039F03A6A3B6A3DC01CF0F70E1C26DF
:1054280038C01DF039C01EF03AC01FF03BC020F054
:105438001C2A05D0D8901D361E361F3620361C2E45
:10544800F9D734D05BA43FD0136A146A156A166A78
:105458008D0E42EC5EF0000901E037D19BEC60F064
:10546800280E0A6E0B6A0D6A100E0C6E0AEC5BF0C1
:10547800000901E12AD1300E3D6E03D09BEC60F0AB
:105488003D063D50FBE132C01CF01C3A0F0E1C16C5
:10549800100E1D6E1E6A1F6A206A1C2A05D0D8903D
:1054A8001D361E361F3620361C2EF9D71AC0D9FFD6
:1054B8001BC0DAFF1DC0DEFF1EC0DEFF1FC0DEFFFF
:1054C80020C0DEFF0AD7136A146A156A166A090E25
:1054D80042EC5EF0000901E0F8D0280E0A6E0B6A73
:1054E8000D6A100E0C6E0AEC5BF0000901E1EDD0BC
:1054F8005BA232D035C01CF0060E1D6ED8901C324F
:105508001D2EFCD7FF0E1C2632503F0B1E6E1F6A45
:10551800D8901E361F363344010B1E26000E1F225C
:105528001E2A1F221C2A03D0D8901E361F361C2E76
:10553800FBD71E50206E1F50216E226A236A1AC0A4
:10554800D9FF1BC0DAFF20C0DEFF21C0DEFF22C06A
:10555800DEFF23C0DEFFC1D63350030B1C6E1D6A6D
:10556800D8901C361D36D8901C361D36D8901C365F
:105578001D363338E842070B1C26000E1D221C2A54
:105588001D223240E8423F0B1F0B1E6E1F6A1E2A67
:10559800000E1F221C501E02F3CF20F0F4CF21F082
:1055A8001F02F35021261D501E02F35021262050C1
:1055B800226E2150236E246A256A1AC0D9FF1BC0A7
:1055C800DAFF22C0DEFF23C0DEFF24C0DEFF25C0D5
:1055D800DEFF83D63EC0D9FF3FC0DAFF5BC0DFFFE6
:1055E8007CD6136A146A156A166A090E42EC5EF0D4
:1055F80000096BE13EC00AF03FC00BF00D6A100EC7
:105608000C6E0AEC5BF0000901E067D65ED0136A05
:10561800146A156A166A0A0E42EC5EF0000955E132
:105628003EC00AF03FC00BF00D6A100E0C6E0AEC7B
:105638005BF0E9D7136A146A156A166A3A0E42ECE7
:105648005EF0000942E1040E3D6E0AD09BEC60F06A
:105658003EC0D9FF3FC0DAFFDF6E3E4A3F2A3D0613
:105668003D5001E13AD6F2D7136A146A156A166AF0
:105678008D0E42EC5EF0000928E19BEC60F03EC024
:105688000AF03FC00BF00D6A400E0C6E0AEC5BF09E
:10569800BAD7040E3C6E19D019501C6E1D6A1D50E5
:1056A800F8E11C5001E114D6010A01E118D6020AFA
:1056B80001E1C8D6090A8EE0010A93E0070AA7E0CB
:1056C800010AB8E0030AD0E0E4D7A8EC60F03C5047
:1056D8001200020E536E46504510441004E1020EAB
:1056E800435C01E2F3D120EE13F04150D926425039
:1056F800DA22DE50435CDE504458DE504558DE5016
:10570800465801E2D0D1E2D143C051F044C052F032
:10571800D8905230616F5130606F6051512661519D
:10572800522241C036F042C037F020EE1FF04150FF
:10573800D9264250DA22DECF60F0DECF61F0DECF2C
:1057480062F0DECF63F051C064F052C065F0090E1C
:10575800666FD89065336433662FFBD76451602534
:10576800386E65516121396E000E62213A6E000E65
:1057780063213B6E5EEC54F0536E535001E0A6D1AA
:1057880051500001606F010E5214616F6051412445
:10579800626F61514220636F2F0E62254F6E000EBB
:1057A8006321506E514A522A43B004D047C04BF08F
:1057B8004C6A1AD04750606F616B603B613BF00EDA
:1057C800611760510F0B6113F00E60174FC0D9FFBE
:1057D80050C0DAFFDF500F0B626F636B60516211CC
:1057E8004B6E615163114C6E4FC0D9FF50C0DAFF48
:1057F8004BC0DFFF20EE03F04150D9264250DA2299
:10580800010EDF6E41C036F042C037F020EE1FF0C7
:105818004150D9264250DA22DECF60F0DECF61F067
:10582800DECF62F0DECF63F051C064F052C065F0A5
:10583800090E666FD89065336433662FFBD76451C1
:105848006025386E65516121396E000E62213A6E0D
:10585800000E63213B6E5EEC54F0536E535001E032
:1058680035D151500001606F010E5214616F6051C3
:105878004124626F61514220636F2F0E62254F6E83
:10588800000E6321506E43B00CD048C060F00F0E7C
:1058980060174FC0D9FF50C0DAFFDF50F00B60111E
:1058A80012D047C060F048C061F049C062F04AC0F9
:1058B80063F0050E05D0D8906333623361336033EB
:1058C800E82EF9D760514D6E4E6A4FC0D9FF50C0CF
:1058D800DAFF4DC0DFFFDED041C036F042C037F0FE
:1058E80020EE1FF04150D9264250DA22DECF60F078
:1058F800DECF61F0DECF62F0DECF63F04450646F3C
:105908004550656F4650666F676B60516425386E09
:1059180061516521396E625166213A6E6351672182
:105928003B6E5EEC54F0536E535001E0CFD043C051
:1059380060F044C061F0D890000160376137605171
:10594800626F010E6115636F62514124646F635188
:105958004220656F2F0E64250A6E000E65210B6EBE
:1059680047C00CF048C00DF079EC5FF093D041C00F
:1059780036F042C037F020EE1FF04150D926425091
:10598800DA22DECF60F0DECF61F0DECF62F0DECF6C
:1059980063F043C064F044C065F045C066F046C09B
:1059A80067F0080E05D0D8906733663365336433E3
:1059B800E82EF9D760516425386E61516521396E3A
:1059C800625166213A6E635167213B6E5EEC54F07A
:1059D800536E53507BE143C060F044C061F0000156
:1059E800D89060376137D890603761376051626FFF
:1059F800010E6115636F62514124646F6351422047
:105A0800656F2F0E64250A6E000E65210B6E1BEC68
:105A180053F00001666B676B686BF00E0D14696FCD
:105A280047506A6F48506B6F49506C6F0F0E4A149D
:105A38006D6F66516A11476E67516B11486E6851F8
:105A48006C11496E69516D114A6E43C060F044C0D3
:105A580061F0D89060376137D8906037613760510E
:105A6800626F010E6115636F62514124646F635167
:105A78004220656F2F0E64250A6E000E65210B6E9D
:105A880047C00CF048C00DF049C00EF04AC00FF0F6
:105A980040EC5AF020EE03F04150D9264250DA2269
:105AA800010EDF6E13D041C0D9FF42C0DAFFDF50CC
:105AB800606F616B61510AE16051010A01E124D60E
:105AC800030A01E109D7010A01E151D75350120035
:105AD8005A6A0101556B5A6A030E5A6401D0A7D15C
:105AE8005A5003E14D6A4E6A03D04E6A010E4D6E5C
:105AF8005A501E0D1B0EF324D96E020EF420DA6ED6
:105B0800DF6A5A501E0D000EF324D96E020EF420DF
:105B1800DA6EDF6A5A501E0D070EF324D96E020E94
:105B2800F420DA6E070EDE6AE806FDE20D0E4D027D
:105B3800F3CF22F0F4CF23F04E02F3502326820E47
:105B48002224D96E020E2320DA6EDF50246E24C080
:105B580025F0266A276A286A27C028F026C027F079
:105B680025C026F0256A0D0E4D02F3CF29F0F4CF9B
:105B78002AF04E02F3502A26810E2924D96E020EED
:105B88002A20DA6EDF502B6E2BC02CF02D6A2E6A7D
:105B98002F6A2DC02FF02CC02EF02D6A2C6A0D0E06
:105BA8004D02F3CF30F0F4CF31F04E02F3503126EE
:105BB800800E3024D96E020E3120DA6EDF50326E3C
:105BC80032C033F0346A356A366A33C036F0356A23
:105BD800346A336A2C503324376E2D503420386E93
:105BE8002E503520396E2F5036203A6E25503724E6
:105BF8003B6E265038203C6E275039203D6E285089
:105C08003A203E6E0D0E4D02F3CF3FF0F4CF40F038
:105C18004E02F3504026830E3F24D96E020E4020D8
:105C2800DA6EDF503B24416E000E3C20426E000EBF
:105C38003D20436E000E3E20446E41C045F042C0F8
:105C480046F043C047F044C048F0496A48BE496836
:105C580049C04AF049C04BF049C04CF05A501E0D9B
:105C68000F0EF324D96E020EF420DA6E45C0DEFF63
:105C780046C0DEFF47C0DEFF48C0DEFF49C0DEFF8A
:105C88004AC0DEFF4BC0DEFF4CC0DEFF5A501E0D7F
:105C98001C0EF324D96E020EF420DA6EDECF22F049
:105CA800DDCF23F022C00AF023C00BF00C6A0D6A86
:105CB8000E6A0F6A106A116A5A501E0D0F0EF324ED
:105CC800D96E020EF420DA6EDECF24F0DECF25F096
:105CD800DECF26F0DECF27F0DECF28F0DECF29F0AA
:105CE800DECF2AF0DECF2BF024C012F025C013F04F
:105CF80026C014F027C015F028C016F029C017F0E8
:105D08002AC018F02BC019F063EC56F00AC02CF02A
:105D18000BC02DF00CC02EF00DC02FF00EC030F0CF
:105D28000FC031F010C032F011C033F05A501E0DC0
:105D38000F0EF324D96E020EF420DA6E2CC0DEFFAB
:105D48002DC0DEFF2EC0DEFF2FC0DEFF30C0DEFF1D
:105D580031C0DEFF32C0DEFF33C0DEFF5A501E0DF9
:105D6800170EF324D96E020EF420DA6EDE6ADE6AAC
:105D7800DE6A010EDD6E040E00019D6FFA0E9E6F45
:105D88005AC09FF0A06B5A501E0D0F0EF324D96E07
:105D9800020EF420DA6EDECF22F0DECF23F0DECF63
:105DA80024F0DECF25F0DECF26F0DECF27F0DECFE1
:105DB80028F0DECF29F022C0A1F023C0A2F024C031
:105DC800A3F025C0A4F026C0A5F027C0A6F028C0DF
:105DD800A7F029C0A8F05A501E0D0F0EF324D96E53
:105DE800020EF420DA6EDECF2AF0DECF2BF0DECF03
:105DF8002CF0DECF2DF0DECF2EF0DECF2FF0DECF71
:105E080030F0DECF31F02AC0A9F02BC0AAF02CC0A8
:105E1800ABF02DC0ACF02EC0ADF02FC0AEF030C04E
:105E2800AFF031C0B0F04FEC60F05A2A55D60101FE
:105E3800586B596A576B446B456B020E586E566F18
:105E48008390020C41C0D9FF42C0DAFFDECF6AF06E
:105E5800DDCF6BF046504510441003E1020E435C61
:105E680010E3000120EE13F06A51D9266B51DA22B3
:105E7800DE50435CDE504458DE504558DE504658EC
:105E880008E3010E0001646F000E656B666B676BBB
:105E980077D164696569666967695ED143C068F0EE
:105EA80044C069F0D8906931486E6831476E4750F0
:105EB8006827485069236AC036F06BC037F020EE77
:105EC8001FF06A51D9266B51DA22DECF47F0DECFB8
:105ED80048F0DECF49F0DECF4AF068C04BF069C029
:105EE8004CF0090E4D6ED8904C324B324D2EFBD7EC
:105EF8004B504724386E4C504820396E000E4920CC
:105F08003A6E000E4A203B6E5EEC54F0000901E048
:105F180037D100016851476E010E6915486E475028
:105F28006A25496E48506B214A6E2F0E4924D96E56
:105F3800000E4A20DA6EDF50626F636B684B692B84
:105F48006AC036F06BC037F020EE1FF06A51D926D0
:105F58006B51DA22DECF47F0DECF48F0DECF49F0D2
:105F6800DECF4AF068C04BF069C04CF0090E4D6EA8
:105F7800D8904C324B324D2EFBD74B504724386EBD
:105F88004C504820396E000E49203A6E000E4A20C7
:105F98003B6E5EEC54F0000901E0F2D0000168515C
:105FA800476E010E6915486E47506A25496E48507C
:105FB8006B214A6E2F0E4924D96E000E4A20DA6EE4
:105FC800DF504C6E4B6A4B5062134C50631343B016
:105FD80006D06251606F0F0E6315616F0FD062C0FB
:105FE80047F063C048F0040E496ED89048324732F3
:105FF800492EFBD747C060F048C061F060C064F02C
:1060080061C065F04AD06AC036F06BC037F020EE48
:106018001FF06A51D9266B51DA22DECF47F0DECF66
:1060280048F0DECF49F0DECF4AF044504B6E455081
:106038004C6E46504D6E4E6A47504B24386E485051
:106048004C20396E49504D203A6E4A504E203B6ED6
:106058005EEC54F0000901E093D043C047F044C01F
:1060680048F0D890473648364750496E010E4814D4
:106078004A6E495000016A254B6E4A506B214C6E9E
:106088002F0E4B240A6E000E4C200B6EAFEC5EF008
:106098000AC064F00BC065F00001666B676B70D0D6
:1060A8006AC036F06BC037F020EE1FF06A51D9266F
:1060B8006B51DA22DECF47F0DECF48F0DECF49F071
:1060C800DECF4AF043C04BF044C04CF045C04DF021
:1060D80046C04EF0080E05D0D8904E324D324C32A4
:1060E8004B32E82EF9D747504B24386E48504C2095
:1060F800396E49504D203A6E4A504E203B6E5EEC48
:1061080054F000093DE143C047F044C048F0D8903E
:1061180047364836D890473648364750496E010EBC
:1061280048144A6E495000016A254B6E4A506B214B
:106138004C6E2F0E4B240A6E000E4C200B6E1BEC7F
:1061480053F00A500001646F0B50656F0C50666F76
:106158000F0E0D14676F14D06AC0D9FF6BC0DAFF39
:10616800DF50476E486A485001E08BD64750010A15
:1061780001E194D6030A01E146D7010A91E081D6EC
:1061880064C041F065C042F066C043F067C044F0A7
:1061980012008BC0D9FF8CC0DAFFDECF9FF0DDCFB5
:1061A800A0F020EE0EF08B51D9268C51DA22DECFEA
:1061B8008FF0DECF90F0DECF91F0DECF92F0200EA0
:1061C8008F259B6F000E90219C6F000E91219D6F73
:1061D800000E92219E6F9E5103E1200E9D5D0AE301
:1061E80020EE16F08B51D9268C51DA22DE6ADE6A4F
:1061F800DE6ADD6A20EE16F08B51D9268C51DA2240
:10620800DE50DE10DE10DE1001E1040C9B518F6FB2
:10621800010E9C15906F916B926B8F1191119211D9
:1062280001E029D120EE16F08B51D9268C51DA22C3
:10623800DE2A000EDE22DE22DE2220EE12F08B5154
:10624800D9268C51DA22DE50DE10DE10DE102CE169
:1062580020EE07F09F51D926A051DA22DECF8FF029
:10626800DDCF90F08F51916F9051926F936B946B3B
:106278009BC095F09CC096F09DC097F09EC098F08A
:10628800060E05D0D8909833973396339533E82E79
:10629800F9D79151955D92519659935197599451C7
:1062A800985901E2E8D06ED020EE09F09F51D92626
:1062B800A051DA22DECF8FF0DDCF90F0FF0E8F25D0
:1062C800916FFF0E9021926F9BC093F09CC094F049
:1062D8009DC095F09EC096F00A0E05D0D8909633D2
:1062E800953394339333E82EF9D791519315976FDB
:1062F80092519415986F996B9A6B971199119A11FD
:1063080001E0B9D08BC041F08CC042F020EE12F011
:106318008B51D9268C51DA22DECF43F0DECF44F000
:10632800DECF45F0DECF46F026EC2FF041C0A1F0DD
:1063380042C0A2F043C0A3F044C0A4F00001A4519D
:10634800A311A21104E1020EA15D01E2020CA12930
:1063580007E1A22905E1A32903E1A42901E1010C30
:1063680020EE13F09F51D926A051DA22DE50A15D0C
:10637800DE50A259DE50A359DE50A45950E38D5186
:106388008E110BE120EE16F08B51D9268C51DA22B2
:10639800DE6ADE6ADE6ADD6A040C8BC06EF08CC0D1
:1063A8006FF020EE12F08B51D9268C51DA22DECF15
:1063B80070F0DECF71F0DECF72F0DECF73F03FEC1D
:1063C80025F06EC0A1F06FC0A2F070C0A3F071C03C
:1063D800A4F0A151A211A311A41101E1070CA10578
:1063E800A211A311A41101E1020CA12907E1A2291C
:1063F80005E1A32903E1A42901E1010C9FC036F0BE
:10640800A0C037F0A1C038F0A2C039F0A3C03AF05C
:10641800A4C03BF0CCEC4BF0000901E0010C0001FA
:1064280020EE12F08B51D9268C51DA22A1C0DEFF62
:10643800A2C0DEFFA3C0DEFFA4C0DEFF9FC00AF03B
:10644800A0C00BF0A1C00CF0A2C00DF0A3C00EF0CC
:10645800A4C00FF036EC4AF0000120EE16F08B5184
:10646800D9268C51DA220AC0DEFF0BC0DEFF0CC031
:10647800DEFF0DC0DEFF20EE0EF08B51D9268C51C9
:10648800DA229BC0DEFF9CC0DEFF9DC0DEFF9EC0FF
:10649800DEFF9B518F6F010E9C15906F8F519F25CA
:1064A800916F9051A021926F2F0E9127000E922389
:1064B80020EE1AF08B51D9268C51DA2291C0DEFFDA
:1064C80092C0DDFF000C4FC0D9FF50C0DAFFDECF0D
:1064D8007EF0DDCF7FF0545009E1200E535CD8B038
:1064E800020C51C06CF01F0E6C1701E0020C20EE7C
:1064F8000EF04F50D9265050DA2251C0DEFF52C05C
:10650800DEFF53C0DEFF54C0DEFF20EE06F04F5022
:10651800D9265050DA22DECF7AF0DECF7BF0DECFFC
:106528007CF0DECF7DF07A517B117C117D1115E175
:106538007EC0D9FF7FC0DAFF020EDF640ED020EEE6
:1065480023F07E51D9267F51DA22DECF7AF0DECFD2
:106558007BF0DECF7CF0DECF7DF07A517B117C11B1
:106568007D1140E120EE07F07E51D9267F51DA22D5
:10657800DECF6CF0DDCF6DF06C516E6F6D516F6FCB
:10658800706B716B51C072F052C073F053C074F0ED
:1065980054C075F0060E05D0D89075337433733334
:1065A8007233E82EF9D76E51725D6F51735970517D
:1065B80074597151755901E3020C20EE23F07E5194
:1065C800D9267F51DA2210EE16F04F50E1265050AE
:1065D800E222DECFE6FFDECFE6FFDECFE6FFDECF4C
:1065E800E6FF86D020EE09F07E51D9267F51DA22C7
:1065F800DECF6CF0DDCF6DF06C516E6F6D516F6F4B
:10660800706B716B090ED8906E376F3770377137B2
:10661800E82EF9D76EC076F06FC077F070C078F0CA
:1066280071C079F040D04FC041F050C042F07AC0FC
:1066380043F07BC044F07CC045F07DC046F026ECBA
:106648002FF041C07AF042C07BF043C07CF044C0D8
:106658007DF000017A2907E17B2905E17C2903E126
:106668007D2901E1010C7D517C117B1104E1020EB1
:106678007A5DD8A0020C20EE13F07E51D9267F5106
:10668800DA22DE507A5DDE507B59DE507C59DE50CE
:106698007D5901E3020C7651515E7751525A785177
:1066A800535A7951545A7651515C7751525878510E
:1066B800535879515458B7E27EC00AF07FC00BF0A6
:1066C8007AC00CF07BC00DF07CC00EF07DC00FF0DE
:1066D80036EC4AF020EE16F04F50D9265050DA2208
:1066E8000AC0DEFF0BC0DEFF0CC0DEFF0DC0DEFF00
:1066F80020EE12F04F50D9265050DA227AC0DEFF31
:106708007BC0DEFF7CC0DEFF7DC0DEFF20EE16F022
:106718004F50D9265050DA22DE50DE10DE10DE103F
:1067280001E1020C51C06CF052C06DF053C06EF024
:1067380054C06FF00A0E06D00001D8906F336E3344
:106748006D336C33E82EF8D720EE16F04F50D9266B
:106758005050DA226C51DE266D51DE226E51DE2257
:106768006F51DE2251506C6F010E52146D6F6C51D7
:106778007E256E6F6D517F216F6F2F0E6E27000E75
:106788006F2320EE1AF04F50D9265050DA226EC0EF
:10679800DEFF6FC0DDFF000C5A500C0D0B0EF3240A
:1067A800D96E010EF420DA6EDF500001DC6FDCC018
:1067B800DDF0DE6BDF6BE06B5A500C0D000EF3243E
:1067C800D96E010EF420DA6EDECFE1F0DDCFE2F013
:1067D800E1C0E3F0E2C0E4F0000EE4BFFF0EE56FB5
:1067E800E66FE351DD03F3CFE7F0F4CFE8F0E96BB0
:1067F800EA6BDE03F350E827F450E923000EEA239E
:10680800E451DD03F350E827F450E923000EEA23AE
:10681800E351DF03F350E927F450EA23E451DE03A0
:10682800F350E927F450EA23E551DD03F350E92753
:10683800F450EA23E051E303F350EA27E451DF037D
:10684800F350EA27E551DE03F350EA27E651DD036A
:10685800F350EA27E7C0ECF0E8C0EDF0E9C0EEF04D
:10686800EAC0EFF0ECC00AF0EDC00BF0EEC00CF09F
:10687800EFC00DF05A500C0D0A0EF324D96E010E1C
:10688800F420DA6EDF50DC6FDCC0DDF0DE6BDF6B2E
:10689800E06BDFC0E0F0DEC0DFF0DDC0DEF0DD6B16
:1068A800DDC00EF0DEC00FF0DFC010F0E0C011F068
:1068B80077EC57F00AC0ECF00BC0EDF00CC0EEF02E
:1068C8000DC0EFF05A500C0D0B0EF324D96E010ECB
:1068D800F420DA6EDF50DC6FDCC0DDF0DE6BDF6BDE
:1068E800E06B5A500C0D020EF324D96E010EF42001
:1068F800DA6EDF50E16FE1C0E2F0E36BE46BE56B69
:10690800E4C0E5F0E3C0E4F0E2C0E3F0E26BE2519A
:10691800DD03F3CFE6F0F4CFE7F0E86BE96BDE03D5
:10692800F350E727F450E823000EE923E351DD0391
:10693800F350E727F450E823000EE923E251DF0380
:10694800F350E827F450E923E351DE03F350E82736
:10695800F450E923E451DD03F350E827F450E92328
:10696800E051E203F350E927E351DF03F350E9274D
:10697800E451DE03F350E927E551DD03F350E9273D
:10698800E651EC27E751ED23E851EE23E951EF23D7
:106998005A500C0D030EF324D96E010EF420DA6E52
:1069A800DF50DC6FDCC0DDF0DE6BDF6BE06BDFC07F
:1069B800E0F0DEC0DFF0DDC0DEF0DD6BDD51EC279E
:1069C800DE51ED23DF51EE23E051EF235A50220D23
:1069D800000EF3248B6F030EF4208C6FECC08DF047
:1069E800EDC08EF0EEC08FF0EFC090F0EFEC0EF03F
:1069F800EB6FEB5111E0330E9D6FFB0E9E6FECC0F9
:106A08009FF0EDC0A0F0EEC0A1F0EFC0A2F0EBC087
:106A1800A3F0A46B4FEC60F0900E9D6FFE0E9E6F7E
:106A28004FEC60F083905A500C0D040EF324D96E8D
:106A3800010EF420DA6EECC0DEFFEDC0DEFFEEC022
:106A4800DEFFEFC0DEFF0101536B526BFCEF3AF043
:106A5800000E0001F46F250EF36F000EF26F050EA5
:106A6800F16F0101F75105E1000E0001F46F280EE6
:106A7800F36F01015C510CE1F86B2F0E1C6E090ECF
:106A88001D6E830E1E6EFE0E1F6E0AEC5EF00DD09C
:106A9800240E00019D6FFA0E9E6F5CC19FF0A06BE3
:106AA800F8C1A1F0A26B4FEC60F0FC0E00019D6FE5
:106AB800FD0E9E6F0101F8510F0D2F0EF3240001FA
:106AC8009F6F090EF420A06F4FEC60F0050E0001D7
:106AD800F06F0F0EEF6FF10EE82EFED7EF2FFCD7F9
:106AE800F02FFAD7C1D0C00E0B6EFC0E0C6E3BEC2B
:106AF8005FF00101DE51ECEC5FF0000E0001B96FB0
:106B0800030EBA6F760EBB6FFE0EBC6F010EBD6F23
:106B1800BDEC11F00101606F605166EC5BF00101A2
:106B280060510AE152EC1CF0000E526E030E536ED7
:106B380026EC5EF00101606F605166EC5BF0F46B6F
:106B4800280EF36F8DD00101F8510F0D2F0EF3248D
:106B5800D96E090EF420DA6E200EDE1806E1F82B45
:106B68000F0EF8657DD0F86B7BD0C10E00019D6FCC
:106B7800FB0E9E6F0101F8510F0D2F0EF32400013B
:106B88009F6F090EF420A06F4FEC60F0000EB96FF4
:106B9800030EBA6F0101F8510F0D2F0EF3240001F7
:106BA800BB6F090EF420BC6F030EBD6FBDEC11F076
:106BB8000101606F605166EC5BF00101605104E116
:106BC8000001F46B3C0EF36F040E0101601904E13F
:106BD8000001F46B410EF36F050E0001F06F0F0E0C
:106BE800EF6FF10EE82EFED7EF2FFCD7F02FFAD774
:106BF80037D0560E9D6FFC0E9E6F0101F8510F0D98
:106C08002F0EF32400019F6F090EF420A06F4FECA4
:106C180060F026D0560E9D6FFC0E9E6F0101F85154
:106C28000F0D2F0EF32400019F6F090EF420A06FA3
:106C38004FEC60F015D0F3C0EFF0F4C0F0F0F05175
:106C48000FE1EF51250A01E14ED70D0A01E17BD78B
:106C5800050A06E01F0A04E00E0ACBE07D0ADAE026
:106C68000001F107D8A0F2070001F2BF08D0F251E5
:106C780002E1F10504E33C0EF319F411DCE1030E23
:106C880001015C193BE1839E000E0A6EC00E38ECD0
:106C98005CF050EC5FF0000E0A6EC00E38EC5CF051
:106CA8003C0E0001F319F41116E10101ED510CE05D
:106CB800ED0E0E6E010E0F6E77EC58F08B0E0E6E09
:106CC800FC0E0F6E77EC58F0A00E0E6EFF0E0F6ED6
:106CD80077EC58F0000C2F0E1E6E090E1F6E510E29
:106CE800206EFF0E216E60C122F0236AC9EC5EF0AF
:106CF8002F0E0E6E090E0F6E77EC58F0000C2F0E4B
:106D08000101866F070E876FE5C00AF0E6C00BF039
:106D180011EC5DF00A5001017A6FC30E00018B6F10
:106D28008C6B8D6B8E6B8F6B906BEFEC0EF00101A3
:106D3800836F83510DE0010E00019D6FFB0E9E6F66
:106D48004FEC60F00001C36BC46BC56BC66B1200DF
:106D5800C30E4F6E506A86C151F087C152F0010EC2
:106D6800546E536A810E556E010E566ED1EC19F0B1
:106D78000101836F835108E0AA0E00019D6FFB0E8D
:106D88009E6F4FEC60F0DED786C1D9FF87C1DAFF6E
:106D9800800EDE1808E0AF0E00019D6FFC0E9E6F9E
:106DA8004FEC60F0CFD720EE0AF08651D9268751F4
:106DB800DA22DF500001E86FE76B010120EE0BF0EB
:106DC8008651D9268751DA22DF500001E7250101D3
:106DD8007F6F000E0001E8210101806F930E000112
:106DE8009D6FFB0E9E6F7FC19FF080C1A0F04FEC9E
:106DF80060F0C30E8B6F8C6B01017F510001E86F4F
:106E0800E76BE7C08DF0E8C08EF08F6B906BEFEC0E
:106E18000EF00101836F835195E1C30E4F6E506AE6
:106E280086C151F087C152F0010E546E536A810E2B
:106E3800556E010E566ED1EC19F00101836F835126
:106E480081E1846B856BE5C00AF0E6C00BF084C174
:106E5800E7F085C1E8F0050ED8900001E737E8377C
:106E6800E82EFAD7E751010186250C6E0001E8519A
:106E7800010187210D6E7AC10EF00F6ABAEC57F046
:106E88000A500B1060E184C1E7F085C1E8F0050EF7
:106E9800D8900001E737E837E82EFAD7E751010123
:106EA80086250001E96FE851010187210001EA6F99
:106EB8000E0EE925D96E000EEA21DA6EDF50EC6F6E
:106EC800EB6B84C1EDF085C1EEF0050ED890ED377F
:106ED800EE37E82EFBD7ED51010186250001EF6F53
:106EE800EE51010187210001F06F0F0EEF25D96ED9
:106EF800000EF021DA6EDF50EB25F16F000EEC2169
:106F0800F26FF1C07BF1F2C07CF10101000E7CBF91
:106F1800FF0E7D6F7E6F840E00019D6FFD0E9E6FCC
:106F28007BC19FF07CC1A0F07DC1A1F07EC1A2F021
:106F38004FEC60F07BC1C3F07CC1C4F07DC1C5F0EB
:106F48007EC1C6F01200844B852B85BF7CD7855146
:106F580005E10F0E845D01E3F5D675D7F3D614501D
:106F6800D96EDA6ADECF1CF0DDCF1DF01C0E1224BC
:106F7800206E000E1320216E20C00AF021C00BF0F5
:106F88000D6A200E0C6E0F6A0B0E0E6EC6EC5FF0CB
:106F9800226A236A1E6A1F6A1B6A080E1A6E1E502E
:106FA8001C24156E1F501D20166E15C0F6FF16C046
:106FB800F7FF000EF86E0E0EF76403D00800F550C8
:106FC80005D0F6CFE9FFF7CFEAFFEF50246E1E4A4F
:106FD8001F2A210E246001D0B9D02F0E241806E0F4
:106FE8005C0E241803E035D01E4A1F2A1E501C24AC
:106FF800156E1F501D20166E15C0F6FF16C0F7FF40
:10700800000EF86E0E0EF76403D00800F55005D098
:10701800F6CFE9FFF7CFEAFFEF502F0AE5E01E5061
:107028001C24156E1F501D20166E15C0F6FF16C0C5
:10703800F7FF000EF86E0E0EF76403D00800F55047
:1070480005D0F6CFE9FFF7CFEAFFEF505C0A7EE103
:10705800CBD72E0E241805E01A50225C1B5023585B
:107068000FE30B0E1A181B10D8B4060C2E0E24189A
:1070780001E0060C236A080E226E1B6A0B0E8ED7DF
:10708800245039EC5BF00A500B1040E01E501C24D1
:10709800156E1F501D20166E15C0F6FF16C0F7FF9F
:1070A800000EF86E0E0EF76403D00800F55005D0F8
:1070B800F6CFE9FFF7CFEAFFEF50196E1E4A1F2AF5
:1070C8001950FCEC57F00A500B10D8B4060CFF0E00
:1070D8001A24156EFF0E1B20166E1550225C1650D2
:1070E800235801E3060C22502024D96E2350212076
:1070F800DA6E24C0DFFF224A232A22502024D96EC8
:1071080023502120DA6E19C0DFFF1DD0A20E0A6EAF
:10711800FD0E0B6E24C00CF00D6A92EC5DF00A5067
:107128000B1001E0060C600E246405D07B0E246071
:1071380002D0200E245E22502024D96E2350212014
:10714800DA6E24C0DFFF224A232A29D71E501C24C6
:10715800156E1F501D20166E1450D96EDA6A15C0B0
:10716800DEFF16C0DDFF2250231001E1060C20C00F
:10717800D9FF21C0DAFFE50EDE1806E120C0D9FFED
:1071880021C0DAFF050EDF6E200E246403D0176AD3
:10719800186A03D0186A040E176E20EE0BF0205000
:1071A800D9262150DA2217C0DFFF000C0F0E5A161D
:1071B800E20E00019D6FF90E9E6F5AC09FF0A06B02
:1071C8005A501E0D1B0EF324D96E020EF420DA6EEF
:1071D800DF50A16FA26B4FEC60F003822F0E0A6E96
:1071E800070E0B6E0D6A0C6A010E0F6E0E6A26EC06
:1071F8005FF0040E5A1804E10F0EE8CF2FF704D001
:1072080027EE2FF05AC0DFFFFF0EE8CF30F702015C
:107218001B5102E0000E0BD0395102E0010E07D0DD
:10722800575102E0020E03D0755103E0030EE8CF78
:1072380030F7050E5A605BD05A501E0D1B0EF32412
:10724800D96E020EF420DA6EDFA403D0810EE8CFE7
:1072580031F75A501E0D1B0EF324D96E020EF4207E
:10726800DA6EDFA803D0020EE8CF31F75A501E0DB0
:107278001B0EF324D96E020EF420DA6EDFA003D0C1
:10728800020EE8CF33F75A501E0D1B0EF324D96EA9
:10729800020EF420DA6EDFA203D0020EE8CF33F735
:1072A8005A501E0D1B0EF324D96E020EF420DA6E0E
:1072B800DFA603D0800EE8CF32F75A501E0D1B0E02
:1072C800F324D96E020EF420DA6EDFAA03D0040E7E
:1072D800E8CF31F75A501E0D1B0EF324D96E020E5B
:1072E800F420DA6EDFAC03D0020EE8CF34F78FA4B7
:1072F80003D0080EE8CF35F7216A226A300E212420
:10730800D96E010E2220DA6EDF1C206E310E212488
:10731800D96E070E2220DA6E310E2124E16E070E97
:107328002220E26EE7502014DF6E214A222A22BE74
:10733800E5D7225003E1070E215CE0E3586A020E0C
:107348000101556548D05A501E0D010EF324D96E1F
:10735800020EF420DA6EDF501F6E1FC039F75A5044
:107368001E0D020EF324D96E020EF420DA6EDF50E1
:107378001F6E1FC03AF75A501E0D030EF324D96E24
:10738800020EF420DA6EDF501F6E1FC03BF75A5012
:107398001E0D040EF324D96E020EF420DA6EDF50AF
:1073A8001F6E1FC03CF75A501E0D050EF324D96EF0
:1073B800020EF420DA6EDF501F6E1FC03DF75A50E0
:1073C8001E0D060EF324D96E020EF420DA6EDF507D
:1073D8001F6E1FC03EF75A501E0D1B0EF324D96EA8
:1073E800020EF420DA6EDF6A140EA9EC56F003924E
:1073F80083901200546E505002E06CEC2DF0536AEA
:107408004F5001E1DFD0040E541802E1595003E156
:10741800140E541808E10101576B446B456B506A10
:10742800070E4F6E070C3F0E541806E1596A01010A
:10743800576B4F6A506A12005F0E541806E101013B
:10744800586B576B4F6A506A12003F0E546407D04E
:107458005F0E546004D00101E0515418F0E10101BD
:10746800E051541806E1010E586F576B4F6A506A85
:107478001200E151541803E1010E596EF6D7650E5A
:10748800541808E1595006E0446B456B010E576FDC
:107498008380ECD76E0E541807E1595002E1585119
:1074A80003E08380020E576F700E541806E158519E
:1074B80004E0446B456B030E576F700E541807E1D8
:1074C800595005E08380446B456B040E0CD0720E56
:1074D800541878E1595076E08380556B1C0E456F3F
:1074E8002A0E446F050E576FC1D7545046EC08F06A
:1074F800536E7AD0BC0E441909E1020E451906E113
:10750800DAEC38F00101576B586AB0D754501CECCC
:1075180049F0536E576B68D083802F0E0A6E070EA2
:107528000B6E0D6A0C6A010E0F6E0E6A26EC5FF088
:10753800038227EE2FF058C0DFFF0101424B432B97
:107548004C51421907E14D51431904E14C514D1179
:1075580001E0889C010EA9EC56F00392080E536EC8
:107568000101576B586A40D08390536A3DD0080E8A
:10757800541815E183905A6A536A586A030E556580
:1075880009D00F0E551906E0010E586E02011B5165
:1075980010091B6F010109D0446B456B25D0090EFA
:1075A800541805E18390536A586A576BF5D71F0E34
:1075B80054641AD0300E546017D054500F0B556FC6
:1075C800536AD0D701015751516E526A52500CE19B
:1075D80051500AE0010A89E0030A8CE0010A9CE0A4
:1075E800070AC2E0010AC3E053C04FF0506A120014
:1075F8000001D26B010ED16F838E8380D36BD46B65
:10760800D56BD66BDCD05A50220D000EF3244F6E8A
:10761800030EF420506E2F0E516E070E526E010E9F
:10762800546E536AD90E556E566AD1EC19F00001A2
:10763800DB6FDB5118E0180E0101516F010E536F1B
:107648000001DA6BD96FC00E9D6FF90E9E6F5AC09C
:107658009FF0A06BDBC0A1F0A26BD9C0A3F0DAC089
:10766800A4F04FEC60F001015A5135E0385139115E
:107678003A113B1130E05A500C0D040EF324D96E28
:10768800010EF420DA6E38C1C8F039C1C9F03AC128
:10769800CAF00001C76B000EC725CB6F010EC821C9
:1076A800CC6F000EC921CD6F000ECA21CE6FDE50FF
:1076B800CB1911E1DE50CC190EE1DE50CD190BE1EA
:1076C800DE50CE1908E12F0E296E070E2A6E010131
:1076D8005A5142EC4EF003920101515101E00382EC
:1076E8000001D951A9EC56F00001D76FD86B010EF3
:1076F8009D6FFF0E9E6F4FEC60F0D751D327D85186
:10770800D423000ED523D6238EBC8EA85DD0D951A4
:10771800D71903E1DA51D8190CE0420E9D6FFE0E1D
:107728009E6FD7C09FF0D8C0A0F04FEC60F0839454
:107738004BD0B5EC60F08BEC60F00A500B1004E015
:10774800010E0101536F40D00001D06B050ECF6FC1
:107758001CD0D00E0001C36FC90EE82EFED7C32F70
:10776800FCD700D08BEC60F00A500B100EE0000143
:10777800D16BD26B040E9D6FFD0E9E6FCFC09FF034
:10778800D0C0A0F04FEC60F008D00001CF07D8A01F
:10779800D007CF29DEE1D029DCE18EB808D0360E3B
:1077A8009D6FFF0E9E6F4FEC60F0D16BD26B8BEC30
:1077B80060F00A500B1003E00001D16BD26B00019E
:1077C800D151D21101E01FD70101536B839E8390E1
:1077D8001200838E8380586ADDEC3CF00101966FBD
:1077E800965102E096511200636B8E6B8F6B906B13
:1077F800916B946B010E936F996BD0D0976B986BCC
:107808001CD08BEC60F00A500B1015E0990E0A6E34
:10781800010E0B6E1CEC60F00101926F000E6325E7
:10782800D96EDA6A040EDA2292C1DFFF632B974B16
:10783800982B99BB05D08EAC03D001019805E1E3E4
:10784800010197518E2798518F23000E9023912381
:107858005A501E0D170EF324D96E020EF420DA6E5C
:10786800DE508E5DDE508F59DE509059DE509159B2
:1078780002E3936B946B99AB02D0936B946B8EBCC1
:1078880002D0936B946B980519E2000E63250A6E7B
:107898000B6A040E0B22FF0E6325D96EDA6A030EFB
:1078A800DA22DF500C6E0D6A635100080E6E000E6E
:1078B800D8A0E82A01080F6E26EC5FF001015A51A2
:1078C80045E0385139113A113B1140E05A503EE138
:1078D8005A501E0D070EF324D96E020EF420DA6EEC
:1078E80038C183F139C184F13AC185F1826B000E48
:1078F8008225866F010E8321876F000E8421886F91
:10790800000E8521896F8A6B8B6B8C6B8D6BDE50BB
:1079180086191CE1DE50871919E1DE50881916E135
:10792800DE50891913E1DE508A1910E1DE508B19F7
:107938000DE1DE508C190AE1DE508D1907E1000EC9
:10794800216E040E226E5A511CEC56F047EC4BF097
:107958000101956F636B955121E04B0E00019D6FFE
:10796800FB0E9E6F95C19FF0A06B4FEC60F0010E6F
:10797800586E5A501E0D1B0EF324D96E020EF420B9
:10798800DA6E5A501E0D1B0EF324E16E020EF4201F
:10799800E26EE7500409DF6E5850120093519411BB
:1079A80001E02CD78FA402D0010E586E8390839EDD
:1079B800000C5A501E0D070EF324D96E020EF42047
:1079C800DA6EDECFD8F0DECFD9F0DECFDAF0DECF58
:1079D800DBF05A501E0D070EF324D96E020EF42068
:1079E800DA6E5A501E0D0F0EF324E16E020EF420CB
:1079F800E26EDE50E65CDE50E658DE50E658DE50B9
:107A0800E658DE50E658DE50E658DE50E658DE50BE
:107A1800E65815E2010E586E5A501E0D1B0EF3243F
:107A2800D96E020EF420DA6E5A501E0D1B0EF32486
:107A3800E16E020EF420E26EE7500409DF6E5A5040
:107A48001E0D070EF324D96E020EF420DA6EDECF77
:107A5800B4F0DECFB5F0DECFB6F0DECFB7F0DECFD4
:107A6800B8F0DECFB9F0DECFBAF0DECFBBF05A50B7
:107A78001E0D170EF324D96E020EF420DA6EDECF37
:107A8800BCF0DECFBDF0DECFBEF0DECFBFF0000130
:107A9800BC51C06FBD51C16FBE51C26FBF51C36FE2
:107AA800C46BC56BC66BC76BB451C025C86FB551E5
:107AB800C121C96FB651C221CA6FB751C321CB6F5B
:107AC800B851C421CC6FB951C521CD6FBA51C62167
:107AD800CE6FBB51C721CF6F5A501E0D0F0EF32426
:107AE800D96E020EF420DA6EC851DE5CC951DE5838
:107AF800CA51DE58CB51DE58CC51DE58CD51DE5834
:107B0800CE51DE58CF51DE5815E2010E586E5A504C
:107B18001E0D1B0EF324D96E020EF420DA6E5A5095
:107B28001E0D1B0EF324E16E020EF420E26EE750E8
:107B38000409DF6E586A5A50220D000EF3248B6F29
:107B4800030EF4208C6FD8C08DF0D9C08EF0DAC047
:107B58008FF0DBC090F0EFEC0EF0DC6FDC5115E03D
:107B6800010E586E5A501E0D1B0EF324D96E020ECC
:107B7800F420DA6E5A501E0D1B0EF324E16E020E2D
:107B8800F420E26EE7500409DF6E585012008EA60A
:107B980004D08A0E1F6EFC0E03D0BA0E1F6EFF0EA5
:107BA800206E8EAA04D08A0E216EFC0E03D0B50E6C
:107BB800216EFF0E226E8EA804D08A0E236EFC0E54
:107BC80003D0D20E236EFE0E246E8EAE04D08A0E23
:107BD800256EFC0E03D0BF0E256EFF0E266E8EACF2
:107BE80004D08A0E276EFC0E03D0B00E276EFF0E4F
:107BF800286E8EA404D08A0E296EFC0E03D0C90EFE
:107C0800296EFF0E2A6E8EA204D08A0E2B6EFC0EF1
:107C180003D0CE0E2B6EFF0E2C6E8EA004D08A0ED3
:107C28002D6EFC0E03D0C40E2D6EFF0E2E6E90AE80
:107C380004D08A0E2F6EFC0E03D0FC0E2F6EFF0EA2
:107C4800306E90AC04D08A0E316EFC0E03D0F90E63
:107C5800316EFF0E326E90AA04D08A0E336EFC0E7F
:107C680003D0F60E336EFF0E346E90A804D08A0E41
:107C7800356EFC0E03D0F30E356EFF0E366E90A6F1
:107C880004D08A0E376EFC0E03D0F00E376EFF0E4E
:107C9800386E90A404D08A0E396EFC0E03D0ED0E17
:107CA800396EFF0E3A6E90A204D08A0E3B6EFC0E1F
:107CB80003D0EA0E3B6EFF0E3C6E90A004D08A0EF5
:107CC8003D6EFC0E03D0E70E3D6EFF0E3E6EB00E0D
:107CD80000019D6FF80E9E6F901C9F6FA06B8ECF5A
:107CE800A1F0A26B3DC0A3F03EC0A4F03BC0A5F03C
:107CF8003CC0A6F039C0A7F03AC0A8F037C0A9F038
:107D080038C0AAF035C0ABF036C0ACF033C0ADF027
:107D180034C0AEF031C0AFF032C0B0F02FC0B1F017
:107D280030C0B2F02DC0B3F02EC0B4F02BC0B5F007
:107D38002CC0B6F029C0B7F02AC0B8F027C0B9F0F7
:107D480028C0BAF025C0BBF026C0BCF023C0BDF0E7
:107D580024C0BEF021C0BFF022C0C0F01FC0C1F0D7
:107D680020C0C2F04FEF60F0070E0A24196E000E13
:107D78000B201A6E0AC0D9FF0BC0DAFFDF500E6E57
:107D88000E380F0B0A0DF3CF0FF0F4CF10F00AC026
:107D9800D9FF0BC0DAFFDF500F0B0F26000E1022A1
:107DA8000F28176E000E1020186E1C6A010E1B6E2D
:107DB8001D6A1E6A1F6A206AB2D01B501C1054E04C
:107DC8001DC00EF01EC00FF01FC010F020C011F033
:107DD8000A0E0E02F3CF12F0F4CF13F0146A156AEC
:107DE8000F02F3501326F4501422000E15220E022F
:107DF800F3501326F4501422000E15220A0E100216
:107E0800F3501426F4501522000E0F02F3501426D6
:107E1800F4501522000E0E02F3501426F4501522C9
:107E28000A0E1102F3501526000E1002F350152603
:107E3800000E0F02F3501526000E0E02F350152601
:107E480019C0D9FF1AC0DAFFDF50166E16380F0BAB
:107E580012241D6E000E13201E6E000E14201F6EBD
:107E6800000E1520206E54D01DC00EF01EC00FF05D
:107E78001FC010F020C011F00A0E0E02F3CF12F04E
:107E8800F4CF13F0146A156A0F02F3501326F45056
:107E98001422000E15220E02F3501326F450142259
:107EA800000E15220A0E1002F3501426F450152263
:107EB800000E0F02F3501426F4501522000E0E0285
:107EC800F3501426F45015220A0E1102F350152609
:107ED800000E1002F3501526000E0F02F35015265F
:107EE800000E0E02F350152619C0D9FF1AC0DAFF8A
:107EF800DF500F0B12241D6E000E13201E6E000E95
:107F080014201F6E000E1520206E1906D8A01A0620
:107F18001B501C10010ED8A4000E1B6E1C6A1706FD
:107F2800D8A01806172802E11828D8A446D71DC0DB
:107F38000AF01EC00BF01FC00CF020C00DF012009C
:107F480040C023F041C024F0AEEC43F04A6E4A50E2
:107F580001E0D2D040C0D9FF41C0DAFF030EDE18DD
:107F680001E0BAD020EE04F04050D9264150DA2280
:107F7800DE0401E0B1D02F0E40240A6E000E41202D
:107F88000B6E0D6A0C6A020E0F6E0E6AC6EC5FF07D
:107F98002D0E40240A6E020E41200B6EAA0E0D6EA5
:107FA800550E0C6E79EC5FF02F0E40240A6E000E11
:107FB80041200B6E520E0C6E0D6E610E0E6E410E50
:107FC8000F6E40EC5AF0130E40240A6E020E412048
:107FD8000B6E720E0C6E0D6E410E0E6E610E0F6EF4
:107FE80040EC5AF0170E40240A6E020E41200B6E28
:107FF80020EE0FF04050D9264150DA22DECF0CF0A7
:10800800DECF0DF0DECF0EF0DECF0FF040EC5AF0F1
:108018001B0E40240A6E020E41200B6E20EE0BF060
:108028004050D9264150DA22DECF0CF0DECF0DF0D9
:10803800DECF0EF0DECF0FF040EC5AF020EE1BF052
:108048004050D9264150DA22DECF42F0DECF43F04D
:10805800DECF44F0DECF45F04228466E000E4320C6
:10806800476E000E4420486E000E4520496E20EEF3
:108078002BF04050D9264150DA2246C0DEFF47C0D7
:10808800DEFF48C0DEFF49C0DEFF2F0E4024196E18
:10809800000E41201A6E20EE2BF04050D926415098
:1080A800DA22DECF1BF0DECF1CF0DECF1DF0DECFF4
:1080B8001EF0206A010E1F6E20EE01F04050D926F6
:1080C8004150DA22DF5032EC4FF020EE04F04050FD
:1080D800D9264150DA22DF6A196A1A6A1B6A20EE29
:1080E80001F04050D9264150DA22DF505FEC29F0E8
:1080F800000902E0010E4A6E4A5012005A51D8B4E3
:108108001200340E00019D6FFD0E9E6F4FEC60F063
:10811800C1EC53F01FC08AF120C08BF121C08CF153
:1081280022C08DF101018A518B118C118D1117E13B
:10813800EF0E00019D6FFB0E9E6F8AC19FF08BC1F1
:10814800A0F08CC1A1F08DC1A2F04FEC60F00A0E36
:108158000D6E000E0E6A0F6A106AE6EC5BF0010104
:108168008E6B8F6BE30E00019D6FFF0E9E6F8A0E64
:1081780001018E25D96E010E8F21DA6EDF500001C4
:108188009F6FA06B4FEC60F001018E4B8F2B8FBF60
:10819800E9D78F5103E1040E8E5DE4E32A0E000156
:1081A8009D6FF90E9E6F4FEC60F0CD0E9D6FFA0E2D
:1081B8009E6F4FEC60F023EE00F000EEC3F0210E4E
:1081C800DBCFEBFFE806FCE2D70EE56FFF0EE66FAC
:1081D80083EC36F0C3C038F1C4C039F1C5C03AF1F8
:1081E800C6C03BF10101385139113A113B11D8B4DD
:1081F8001200B30E00019D6FFA0E9E6F38C19FF0FA
:1082080039C1A0F03AC1A1F03BC1A2F04FEC60F037
:10821800000E8B6F030E8C6F38C1F4F039C1F5F086
:108228003AC1F6F0F36B000EF3258D6F010EF421C1
:108238008E6F000EF5218F6F000EF621906FEFEC18
:108248000EF00101606F000E4F6E030E506E2F0E80
:10825800516E070E526E546A080E536E880E556E94
:10826800010E566ED1EC19F00101606F906B916BA5
:10827800AB0E00019D6FFC0E9E6F2F0E0101902525
:10828800D96E070E9121DA6EDF5000019F6FA06B47
:108298004FEC60F00101904B912B91BFE9D79151C0
:1082A80005E1080E905DD8B01200E2D712006EC04A
:1082B800D9FF6FC0DAFFDECF85F0DDCF86F07351CE
:1082C8007211711104E1020E705DD8A0020C20EE4B
:1082D80013F08551D9268651DA22DE50705DDE50C2
:1082E8007159DE507259DE50735901E3020C745112
:1082F80075117611771118E085C041F086C042F0FB
:1083080074C043F075C044F076C045F077C046F0BD
:108318004768486849684A686DEC2BF00001846F2B
:10832800845102E0845112006EC041F06FC042F0E7
:1083380070C043F071C044F072C045F073C046F09D
:1083480026EC2FF041C080F042C081F043C082F09B
:1083580044C083F00001805181118211831171E0C2
:10836800800581118211831101E1020C802907E146
:10837800812905E1822903E1832901E1010C85C0F6
:1083880041F086C042F070C043F071C044F072C042
:1083980045F073C046F0476A486A496A4A6A6DEC14
:1083A8002BF00001846F8451BDE120EE13F085515C
:1083B800D9268651DA22FE0EDE24786FFF0EDE20E3
:1083C800796FFF0EDE207A6FFF0EDE207B6F20EEC6
:1083D8000FF08551D9268651DA227851DE5C795121
:1083E800DE587A51DE587B51DE5813E220EE0FF04A
:1083F8008551D9268651DA22DE2A000EDE22DE22B7
:10840800DE2220EE04F08551D9268651DA22000EAC
:10841800DB8080C070F081C071F082C072F083C0D0
:1084280073F020EE13F08551D9268651DA22DE50FA
:10843800705DDE507159DE507259DE50735901E299
:1084480073D7000CABC0D9FFACC0DAFFDECFB5F0F4
:10845800DDCFB6F003D00001AD4BAE2BADC0F6FFBB
:10846800AEC0F7FF000EF86E0E0EF76403D00800DA
:10847800F55005D0F6CFE9FFF7CFEAFFEF502F0A06
:10848800EAE0ADC0F6FFAEC0F7FF000EF86E0E0EC4
:10849800F76403D00800F55005D0F6CFE9FFF7CF11
:1084A800EAFFEF505C0AD7E0000120EE06F0AB517E
:1084B800D926AC51DA22DE6ADE6ADE6ADD6AADC030
:1084C800F6FFAEC0F7FF000EF86E0E0EF76403D08D
:1084D8000800F55005D0F6CFE9FFF7CFEAFFEF50D7
:1084E8000001AF6F200EAF6115D020EE27F0AB5121
:1084F800D926AC51DA22800EDF6EABC04FF0ACC08B
:1085080050F0000E516E526E536E546E67EC32F09E
:10851800000123D0ABC012F0ACC013F0AD0E146E46
:10852800B3EC37F00001B86FB85154E1ABC0A5F017
:10853800ACC0A6F06EEC47F0B86F20EE27F0AB5158
:10854800D926AC51DA22DF50B76FB85108E0040ED3
:10855800B81940E1B7B53ED0050EB86F3BD0B7B5F6
:1085680039D020EE04F0AB51D926AC51DA22DFA87D
:10857800F3D7B5C011F0B6C012F020EE0EF0AB5133
:10858800D926AC51DA22DECFAFF0DDCFB0F0AF5153
:10859800B16F010EB015B26FB151B525B36FB251BD
:1085A800B621B46F2F0EB325136E000EB421146ECE
:1085B80029EC59F0000120EE06F0AB51D926AC5158
:1085C800DA2211C0DEFF12C0DEFF13C0DEFF14C0C6
:1085D800DEFFA0D7B85112001A6E1A5001E0010C44
:1085E8005CA202D05C501200000E65EC5FF00A0E2F
:1085F800256E03D09BEC60F025062550FBE1226A2E
:10860800000E136A146A156A166A42EC5EF0E806F0
:1086180001E097D0AA0E136E010E146E156A166A41
:10862800080E42EC5EF0E80651E1256A25501B0F62
:10863800D96EDA6A9BEC60F0DF6E252A030E25649A
:10864800F5D71D047EE1AA0E1E187BE1030E246EE9
:10865800E80E236E15D0136A146A156A400E166E5A
:10866800A90E42EC5EF000090EE0150E196EC60E5A
:10867800E82EFED7192EFCD700D02306D8A0240652
:1086880023502410E8E1235024105BE0136A146A95
:10869800156A166A3A0E42EC5EF0000952E1256A44
:1086A80025501B0FD96EDA6A9BEC60F0DF6E252A25
:1086B800030E2564F5D71BBC03D0206A040E02D034
:1086C800206A0C0E1F6E1FC022F03BD0136A146A7A
:1086D800156A166AA90E42EC5EF0196E020E196050
:1086E80003D0226EA90E02D0010E226E216E030E57
:1086F800246EE80E236E14D0136A146A156A166A7B
:10870800215042EC5EF000090EE0150E196EC60EFF
:10871800E82EFED7192EFCD700D02306D8A02406B1
:1087280023502410E9E1235024100AE0136A020EB2
:10873800146E156A166A100E42EC5EF0000901E02C
:10874800226A22C05BF0A8EC60F0225001E14AD70F
:108758005C9048D7356A20EE03F02350D926245080
:10876800DA22DF5001E1A7D02F0E2324196E000E64
:1087780024201A6E20EE2BF02350D9262450DA221A
:10878800DECF1BF0DECF1CF0DECF1DF0DECF1EF0FB
:10879800206A010E1F6E20EE01F02350D9262450C6
:1087A800DA22DF5032EC4FF0000901E082D020EEEF
:1087B80003F02350D9262450DA22DF6A20EE17F07E
:1087C8002350D9262450DA2210EE1FF02350E12638
:1087D8002450E222E6CF29F0E6CF2AF0E6CF2BF0AC
:1087E800E6CF2CF010EE2BF02350E1262450E222A5
:1087F800E6CF2DF0E6CF2EF0E6CF2FF0E6CF30F023
:1088080029502D5C316E2A502E58326E2B502F581D
:10881800336E2C503058346EDE50315CDE50325896
:10882800DE503358DE50345846E220EE02F0235032
:10883800D9262450DA22020EDE183DE12F0E232419
:10884800196E000E24201A6E20EE17F02350D92638
:108858002450DA22DECF25F0DECF26F0DECF27F057
:10886800DECF28F020EE2BF02350D9262450DA2230
:10887800DECF29F0DECF2AF0DECF2BF0DECF2CF0D2
:10888800255029241B6E26502A201C6E27502B2089
:108898001D6E28502C201E6E206A010E1F6E20EEC1
:1088A80001F02350D9262450DA22DF5032EC4FF061
:1088B80002D0010E356E3550120089688B68F29E21
:1088C8008E280BE11A0E00019D6FFB0E9E6F8ECF56
:1088D8009FF0A06B4FEC60F00AD0780E00019D6FFE
:1088E800F90E9E6F8ECF9FF0A06B4FEC60F0902832
:1088F8000AE1D80E9D6FFB0E9E6F8ECF9FF0A06B86
:108908004FEC60F009D09D0E9D6FF90E9E6F8ECFD3
:108918009FF0A06B4FEC60F0290E406E960E3F6EF4
:108928007F0EE82EFED73F2EFCD7402EFAD7000048
:108938005C0E00019D6FFE0E9E6F4FEC60F08998F3
:108948008498090E406E1E0E3F6EE40EE82EFED788
:108958003F2EFCD7402EFAD700D04F0E00019D6F56
:10896800FE0E9E6F4FEC60F0899A849A090E406E55
:108978001E0E3F6EE40EE82EFED73F2EFCD7402E8B
:10898800FAD700D0C00E00019D6FFE0E9E6F4FEC0F
:1089980060F088908D9090280AE0D80E9D6FFB0EAD
:1089A8009E6F90CF9FF0A06B4FEC60F009D02D0E1A
:1089B8009D6FF90E9E6F90CF9FF0A06B4FEC60F00B
:1089C8008D80A30E406E570E3F6E020EE82EFED726
:1089D8003F2EFCD7402EFAD700D089688B688A686A
:1089E80083928382290E406E960E3F6E7F0EE82E8C
:1089F800FED73F2EFCD7402EFAD70000CBEC3DF037
:108A0800EFD74BC00BF04CC00CF04E0E0D6EC5EC02
:108A180052F04D6E4D5001E093D020EE0EF04B50C9
:108A2800D9264C50DA22DFAC8BD04EC036F04FC07E
:108A380037F020EE1CF04B50D9264C50DA22DECF0E
:108A480038F0DECF39F0DECF3AF0DECF3BF05EEC27
:108A580054F04D6E4D5074E120EE20F04B50D92665
:108A68004C50DA22DECF50F0DDCF51F020EE0BF083
:108A78005050D9265150DA22000EDB8A4BC0D9FF5C
:108A88004CC0DAFFDECF0EF0DDCF0FF050C010F093
:108A980051C011F020EE06F04B50D9264C50DA2286
:108AA800DECF12F0DECF13F0DECF14F0DECF15F0FC
:108AB80072EC5DF01C0E50240A6E000E51200B6EF5
:108AC80020EE0AF04B50D9264C50DA22DECF0CF0BB
:108AD800DECF0DF0DECF0EF0DECF0FF040EC5AF017
:108AE800160E50240A6E000E51200B6E0C6A0D6A89
:108AF800210E0E6E500E0F6E40EC5AF0120E5024DE
:108B08000A6E000E51200B6E000E0D6A0C6A79EC8D
:108B18005FF020EE03F04E50D9264F50DA22010EB6
:108B2800DF6E4EC040F04FC041F0A4EC3FF04D6EF8
:108B380020EE0EF04B50D9264C50DA22BF0EDF162D
:108B48004D501200136814680A50D96EDA6ADECFE5
:108B580015F0DDCF16F015C010F016C011F0155045
:108B6800161003E10A680B68120010C0F6FF11C066
:108B7800F7FF000EF86E0E0EF76403D00800F550EC
:108B880005D0F6CFE9FFF7CFEAFFEF50126E104A93
:108B9800112A200E126403D03A0E1218E6E13A0E9A
:108BA800121868E1000E0F6E010E0E6E15C0F6FF6A
:108BB80016C0F7FF000EF86E0E0EF76403D008001B
:108BC800F55005D0F6CFE9FFF7CFEAFFEF500C6E6E
:108BD8002F0E0C6439D015C0F6FF16C0F7FF000E33
:108BE800F86E0E0EF76403D00800F55005D0F6CFE6
:108BF800E9FFF7CFEAFFEF500C6E3A0E0C6024D075
:108C0800020E15240C6E000E16200D6E10500C1856
:108C18001BE111500D1818E115C0F6FF16C0F7FF3B
:108C2800000EF86E0E0EF76403D00800F55005D05C
:108C3800F6CFE9FFF7CFEAFFEF500C6ED00E0C2409
:108C48000E6E0F6AFF0E0F220FBE04D00F500DE1FB
:108C58000E040BE20EC013F00FC014F00A50D96EC8
:108C6800DA6A10C0DEFF11C0DDFF13C00AF014C0BD
:108C78000BF012000A6A0B6A120048C041F049C0A2
:108C880042F0436A446A456A466A4AEC4DF041C07C
:108C980070F042C071F0020E0001701971110DE000
:108CA800715106E1030E705D03E24A504B1005E175
:108CB80070C048F071C049F01200726B736B72C0DB
:108CC8004CF073C04DF04C3A4D3AF00E4D164C50E6
:108CD8000F0B4D12F00E4C164C5048244E6E4D5052
:108CE80049204F6EF50E4E240A6E010E4F200B6E72
:108CF8001BEC53F000017251040DF350600FD96E54
:108D0800DA6A0AC0DEFF0BC0DEFF0CC0DEFF0DC052
:108D1800DEFF724B732B735103E1040E725DCFE3D8
:108D28004A504B1003E1726B736B06D0FF0E4A2456
:108D3800726FFF0E4B20736F7251040DF350600F6A
:108D4800D96EDA6ADE50DE10DE10DE1004E1716BD7
:108D5800030E706F18D048C041F049C042F07251FC
:108D6800040DF350600FD96EDA6ADECF43F0DECF20
:108D780044F0DECF45F0DECF46F04AEC4DF041C07E
:108D880070F042C071F04A504B1092E100017151ED
:108D980003E1020E705D8CE3724B732B735188E113
:108DA800040E725D85E2C8D72F6C696664617461D0
:108DB800302E62696E20002F6C69666461746131BF
:108DC8002E62696E20002F6C696664617461322EB0
:108DD80062696E20002F6C696664617461332E626B
:108DE800696E20002F6C696664617461342E626953
:108DF8006E20002F6C696664617461352E62696E3D
:108E080020002F6C696664617461362E62696E2079
:108E1800002F6C696664617461372E62696E200088
:108E28002F6C696664617461382E62696E20002F48
:108E38006C696664617461392E62696E20002F6CFA
:108E4800696664617461612E62696E20002F6C69C5
:108E58006664617461622E62696E20002F6C6966B7
:108E680064617461632E62696E20002F6C696664A8
:108E7800617461642E62696E20002F6C696664619A
:108E88007461652E62696E20002F6C696664617476
:108E980061662E62696E200000000000000000007C
:108EA80000000000000000000000000000000000BA
:108EB80000000000000000000000000000000000AA
:108EC800000000000000000000000000000000009A
:108ED80000000000A5C0D9FFA6C0DAFFDECFA7F0CA
:108EE800DDCFA8F0A5C04FF0A6C050F0000E516E1F
:108EF800526E536E546E67EC32F00001AA6FAA519D
:108F080003E00001AA511200A7C036F0A8C037F04C
:108F180020EE16F0A551D926A651DA22DECF38F078
:108F2800DECF39F0DECF3AF0DECF3BF05EEC54F026
:108F38000001AA6FAA51E5E120EE1AF0A551D92641
:108F4800A651DA22DECF55F0DDCF56F055C0D9FF55
:108F580056C0DAFFDF50A96FA95103E1040EAA6FCA
:108F6800D0D720EE04F0A551D926A651DA2210EE6A
:108F78001AF0A551E126A651E22200EE0BF0E650C8
:108F8800E926E550EA22EF503F0BDF6E20EE1AF09B
:108F9800A551D926A651DA2210EE0BF0DE50E126B3
:108FA800DD50E222E7B618D020EE1AF0A551D926F6
:108FB800A651DA22DECF0AF0DDCF0BF01C0EA52574
:108FC8000C6E000EA6210D6E0F6A0B0E0E6E0AECCB
:108FD8005AF00A500B1095E0A5C08BF0A6C08CF093
:108FE80000018E6B8D6BCDEC30F00001AA6FAA5199
:108FF80088E18AD7F8C121F07CD0D9EC5FF0216EE6
:10900800F81901E185D0290E206E960E1F6E7F0E8D
:10901800E82EFED71F2EFCD7202EFAD7000078D0D6
:1090280086EC5CF0226E225073E022A002D001018F
:10903800592B22A202D0010159070F0E010159171D
:10904800000E0A6EC00E38EC5CF050EC5FF0000EBB
:109058000A6EC00E38EC5CF0010159510F0D2F0E4D
:10906800F3240E6E090EF4200F6E77EC58F0110EF3
:10907800206E3C0E1F6ECB0EE82EFED71F2EFCD79F
:10908800202EFAD7000022A443D0070E221840E071
:109098000B6A0A6A59C10CF0EDEC5DF01B0E000179
:1090A8009D6FFC0E9E6F59C19FF0A06B4FEC60F056
:1090B80059C121F0000E0A6E800E38EC5CF050ECBD
:1090C8005FF0000E0A6E800E38EC5CF00101595119
:1090D8000F0D2F0EF3240E6E090EF4200F6E77EC91
:1090E80058F0000E0A6EC00E38EC5CF050EC5FF0E1
:1090F8000FD001015C511F6E206A205009E11F50FA
:10910800010A01E17AD7030A01E177D7010A88E069
:109118002150120017C00AF018C00BF00D6A0C6A33
:109128000F6A080E0E6E26EC5FF0226A020E216EA0
:1091380021501724D96E22501820DA6E2150172496
:109148001D6E225018201E6E1D28E16E000E1E2076
:10915800E26EE7501F6E1F3AF00E1F161F162150C1
:109168001724E16E22501820E26EE750206E203856
:109178000F0B1F10DF6E214A222A22BED9D7225098
:1091880003E1070E215CD4E321501724D96E225045
:109198001820DA6E19C00AF01AC00BF01BC00CF0C8
:1091A8001CC00DF00A0E0E6E0F6A106A116AA9EC47
:1091B8005AF00A3AF00E0A1621501724E16E22508E
:1091C8001820E26EE7501D6E1D380F0B0A10DF6E77
:1091D80017C0D9FF18C0DAFFDF2A19C00AF01AC071
:1091E8000BF01BC00CF01CC00DF00A0E0E6E0F6ABF
:1091F800106A116AB4EC58F00AC019F00BC01AF0E2
:109208000CC01BF00DC01CF019501A101B101C10BC
:109218008CE117C0D9FF18C0DAFFDF06090EDF643A
:10922800090C17C0D9FF18C0DAFF100EDF6E100C3A
:109238002768930E00019D6FFD0E9E6F44C19FF03D
:1092480045C1A0F042C1A1F043C1A2F04FEC60F0CB
:10925800838003D02D0E82EC60F08EA88EAA03D0F6
:1092680027062728F7E15A501E0D070EF324D96E5A
:10927800020EF420DA6EDECF1FF0DECF20F0DECF54
:1092880021F0DECF22F0DECF23F0DECF24F0DECFD8
:1092980025F0DECF26F01FC00BF020C00CF021C057
:1092A8000DF022C00EF023C00FF024C010F025C02E
:1092B80011F026C012F010EC54F00D0E82EC60F0A4
:1092C8000A0E82EC60F001014C51421918E14D512F
:1092D800431915E14C514D1112E0889C10D0030E32
:1092E8000AD0050E286E446B456B2ED00A0E03D0AB
:1092F800010E01D0020E286E27D0286A25D044C15D
:109308001FF045C120F0205009E0020A0EE00E0AC5
:1093180010E0010A12E02A0A14E0EFD71F50DFE03C
:109328000A0ADDE01E0ADDE0E8D71F50BC0AE2E0C9
:10933800E4D71F501C0ADAE0E0D71F50AC0AD8E087
:10934800DCD71F500F0AD9E128501200000E010186
:10935800BE6F0A0EBD6F000EBC6F050EBB6F7BD0D3
:10936800BE6B140EBD6F6FD02F0E0B6EFC0E0C6E05
:109378003BEC5FF08FB204D00101BE6B1E0EBD6FD7
:10938800090E0101BA6F1E0EB96FE40EE82EFED762
:10939800B92FFCD7BA2FFAD7000055D0A80E0B6EFC
:1093A800FE0E0C6E3BEC5FF0000E0001A56F050E83
:1093B800A66F2C0EA76FF90EA86FA96BD4EC55F009
:1093C8000101606F605166EC5BF001016051D8E10A
:1093D800BE6B230ED4D7ED0E0B6EFD0E0C6E3BEC60
:1093E8005FF0000E0001B96F030EBA6FE20EBB6F9B
:1093F800010EBC6F010EBD6FBDEC11F00101606F75
:10940800605166EC5BF0010160510AE14FEC27F016
:10941800000E526E030E536E26EC5EF00101606F73
:10942800605166EC5BF0010CBDC1B9F1BEC1BAF187
:10943800BA5109E1B9510A0A93E01E0A95E00A0AED
:10944800ADE03D0AC8E0140E0101BD19BE1103E0EC
:10945800BB07D8A0BC07BCBF000CBC51E5E1BB05ED
:10946800E3E2000C020E0C5E000E0D5A0E5A0F5A63
:1094780020EE13F00A50D9260B50DA22FE0EDE2415
:10948800106EFF0EDE20116EFF0EDE20126EFF0E34
:10949800DE20136E10500C5C11500D5812500E58EF
:1094A80013500F5805E30A6A0B6A0C6A0D6A12001A
:1094B80020EE27F00A50D9260B50DA22DECF10F022
:1094C800DECF11F0DECF12F0DECF13F020EE09F080
:1094D8000A50D9260B50DA22DECF14F0DDCF15F072
:1094E8001450166E1550176E186A196A16500C0229
:1094F800F3CF1AF0F4CF1BF01C6A1D6A0D02F3506B
:109508001B26F4501C22000E1D2217500C02F3508B
:109518001B26F4501C22000E1D2216500E02F3507A
:109528001C26F4501D2217500D02F3501C26F4502F
:109538001D2218500C02F3501C26F4501D220F5007
:109548001602F3501D2617500E02F3501D26185010
:109558000D02F3501D2619500C02F3501D26105011
:109568001A240A6E11501B200B6E12501C200C6E10
:1095780013501D200D6E1200838E83800001DF6B57
:10958800E06B3AEC58F01FC0E1F020C0E2F0040EA6
:109598000001E25D07E3000EE125DF6FFC0EE2212A
:1095A800E06F04D0E1C0DFF0E2C0E0F001015A5101
:1095B80035E0385139113A113B1130E05A500C0D51
:1095C800040EF324D96E010EF420DA6E38C1D7F0F8
:1095D80039C1D8F03AC1D9F00001D66B000ED625B2
:1095E800DA6F010ED721DB6F000ED821DC6F000E79
:1095F800D921DD6FDE50DA1911E1DE50DB190EE1F9
:10960800DE50DC190BE1DE50DD1908E1000E216E99
:10961800040E226E01015A511CEC56F08FB415D07D
:109628005A50220D000EF32400018B6F030EF42014
:109638008C6F000E8D6F040E8E6F010E906F8F6B06
:10964800DF0E916FB6EC0BF0DE6F0001DE5109E022
:10965800240E9D6FFD0E9E6FDEC09FF0A06B4FEC39
:1096680060F0FEEC20F0536B8390839E8D0E00011A
:109678009D6FFC0E9E6FCECF9FF0A06BCDCFA1F05B
:10968800A26B4FEF60F05A501E0D070EF324D96EEF
:10969800020EF420DA6EDECFDDF0DECFDEF0DECFB4
:1096A800DFF0DECFE0F0DECFE1F0DECFE2F0DECFBC
:1096B800E3F0DECFE4F0DDC00AF0DEC00BF0DFC07F
:1096C8000CF0E0C00DF0E1C00EF0E2C00FF0E3C016
:1096D80010F0E4C011F05A501E0D1C0EF324D96E80
:1096E800020EF420DA6EDECFE5F0DDCFE6F0E5C05D
:1096F80012F0E6C013F0146A156A166A176A186A37
:10970800196AECEC50F00AC0E7F00BC0E8F00CC0A6
:10971800E9F00DC0EAF00EC0EBF00FC0ECF010C09D
:10972800EDF011C0EEF0E7C0EFF0E8C0F0F0E9C0EE
:10973800F1F0EAC0F2F0DDEC3CF0F56FF55102E033
:10974800F55112008FB414D05A50220D000EF32494
:109758008B6F030EF4208C6F000E8D6F040E8E6FCE
:10976800010E906F8F6BF30E916FB6EC0BF0F66FE6
:10977800F6510BE0240E9D6FFD0E9E6FF6C09FF014
:10978800A06B4FEC60F0F6511200CCEC4CF0000CE2
:1097980036C023F037C024F0AEEC43F0000901E0F6
:1097A800010C36C00AF037C00BF038C00CF039C0D5
:1097B8000DF03AC00EF03BC00FF036EC4AF00AC08C
:1097C80040F00BC041F00CC042F00DC043F020EE59
:1097D8002BF03650D9263750DA2240C0DEFF41C080
:1097E800DEFF42C0DEFF43C0DEFF2F0E36240A6EC6
:1097F800000E37200B6E0D6A0C6A020E0F6E0E6A91
:10980800C6EC5FF02F0E36243E6E000E37203F6EFA
:10981800456A010E446E466A476A04D0445046269B
:109828004550472220EE09F03650D9263750DA2223
:10983800DE50465CDE5047581FE23EC019F03FC07C
:109848001AF0465040241B6E475041201C6E000EF3
:1098580042201D6E000E43201E6E44C01FF045C0FE
:1098680020F020EE01F03650D9263750DA22DF50AA
:1098780032EC4FF00009D2E020EE09F03650D9263C
:109888003750DA224650DE1803E14750DE18D8A4D4
:10989800010C000C818E819CB00EF66E8D0EF76E59
:1098A800000EF86E09EE2FF011EE2CF00900F5CF3E
:1098B800EEFFE550E150FAE1E250F8E1C00EF66E35
:1098C800B80EF76E000EF86E03EEAAF010EE4CF02C
:1098D8000900F5CFEEFFE550E150FAE1560EF66EBD
:1098E800B90EF76E000EF86E02EE78F010EE48F042
:1098F8000900F5CFEEFFE550E150FAE1200EF66ED3
:10990800BE0EF76E000EF86E01EECCF010EE2BF0E6
:109918000900F5CFEEFFE550E150FAE1760EF66E5C
:10992800C10EF76E000EF86E0900F5CF5CF005EE7B
:1099380000F014EE2FF0EE6AE550E150FCE1E25041
:10994800FAE104EE00F011EE00F0EE6AE550E150A5
:10995800FCE1E250FAE103EE00F0AA0EEE6AE80636
:10996800FDE102EE00F0780EEE6AE806FDE101EE98
:1099780000F07A0EEE6AE806FDE10001FE6B5B6A14
:109988005A6A596A586A5D905D920001D4EF04F0F2
:109998005A501E0D070EF324D96E020EF420DA6E0B
:1099A800DECFB4F0DECFB5F0DECFB6F0DECFB7F065
:1099B800DECFB8F0DECFB9F0DECFBAF0DECFBBF045
:1099C8005A501E0D1C0EF324D96E020EF420DA6EC6
:1099D800DECFBCF0DDCFBDF0BC51B425BE6FBD51AC
:1099E800B521BF6F000EB621C06F000EB721C16F41
:1099F800000EB821C26F000EB921C36F000EBA2144
:109A0800C46F000EBB21C56F5A501E0D070EF324FC
:109A1800D96E020EF420DA6EBEC0DEFFBFC0DEFFD4
:109A2800C0C0DEFFC1C0DEFFC2C0DEFFC3C0DEFFB4
:109A3800C4C0DEFFC5C0DEFF5A501E0D070EF3245A
:109A4800D96E020EF420DA6EDECFC6F0DECFC7F094
:109A5800DECFC8F0DECFC9F05A50220D000EF32435
:109A68008B6F030EF4208C6FC6C08DF0C7C08EF0CC
:109A7800C8C08FF0C9C090F0EFEC0EF0CA6FCA51A1
:109A880003E0010E586E010C586A120020EE03F034
:109A98004150D9264250DA22DF6A20EE2BF041509D
:109AA800D9264250DA22DE68DE68DE68DD6841C009
:109AB80036F042C037F043C038F044C039F045C0F2
:109AC8003AF046C03BF05EEC54F0000904E0426A0C
:109AD800040E416E040C2D0E41240A6E020E422023
:109AE8000B6EAFEC5EF0550E0A1803E1AA0E0B18C8
:109AF80004E0426A030E416E030C20EE2FF0415041
:109B0800D9264250DA22E90EDE1812E020EE2FF0B4
:109B18004150D9264250DA22EB0EDE1809E020EE39
:109B28002FF04150D9264250DA22E80EDE1827E1FC
:109B3800650E41240A6E000E42200B6ED30E0C6E89
:109B4800FF0E0D6E0F6A030E0E6E0AEC5AF00A50E5
:109B58000B1003E1416A426A1200810E41240A6E29
:109B6800000E42200B6E8E0E0C6EFF0E0D6E0F6AED
:109B7800050E0E6E0AEC5AF00A500B10EBE0426A22
:109B8800020E416E020C1F6A226A8380990E000140
:109B98009D6FFA0E9E6FCECF9FF0A06BCDCFA1F038
:109BA800A26B4FEC60F019D0210E0A6E0B6A1CEC08
:109BB80060F0206E2C0E00019D6FFF0E9E6F1F2A15
:109BC8001FC09FF0A06B20C0A1F0A26B4FEC60F00B
:109BD80021AA03D020C022F005D08BEC60F00A50F7
:109BE8000B10E2E1140E00019D6FFD0E9E6F22C066
:109BF8009FF0A06B4FEC60F0020E22183CE15A5027
:109C0800130DAE0EF324D96E030EF420DA6E020E95
:109C1800DF6E5A50130DBA0EF324D96E030EF420DA
:109C2800DA6E080EDF6E5A500D0D7A0EF324D96ED7
:109C3800020EF420DA6E4C0EDF6E5A500D0D7D0EBA
:109C4800F324D96E020EF420DA6E080EDF6E5A5035
:109C58000D0D820EF324D96E020EF420DA6E050E75
:109C6800DF6E5A500D0D830EF324D96E020EF420C8
:109C7800DA6E690EDF6E586A839012002D6E690ED7
:109C880000019D6FFC0E9E6F2DC09FF0A06B29C038
:109C9800A1F02AC0A2F04FEC60F05DD0C1EC53F007
:109CA8001FC02EF020C02FF021C030F022C031F0AC
:109CB80029C0D9FF2AC0DAFFDF6A20EE01F0295057
:109CC800D9262A50DA2231C0DFFF20EE02F02950CF
:109CD800D9262A50DA22DF6A20EE03F02950D92645
:109CE8002A50DA2230C0DFFF20EE04F02950D926AE
:109CF8002A50DA22DF6A20EE05F02950D9262A50A8
:109D0800DA222FC0DFFF20EE06F02950D9262A508C
:109D1800DA22DF6A20EE07F02950D9262A50DA2203
:109D28002EC0DFFF1200C1EC53F01FC02EF020C080
:109D38002FF021C030F022C031F029C017F02AC01E
:109D480018F02EC019F02FC01AF030C01BF031C027
:109D58001CF08EEF48F02D502B6E2C6A2C50D8A496
:109D680012002B50010A9AE0030ADDE012000001FC
:109D7800E06B8380838E6CD03AEC58F01FC0DEF025
:109D880020C0DFF0040E0001DF5D03E3010EE06F89
:109D980003D0E3C0E1F0E26B8FB414D05A50220D27
:109DA800000EF3248B6F030EF4208C6F000E8D6F62
:109DB800040E8E6F010E906F8F6BE10E916FB6ECF3
:109DC8000BF0E36FE35109E0240E9D6FFD0E9E6FCB
:109DD800E3C09FF0A06B4FEC60F001015A5135E0F1
:109DE800385139113A113B1130E05A500C0D040E1C
:109DF800F324D96E010EF420DA6E38C1D7F039C1D8
:109E0800D8F03AC1D9F00001D66B000ED625DA6F2A
:109E1800010ED721DB6F000ED821DC6F000ED9218F
:109E2800DD6FDE50DA1911E1DE50DB190EE1DE508C
:109E3800DC190BE1DE50DD1908E1000E216E040E7D
:109E4800226E01015A511CEC56F0FEEC20F0536BC7
:109E58000001E05191E0839E83901200226E22500F
:109E6800D8A4040C1F50201001E1040C5CB0030CB2
:109E78005CB4020C5BB608D0090ED8901B361C36B1
:109E88001D361E36E82EF9D71F0420101AE11BC014
:109E980013F01CC014F01DC015F01EC016F0180EEB
:109EA80042EC5EF0000945E119C00CF01AC00DF053
:109EB800FE0E0E6EBCEC5BF000093BE01F6A206AE8
:109EC80038D05BC021F0060E211609E01FC013F040
:109ED80020C014F0156A166A970E42EC5EF01BC09B
:109EE80013F01CC014F01DC015F01EC016F0190E9A
:109EF80042EC5EF000091DE119C00CF01AC00DF02B
:109F0800FC0E0E6EBCEC5BF0000908E0020E1A268F
:109F18001F06D8A020061F502010EEE10C6A0D6A1B
:109F2800FD0E0E6EBCEC5BF0000903E1206A010E29
:109F38001F6EA8EC60F01F502010D8A4010C000C74
:109F4800A5C0D9FFA6C0DAFFDECFA9F0DDCFAAF001
:109F5800A5C04FF0A6C050F0000E516E526E536E61
:109F6800546E67EC32F00001AD6FAD5153E1AB6B4D
:109F7800AC6BA9C036F0AAC037F020EE16F0A55198
:109F8800D926A651DA22DECF38F0DECF39F0DECF7F
:109F98003AF0DECF3BF05EEC54F00001AD6FAD510E
:109FA80039E120EE1AF0A551D926A651DA22DECFE2
:109FB80055F0DDCF56F055C0D9FF56C0DAFFE50E93
:109FC800DE1810E020EE1AF0A551D926A651DA22A3
:109FD800DECF55F0DDCF56F055C0D9FF56C0DAFFB9
:109FE800DF5009E1AB4BAC2BA751AB1906E1A851E7
:109FF800AC1910E002D0AB6BAC6BA5C08BF0A6C05F
:10A008008CF08E6B010E8D6FCDEC30F00001AD6FD2
:10A01800AD51AFE0040EAD1902E1070EAD6FAD51C1
:10A0280012008C948C928C90889A110E0F6E3C0EB4
:10A038000E6ECB0EE82EFED70E2EFCD70F2EFAD7BB
:10A048000000110E0F6E3C0E0E6ECB0EE82EFED7E2
:10A058000E2EFCD70F2EFAD70000020E0F6EA00EA0
:10A068000E6E920EE82EFED70E2EFCD70F2EFAD7C4
:10A0780000D0000E0A6E300E38EC5CF02A0E0E6E20
:10A088008E0EE82EFED70E2EFCD7000E0A6E300E6E
:10A0980038EC5CF0000E0A6E300E38EC5CF0000E06
:10A0A8000A6E390E38EC5CF0000E0A6E140E38ECAD
:10A0B8005CF0000E0A6E560E38EC5CF0000E0A6E6C
:10A0C8006D0E38EC5CF0000E0A6E700E38EC5CF029
:10A0D800000E0A6E0C0E38EC5CF0000E0A6E060ECE
:10A0E80038EC5CF0000E0A6E010E38EC5CF0D00E15
:10A0F8000E6ECA0EE82EFED70E2EFCD71200838EE7
:10A1080083800001D26BD36BD46BD56B5A50220D70
:10A11800000EF3244F6E030EF420506E2F0E516E76
:10A12800070E526E010E546E536AD60E556E566A5D
:10A13800D1EC19F00001D16F01015A5135E03851C5
:10A1480039113A113B1130E05A500C0D040EF3242A
:10A15800D96E010EF420DA6E38C1C8F039C1C9F0E1
:10A168003AC1CAF00001C76B000EC725CB6F010EBC
:10A17800C821CC6F000EC921CD6F000ECA21CE6F49
:10A18800DE50CB1911E1DE50CC190EE1DE50CD19AD
:10A198000BE1DE50CE1908E12F0E296E070E2A6E4C
:10A1A80001015A5142EC4EF003920001D651A9EC3C
:10A1B80056F00001CF6FD06BCF51D227D051D323A7
:10A1C800000ED423D5230101536B839E8390120084
:10A1D8001A6A1B6A1C6A1D6A1E6A1F6A206A216A3B
:10A1E80012501310141015101610171018101910FB
:10A1F80045E0010E226E0AD0D89012361336143676
:10A2080015361636173618361936222A19AEF4D7E7
:10A21800D8901A361B361C361D361E361F36203689
:10A22800213612500A5C13500B5814500C58155014
:10A238000D5816500E5817500F58185010581950DE
:10A24800115811E312500A5E13500B5A14500C5A4D
:10A2580015500D5A16500E5A17500F5A1850105ABA
:10A268001950115A1A80D8901932183217321632EA
:10A278001532143213321232222ECAD71AC00AF0FB
:10A288001BC00BF01CC00CF01DC00DF01EC00EF062
:10A298001FC00FF020C010F021C011F01200010102
:10A2A800546B0001FE6B0101406B416B020E536F52
:10A2B8008390526B516B5A6A030E5A6401D049D08D
:10A2C8005A500C0D030EF324D96E010EF420DA6EE9
:10A2D800DF6A5A500C0D020EF324D96E010EF420D9
:10A2E800DA6EDF6A5A500C0D000EF324D96E010E97
:10A2F800F420DA6EDE6ADD6A5A500C0D040EF3247F
:10A30800D96E010EF420DA6EDE6ADE6ADE6ADD6A74
:10A318005A500C0D0B0EF324D96E010EF420DA6E90
:10A32800100EDF6E5A500C0D0A0EF324D96E010E72
:10A33800F420DA6E020EDF6E5A500C0D080EF3246C
:10A34800D96E010EF420DA6E240EDE6EDD6A5A2A0A
:10A35800B3D75A6A0101506B1200AEC0D9FFAFC023
:10A36800DAFFDECFB0F0DDCFB1F0AEC0A5F0AFC000
:10A37800A6F0000EA86F010EA76FA4EC4FF0B26F05
:10A38800B25147E1B0C036F0B1C037F020EE16F058
:10A39800AE51D926AF51DA22DECF38F0DECF39F010
:10A3A800DECF3AF0DECF3BF05EEC54F00001B26F46
:10A3B800B2512FE120EE1AF0AE51D926AF51DA2270
:10A3C800DECF0AF0DDCF0BF00D6A0C6A0F6A200EA3
:10A3D8000E6EC6EC5FF0000120EE1AF0AE51D926E1
:10A3E800AF51DA22DECF0AF0DDCF0BF01C0EAE251E
:10A3F8000C6E000EAF210D6E0F6A0B0E0E6EF0EC98
:10A408005CF020EE03F0B051D926B151DA22010EEA
:10A41800DF6EB25112008380838E000E0A6E040E26
:10A428000B6E0D6A0C68010E0F6E0E6A26EC5FF05B
:10A438000B0E00019D6FFE0E9E6F4FEC60F0C66B19
:10A44800C76BC6C054F0010E5416543254328350B0
:10A4580054187F0B5418836E2E0E82EC60F08FB464
:10A4680015D05A50220D000EF32400018B6F030EF5
:10A47800F4208C6F000E8D6F040E8E6F010E906F9E
:10A488008F6BC30E916FB6EC0BF0C56F0001C55111
:10A4980009E0720E9D6FFF0E9E6FC5C09FF0A06B06
:10A4A8004FEF60F0C64BC72BC7BFCBD7C75103E1EF
:10A4B8000A0EC65DC6E3180E9D6FFF0E9E6F4FEC29
:10A4C80060F0839E83908390586A12000F6A106A26
:10A4D8000E6A01D00A2A0A50D96EDA6A200EDE18EE
:10A4E800F9E00A50D96EDA6ADF500C6EF70E0C26C6
:10A4F800040E0C64EFD70A50D96EDA6A2D0EDE18F6
:10A5080004E1010E0E6E0A2A1ED00A50D96EDA6ACC
:10A518002B0EDE18F8E017D00A0E0F02F3CF0CF05E
:10A52800F4CF0DF01002F3500D260A50D96EDA6AF6
:10A53800DF500C5E000E0D5A300E0C240F6E000E0C
:10A548000D20106EE0D70A50D96EDA6ADF500C6E13
:10A55800D00E0C26090E0C64DFD70E500DE10FC08B
:10A568000CF010C00DF00C1E0D1E0C4A0D2A0CC06C
:10A578000AF00DC00BF012000FC00AF010C00BF06B
:10A588001200090E146E0B500C103BE00BC0D9FFE3
:10A598000CC0DAFFDE50DE1034E00BC0D9FF0CC06F
:10A5A800DAFFDECF0EF0DDCF0FF00EC0D9FF0FC0FF
:10A5B800DAFFDF5026E00BC0D9FF0CC0DAFF10EE3F
:10A5C80005F0DE50E126DD50E22220EE02F00B50CD
:10A5D800D9260C50DA22E650DE1813E1E650DE18D0
:10A5E80010E10BC0D9FF0CC0DAFF10EE01F0DE500D
:10A5F800E126DD50E222E750A2EC60F00E6E0EA0DC
:10A60800146A145003E0126A136A08D00BC0D9FF09
:10A618000CC0DAFFDECF12F0DDCF13F00D50D96E8B
:10A62800DA6A12C0DEFF13C0DDFF1450120020EEFC
:10A6380003F00A50D9260B50DA22DF50126E136A43
:10A64800146A156A20EE02F00A50D9260B50DA2255
:10A65800DF5012C00FF013C010F014C011F00E6AD2
:10A668000E10126E0F50136E1050146E1150156E9E
:10A6780020EE01F00A50D9260B50DA22DF5012C022
:10A688000FF013C010F014C011F00E6A0E10126E05
:10A698000F50136E1050146E1150156E0AC0D9FF6A
:10A6A8000BC0DAFFDF5012C00FF013C010F014C057
:10A6B80011F00E6A0E10126E0F50136E1050146EB9
:10A6C8001150156E12C00AF013C00BF014C00CF034
:10A6D80015C00DF01200216E2150D8A4040C1F5093
:10A6E800201001E1040C5CB0030C5BB608D0090E25
:10A6F800D8901B361C361D361E36E82EF9D720504A
:10A7080006E1020E1F5C03E2236A110E02D0236ADF
:10A71800120E226E22C024F01BC013F01CC014F0CD
:10A728001DC015F01EC016F0245042EC5EF0000962
:10A738001DE119C00AF01AC00BF0020E0D6E0C6A6A
:10A748000AEC5BF0000908E0020E1A261F06D8A0E2
:10A7580020061F502010EDE1120E241807E1136A9D
:10A76800146A156A166A0C0E42EC5EF0A8EC60F0EA
:10A778001F502010D8A4010C000C5EEC5EF0CC0E2B
:10A788002AEC60F0660E2AEC60F00DEC60F0256EA5
:10A79800255005E11F6A206A216A226A1200236A8D
:10A7A800246A2350250FD96EDA6A0DEC60F0DF6E4B
:10A7B800234A242A24BEF5D7245003E1040E235C3F
:10A7C800F0E3060E00019D6FFC0E9E6F25C09FF002
:10A7D800A06B26C0A1F0A26B27C0A3F0A46B28C071
:10A7E800A5F0A66B25C0A7F026C0A8F027C0A9F041
:10A7F80028C0AAF04FEC60F028502710261003E17B
:10A80800060E255CC7E325C01FF026C020F027C030
:10A8180021F028C022F01200156A0B0E146E070EE4
:10A828001426136A1450D96EDA6ADF50166E163A77
:10A838000F0E1616161616500CE0CC0E1624D96EEE
:10A84800DA6A010EDA22DF5082EC60F0010E156E32
:10A858000BD0150409E1CC0E1624D96EDA6A010E64
:10A86800DA22DF5082EC60F01450D96EDA6ADF50D9
:10A87800166E0F0E161616500CE0CC0E1624D96E56
:10A88800DA6A010EDA22DF5082EC60F0010E156EF2
:10A898000BD0150409E1CC0E1624D96EDA6A010E24
:10A8A800DA22DF5082EC60F01406132A070E1364D4
:10A8B800B9D7070C406A20EE2BF03650D92637500E
:10A8C800DA223850DE1809E13950DE1806E13A502C
:10A8D800DE1803E13B50DE1839E036C023F037C0FC
:10A8E80024F0AEEC43F0406E405030E12F0E362499
:10A8F800196E000E37201A6E38C01BF039C01CF0D4
:10A908003AC01DF03BC01EF0206A010E1F6E20EEFB
:10A9180001F03650D9263750DA22DF506FEC53F069
:10A92800000906E0386839683A683B68010E406EED
:10A9380020EE2BF03650D9263750DA2238C0DEFF09
:10A9480039C0DEFF3AC0DEFF3BC0DEFF40501200D8
:10A95800996B9A6B8FC09BF090C09CF09107D8A020
:10A96800920728D093C04FF094C050F0950E516EC6
:10A97800526A546A010E536EA10E556E566AD1EC96
:10A9880019F00001A105A2111EE195519D6F9E6B62
:10A998009F6BA06B9BC0D9FF9CC0DAFF9DC0DFFFF7
:10A9A8009B4B9C2B994B9A2B0A0E9D199E119F111C
:10A9B800A01109E09151995D9A51800A576E925100
:10A9C800800A5758CFE39BC0D9FF9CC0DAFFDF6AE3
:10A9D80099519A1103E18F6B906B12008FC08FF021
:10A9E80090C090F0120003D00A4A0B2A0C2A0C508F
:10A9F800D96EDA6ADF500D6E0AC0F6FF0BC0F7FF9A
:10AA0800000EF86E0E0EF76403D00800F55005D05E
:10AA1800F6CFE9FFF7CFEAFFEF500D1813E10AC0B0
:10AA2800F6FF0BC0F7FF000EF86E0E0EF76403D0AA
:10AA38000800F55005D0F6CFE9FFF7CFEAFFEF5051
:10AA48000009D2E10AC0F6FF0BC0F7FF000EF86E4E
:10AA58000E0EF76403D00800F55005D0F6CFE9FFD5
:10AA6800F7CFEAFFEF500D6E0C50D96EDA6ADF505F
:10AA78000D5C0A6E0B6AD8A00B0612000382040E46
:10AA88005A6033D02F0E0A6E070E0B6E5A50050D02
:10AA9800AC0EF3240C6E020EF4200D6E0F6A050E38
:10AAA8000E6ECFEC5CF0340E0A6E070E0B6E5A5029
:10AAB800130DAA0EF3240C6E030EF4200D6E0F6A0C
:10AAC800130E0E6ECFEC5CF0470E0A6E070E0B6E7F
:10AAD8005A500D0D780EF3240C6E020EF4200D6EF4
:10AAE8000F6A0D0E0E6ECFEC5CF0030E5A6409D09F
:10AAF800010E586E02011B5110091B6F000EE8CFA2
:10AB080030F7250EA9EC56F00392839012001350EB
:10AB180014100AE13CC113F03DC114F01350141095
:10AB280003E1136A146A120013C00EF014C00FF088
:10AB380015C010F032EC5DF00E5013260F501422A1
:10AB480013C0D9FF14C0DAFFDF5006E101013C6BE6
:10AB58003D6B136A146A120013C00EF014C00FF094
:10AB680015C010F052EC5DF00E50132401013C6F3B
:10AB78000F5014203D6F3CC1D9FF3DC1DAFFDF50B3
:10AB880008E03CC1D9FF3DC1DAFFDF6A3C4B3D2BF1
:10AB980002D03C6B3D6B13C013F014C014F01200CC
:10ABA800A7C0ABF0A8C0ACF0AB0E0A6EA6EC45F09F
:10ABB8000AC0AFF00BC0B0F00001B0BF0B0CD890CA
:10ABC800AF35D96EB035DA6E480ED926010EDA22C5
:10ABD800DECFADF0DDCFAEF0AD51AE1105E0ADC0CA
:10ABE800D9FFAEC0DAFFDF6AA551A61105E0A5C0FE
:10ABF800D9FFA6C0DAFFDF6AD890AF35D96EB03575
:10AC0800DA6E480ED926010EDA22A5C0DEFFA6C0EC
:10AC1800DDFFA95101E1000CA70E506EA50E516E83
:10AC2800526A536A5EEC00F00001AA6FAA51120042
:10AC3800256E39D020EE01F02150D9262250DA2293
:10AC4800DF50296E20EE03F02150D9262250DA2257
:10AC5800DF50286E20EE05F02150D9262250DA2246
:10AC6800DF50276E20EE07F02150D9262250DA2235
:10AC7800DF50266E26C00DF027C00EF028C00FF05A
:10AC880029C010F0E6EF5BF021C00AF022C00BF0FB
:10AC9800B8EC3EF00AC026F00BC027F00CC028F034
:10ACA8000DC029F0E7D72550236E246A2450D8A474
:10ACB80012002350010ABEE0030AE6E012001A6AF5
:10ACC8001B6A1C6A1D6A1E6A1F6A206A216A0AA01A
:10ACD80010D012501A2613501B2214501C22155043
:10ACE8001D2216501E2217501F22185020221950BC
:10ACF8002122D890123613361436153616361736E2
:10AD080018361936D890113210320F320E320D32F1
:10AD18000C320B320A320A500B100C100D100E10A8
:10AD28000F1010101110D3E11AC00AF01BC00BF05D
:10AD38001CC00CF01DC00DF01EC00EF01FC00FF09F
:10AD480020C010F021C011F01200026E07EE2FF0A3
:10AD58008490849A0F011391F29E83A4FED7896888
:10AD68008EA8FED78EA81DD0020425E0EE50866E70
:10AD7800861E8B6A8EA815D08EA2FCD78EA2FAD713
:10AD880089908EA80ED08EB2FCD78EA4FED789806B
:10AD9800898A8EA806D08EB4FCD78EA802D0022E3F
:10ADA800E1D78B68F90E896E0F0112911299138100
:10ADB800F28E025012008EA2FED703B2899AEE508C
:10ADC800866E861E8B6ADCD70000EBD70000042E47
:10ADD800FDD7120017C01AF018C01BF035D016C0E6
:10ADE80013F01A0E146E19C015F01450D96EDA6AE1
:10ADF800DECFF6FFDDCFF7FFF86A000EF86E080029
:10AE0800F550250A09E101D007D01450D96EDA6A45
:10AE1800DE2A000EDD2212D01450D96EDA6ADECF97
:10AE2800F6FFDDCFF7FFF86A000EF86E0800F55060
:10AE38000B6E0C6A13C00DF033EC57F01450D96E3A
:10AE4800DA6ADE2A000EDD221AC0F6FF1BC0F7FF01
:10AE5800F86A0800F550C3E1166A176A12000D5027
:10AE680002E00D5003E10B5070EF60F00D50D96E09
:10AE7800DA6A0A0ED926DE50DE1014E00D50D96EBB
:10AE8800DA6A0A0ED9260D50E16EE26A030EE1264F
:10AE9800DE50E65CE650800A126EDE50800A1258D8
:10AEA800D8B012000D50D96EDA6A030ED926DECF5B
:10AEB8000EF0DDCF0FF00D50D96EDA6ADECF10F04C
:10AEC800DDCF11F00E501024D96E0F501120DA6E1C
:10AED8000BC0DFFF0D50D96EDA6A030ED926DE2AC1
:10AEE800000EDD22000C0A500E02F3CF12F0F4CF50
:10AEF80013F0146A156A0A500F02F3501326F4501F
:10AF08001422000E15220B500E02F3501326F45093
:10AF18001422000E15220A501002F3501426F45081
:10AF280015220B500F02F3501426F45015220C5022
:10AF38000E02F3501426F450152211500A02F35051
:10AF480015260B501002F35015260C500F02F35023
:10AF580015260D500E02F350152612C00AF013C024
:10AF68000BF014C00CF015C00DF012000E06D8A09E
:10AF78000F060E280CE10F280AE10A6A0B6A120074
:10AF88000A4A0B2A0C4A0D2A0E06D8A00F060AC038
:10AF9800F6FF0BC0F7FFF86A0800F55016E00CC082
:10AFA800D9FF0DC0DAFFDF5010E00E500F100DE092
:10AFB8000CC0D9FF0DC0DAFF0AC0F6FF0BC0F7FFBF
:10AFC800F86ADE500900F518DBE00AC0F6FF0BC08E
:10AFD800F7FFF86A0800F5CF10F00CC0D9FF0DC0D4
:10AFE800DAFFDF50105C0A6E0B6AD8A00B0612005D
:10AFF8000C6E630EF66EF80EF76EF86A0900F550DF
:10B008000C5C31E3640EF66EF80EF76EF86A0C50BD
:10B018000900F55C04E30B6A010E0A6E010C650E6B
:10B02800F66EF80EF76EF86A0900F5500C5C09E345
:10B03800660EF66EF80EF76EF86A0C500900F55CAD
:10B04800EAE2670EF66EF80EF76EF86A0900F55038
:10B058000C5C09E3680EF66EF80EF76EF86A0C5091
:10B068000900F55CD8E20A6A0B6A1200226A236AB0
:10B078000101636B246A30D08BEC60F00A500B102E
:10B0880020E0240E0A6E0B6A1CEC60F0216E24A8E6
:10B098000CD0CC0E00019D6FFE0E9E6F21C09FF05C
:10B0A800A06B4FEC60F083900CD0000E010163257B
:10B0B800D96EDA6A040EDA2221C0DFFF632B224A36
:10B0C800232A24AA07D0000E22241F6E040E232050
:10B0D800206E12008EAC02D02304CEE322C01FF0F3
:10B0E80023C020F01200150E106EC60EE82EFED7F3
:10B0F800102EFCD700D020D0150E106EC60EE82EEC
:10B10800FED7102EFCD700D0010E0A6E0EC0F6FF37
:10B118000FC0F7FF000EF86E0E0EF76403D008009C
:10B12800F55005D0F6CFE9FFF7CFEAFFEF5038EC3E
:10B138005CF00E4A0F2AD7D70EC0F6FF0FC0F7FFF4
:10B14800000EF86E0E0EF76403D00800F55005D017
:10B15800F6CFE9FFF7CFEAFFEF500009CDE1120083
:10B16800126A136A146A156A0E500F101010111023
:10B1780029E0010E166E06D0D8900E360F3610361E
:10B188001136162A11AEF8D7D8901236133614365F
:10B1980015360E500A5C0F500B5810500C581150B1
:10B1A8000D5809E30E500A5E0F500B5A10500C5AF6
:10B1B80011500D5A1280D890113210320F320E32BF
:10B1C800162EE2D712C00AF013C00BF014C00CF010
:10B1D80015C00DF01200866A846A8B6889680101BF
:10B1E800636B039E839283944E6B4F6B09D0000E62
:10B1F8004E25D96E040E4F21DA6EDF6A4E4B4F2B67
:10B208004FBFF5D74F5102E14E05F1E34E6B4F6B3F
:10B2180009D02F0E4E25D96E070E4F21DA6EDF6A40
:10B228004E4B4F2B4FBFF5D74F05F3E30F0117696F
:10B23800D6501F0B4009D66ED6980F0ED612D58859
:10B24800D5120E01C29BD58E0F0C1A0E13240A6E4E
:10B25800000E14200B6EAFEC5EF00AC019F00BC0A4
:10B268001AF01B6A1C6A11C0D9FF12C0DAFF030E5C
:10B27800DE181CE1140E13240A6E000E14200B6E47
:10B28800AFEC5EF00A50156E0B50166E176A186A0E
:10B2980016C018F015C017F0166A156A155019125D
:10B2A80016501A1217501B1218501C1219C011F000
:10B2B8001AC012F01BC013F01CC014F01200126E5A
:10B2C8000C0E121807E0A8EC60F043EC60F00009DF
:10B2D80001E1FF0C1250400979EC60F00F5079EC55
:10B2E80060F00E5079EC60F00D5079EC60F00C5085
:10B2F80079EC60F0010E116E125002E1950E116E9C
:10B30800080E121802E1870E116E115079EC60F0E8
:10B318000C0E121802E19BEC60F00A0E116E9BEC09
:10B3280060F0106E10AE02D0112EF9D71050120036
:10B338000E500F10D8B4000C0EC0D9FF0FC0DAFFA2
:10B34800DF5001E1000C0EC00AF00FC00BF011EC49
:10B358005DF00AC010F00BC011F0020E10181110A9
:10B3680001E0000C120E0A6E0EC0D9FF0FC0DAFF02
:10B37800DF500FEC5CF00009D8B4000C130E0A6E15
:10B3880020EE01F00E50D9260F50DA22DF500FECD4
:10B398005CF0000901E1000C1238F00B13101200E8
:10B3A8008380038250050DE1000EE8CF2FF7500E81
:10B3B800E8CF30F7000EE8CF31F7E8CF32F7506B1F
:10B3C8001DD027EE2FF051C1DFFF000EE8CF30F778
:10B3D8000D0EE8CF31F7000EE8CF32F78FA403D077
:10B3E800600EE8CF32F78FA406D031C70AF0200EDE
:10B3F8000A120AC031F7010EE8CF33F7050EA9EC9F
:10B4080056F003920101516B839012000AC011F0AB
:10B418000BC012F00CC013F00DC014F011C0D9FF0E
:10B4280012C0DAFFDF50106E13C0F6FF14C0F7FF2A
:10B43800000EF86E0E0EF76403D00800F55005D024
:10B44800F6CFE9FFF7CFEAFFEF50105C156E166AEA
:10B45800D8A01606134A142A114A122A0E06D8A092
:10B468000F060E500F1003E015501610D7E015C048
:10B478000AF016C00BF012000AC0D9FF0BC0DAFFA1
:10B488000CC0DFFF0A4A0B2A0D500C6E0E500D6ED1
:10B498000F500E6E0F6A0AC0D9FF0BC0DAFF0CC03E
:10B4A800DFFF0A4A0B2A0D500C6E0E500D6E0F501E
:10B4B8000E6E0F6A0AC0D9FF0BC0DAFF0CC0DFFF9F
:10B4C8000A4A0B2A0D500C6E0E500D6E0F500E6E60
:10B4D8000F6A0AC0D9FF0BC0DAFF0CC0DFFF0A4AA7
:10B4E8000B2A12005A6A030E5A6401D02AD05A5005
:10B4F8000C0D030EF324D96E010EF420DA6EDF6A08
:10B508005A500C0D020EF324D96E010EF420DA6E97
:10B51800DF6A5A500C0D000EF324D96E010EF42088
:10B52800DA6EDE6ADD6A5A500C0D040EF324D96E09
:10B53800010EF420DA6EDE6ADE6ADE6ADD6A5A2AF5
:10B54800D2D75A6A8390536B12000E500F10101006
:10B55800111023E0010E126E06D0D8900E360F3669
:10B5680010361136122A11AEF8D70E500A5C0F5059
:10B578000B5810500C5811500D5808E30E500A5E25
:10B588000F500B5A10500C5A11500D5AD8901132B6
:10B5980010320F320E32122EE8D70AC00AF00BC052
:10B5A8000BF00CC00CF00DC00DF012005A6A0A6ABC
:10B5B8000B6A5A501E0D070EF324D96E020EF420A2
:10B5C800DA6E070EDE6AE806FDE25A501E0D1B0E03
:10B5D800F324D96E020EF420DA6EDF6A5A501E0D7B
:10B5E800170EF324D96E020EF420DA6EDE6ADE6AD4
:10B5F800DE6ADD6A0A4A0B2A0BBEDBD70B5003E171
:10B60800040E0A5CD6E38390586A1200070E0F6E88
:10B61800D00E0E6E0FD09BEC60F0106E10280DE16E
:10B62800E40E00D000D0E82EFCD700D000D00E06E3
:10B63800D8A00F060E500F10EEE1FE0E101801E014
:10B64800000C9BEC60F00AC0D9FF0BC0DAFFDF6E7C
:10B658000A4A0B2A0C06D8A00D060C500D10F1E171
:10B668009BEC60F09BEC60F0010C0C6E5F0EF66ECC
:10B67800F80EF76E000EF86E0900F5500C5C1FE32B
:10B68800600EF66EF80EF76EF86A0C500900F55C5D
:10B6980004E30B6A010E0A6E010C610EF66EF80ED9
:10B6A800F76EF86A0900F5500C5C09E3620EF66E55
:10B6B800F80EF76EF86A0C500900F55CEAE20A6ABF
:10B6C8000B6A1200206E6B0E216EF80E226E1F6A36
:10B6D8000BD021C0F6FF22C0F7FF214A222AF86AC0
:10B6E8000800F550F6E11F2A20501F1808E021C075
:10B6F800F6FF22C0F7FFF86A0800F550EAE1190ED4
:10B7080000019D6FFE0E9E6F20C09FF0A06B21C0B0
:10B71800A1F022C0A2F04FEF60F00AC010F00BC0F9
:10B7280011F013D00E06D8A00F060CC0D9FF0DC01B
:10B73800DAFF0C4A0D2A10C0E1FF11C0E2FF104ADF
:10B74800112ADFCFE7FFE7500BE00E500F1008E09B
:10B75800E9D710C0D9FF11C0DAFFDF6A104A112AF1
:10B768000E06D8A00F060E28F4E10F28F2E1120009
:10B7780079EC5EF0000901E1000C0E5079EC60F004
:10B78800FD0E0E181EE0020E106E0F6A0CC0D9FFD7
:10B798000DC0DAFFDF5079EC60F00C4A0D2A0F0675
:10B7A800D8A010060F501010F1E19BEC60F09BEC54
:10B7B80060F09BEC60F0116E11501F0B050A01E060
:10B7C800000C010C0DC011F00EC012F00FC013F0E8
:10B7D80010C014F05EEC5EF0CC0E2AEC60F0990E0E
:10B7E8002AEC60F00C0E2AEC60F0156A166A155007
:10B7F800110FD96EDA6ADF502AEC60F0154A162A62
:10B8080016BEF5D7165002E05EEF5EF0040E155C2A
:10B81800EEE35EEF5EF00B6E0A5001E1000C2F0EB6
:10B828000B6409D03A0E0B6006D00A50D96EDA6A5A
:10B838000B50D00F17D0400E0B6409D0470E0B6089
:10B8480006D00A50D96EDA6A0B50C90F0BD0600EB9
:10B858000B64000C670E0B60000C0A50D96EDA6A94
:10B868000B50A90FDF6E010C0B6E87920A0EE82EA3
:10B87800FED700D00AB002D0879401D08784000E8A
:10B888000D6E010E0C6E0BAE02D0838A01D0839A26
:10B89800D8900B36879000000000878000000000D9
:10B8A80087900C4A0D2A0DBEEED70D5003E1090E04
:10B8B8000C5CE9E3878212000109122001000100F3
:10B8C8001700002D119420D00F000101091220014A
:10B8D8000001001700002D119420D00F000101096C
:10B8E8001220010001001700002D119420D00F0034
:10B8F8000101091220010001001700002D119420F8
:10B90800D00F0001010E0A6E0B6A88868782878431
:10B91800000000008794000000000C6A0D6A8DA6E4
:10B9280002D00A500B12D8900A3687900000000007
:10B9380087800000000087900C4A0D2A0DBEEFD7C3
:10B948000D5003E1030E0C5CEAE30B5012000000FB
:10B958004F01000F0000000009FF0000004F010028
:10B968000F0000000009FF0000004F01000F000059
:10B97800000009FF0000004F01000F00000000094F
:10B98800FF00800102E805800102E805800102E865
:10B9980005800102E8050CC012F00DC013F00AC0C2
:10B9A80010F00BC011F010D012C0D9FF13C0DAFF8D
:10B9B800DF50146E124A132A10C0D9FF11C0DAFFE3
:10B9C80014C0DFFF104A112A0E06D8A00F060E2851
:10B9D800EBE10F28E9E112000AC010F00BC011F0EA
:10B9E8000CC012F00DC013F00E500F10D8B4120096
:10B9F80012C0D9FF13C0DAFF10C0E1FF11C0E2FF87
:10BA0800DFCFE7FF124A132A104A112A0E06D8A0E0
:10BA18000F060E500F10ECE112000AC00CF00BC01C
:10BA28000DF002D00A4A0B2A0AC0F6FF0BC0F7FF36
:10BA3800000EF86E0E0EF76403D00800F55005D01E
:10BA4800F6CFE9FFF7CFEAFFEF500009EBE10C5022
:10BA58000A5C0A6E0D500B580B6E1200116A126ABE
:10BA680004D00E4A0F2A114A122A0EC0D9FF0FC05D
:10BA7800DAFFDF500EE010C00AF00EC0D9FF0FC089
:10BA8800DAFFDF500B6E0C6AB3EC5FF00A500B1054
:10BA9800E8E111C00EF012C00FF01200116A126A2C
:10BAA80004D00E4A0F2A114A122A0EC0D9FF0FC01D
:10BAB800DAFFDF500EE010C00AF00EC0D9FF0FC049
:10BAC800DAFFDF500B6E0C6AB3EC5FF00A500B1014
:10BAD800E8E011C00EF012C00FF012001A0E102488
:10BAE8000A6E000E11200B6E12C00CF013C00DF080
:10BAF80079EC5FF00EC0D9FF0FC0DAFF030EDE1835
:10BB0800D8A41200140E10240A6E000E11200B6E19
:10BB180014C00CF015C00DF079EF5FF002D00A4A9E
:10BB28000B2A0AC0F6FF0BC0F7FFF86A0800F550A9
:10BB38000AE00AC0F6FF0BC0F7FFF86A0800F550E4
:10BB48000C180D10ECE10AC0F6FF0BC0F7FFF86AFD
:10BB58000800F5500A6E0B6A12008380838E000E6F
:10BB68000A6E040E0B6E0D6AF60E0C6E010E0F6E49
:10BB78000E6A26EC5FF00B0E00019D6FFE0E9E6FA5
:10BB88004FEC60F0180E9D6FFF0E9E6F4FEC60F04B
:10BB9800839E839012000A6E0A500EE0AFEC60F0AC
:10BBA800200EE82EFED7B2EC60F0CC0E00D0E82EC6
:10BBB800FDD700D000D01200AFEC60F0C00E00D06E
:10BBC800E82EFDD7B2EC60F0350EE82EFED7000067
:10BBD8001200000EF2BE010E0D6E0B50030B7F6EAD
:10BBE8000AC07EFF0CC080FF3F0E81168184F29E42
:10BBF800550E826EAA0E826E818281B2FED7819422
:10BC08000DB002D0F29E01D0F28E1200200E206EEE
:10BC18001CC021F01DC022F0246A256A2B6A2C6AF8
:10BC2800210E166E1EC017F01FC018F0200E196ED8
:10BC3800EEEC56F024501C24D96E25501D20DA6EE7
:10BC4800DF6A120052C04BF053C04CF005EC45F0CF
:10BC5800566E565011E152C00BF053C00CF0540E02
:10BC68000D6EC5EC52F0566E565006E152C0D9FF23
:10BC780053C0DAFFDE6ADD6A56501200176E17AE3F
:10BC88000ED0179E0C6A0D6A0E6A0F6A370E63ECA7
:10BC980059F0186E010E186402D01850120013C023
:10BCA8000CF014C00DF015C00EF016C00FF01750B0
:10BCB80063EF59F0AFEC60F00A0E0B6EF80EE82E49
:10BCC800FED70B2EFCD700D0B2EC60F0E00E00D00F
:10BCD800E82EFDD767EC60F0090E0B6E840EE82E97
:10BCE800FED70B2EFCD7B2EF60F0130E0B6E880E4A
:10BCF8000A6E0ED09BEC60F0FF0A0DE0E40E00D057
:10BD080000D0E82EFCD700D000D00A06D8A00B0639
:10BD18000A500B10EFE10A500B10D8A4010C000CCC
:10BD280060900F0E0F01596F070E396F356F4F0E68
:10BD3800936E8A6A8A888A828A82010E8F6E130EAF
:10BD48000E01B76F0F0EFA6F100EFC6F140EB86F5E
:10BD5800090EFD6F090C20EE01F00A50D9260B5090
:10BD6800DA22DF500F6E106A0AC0D9FF0BC0DAFF63
:10BD7800DF500C6E0F500D6E0C500F6E0DC010F092
:10BD88000FC00AF010C00BF012001EC03EF11FC019
:10BD98003FF1220E246E176A186A20C019F021C0DC
:10BDA8001AF0240E1B6E85EC14F03EC1D9FF3FC17A
:10BDB800DAFFDF6A01013E6B3F6B12002F0E0A6E3D
:10BDC800070E0B6E0D6A0C6A010E0F6E0E6A26ECDA
:10BDD8005FF0038227EE2FF053C1DFFF0392010EBD
:10BDE800A9EC56F083800101536B12009F869E8454
:10BDF800090E0E01FD6F9F989C6A890E9B6E9C6AC6
:10BE08009E989D8E9D889D9AC599F28AF28E9E90E5
:10BE18009D9C9E9A9E8A12003031323334353637D3
:10BE280038394142434445462F071F604020687017
:10BE38006469736B2E636667004850393132314448
:03BE4800000000F7
:10BE4C000AC010F00BC011F008D010C0D9FF11C0FF
:10BE5C00DAFF0CC0DFFF104A112A0E06D8A00F061D
:10BE6C000E28F3E10F28F1E112000BD00BC0F6FF06
:10BE7C000CC0F7FFF86A0800F55082EC60F00B4A32
:10BE8C000C2A0BC0F6FF0CC0F7FFF86A0800F5503F
:10BE9C00EDE112000F6A110E0E6E09D00A0EE82E9B
:10BEAC00FED700D0010E0A6E200E38EC5CF00E06A8
:10BEBC00D8A00F060E28F2E10F28F0E112000A6E4E
:10BECC000A5009E0966A4F0E936E220E966E400E43
:10BEDC00956E968A400C966A100E966E2A0E966E89
:10BEEC00900E936EF4D70AC0D9FF0BC0DAFF0CC0CA
:10BEFC00DFFF0A4A0B2A0DC00CF00D6A0AC0D9FFED
:10BF0C000BC0DAFF0CC0DFFF0A4A0B2A1200AFECA1
:10BF1C0060F0200EE82EFED7B2EC60F0300EE82E6A
:10BF2C00FED767EC60F00B6EB00E00D0E82EFDD79C
:10BF3C000B5012002F0E0A6E070E0B6E0D6A0C6A58
:10BF4C00010E0F6E0E6A26EC5FF0010EE8CF2FF794
:10BF5C000382A9EC56F0039212000A50D96EDA6AE9
:10BF6C000B50DE1804E10AC00AF00B6A12000A2A10
:10BF7C000A04D96EDA6ADF50F0E10A6A0B6A120021
:10BF8C000AC010F00BC011F010C0D9FF11C0DAFFBD
:10BF9C000CC0DFFF104A112A0E06D8A00F060E5057
:10BFAC000F10F2E11200070E8C6E9150070B0A6E07
:10BFBC00888A8DAA02D0080E0A26020E01015C198D
:10BFCC0003E10A1C0F0B0A6E0A5012000A6E030ED4
:10BFDC000A6006D096500A18F00B0A18966E1200DA
:10BFEC000AC093FF9650F00B0A09966E12000101DD
:10BFFC003E513F1109E03EC1D9FF3FC1DAFF0DC0F0
:10C00C00DFFF3E4B3F2B12000D5082EF60F00C6AAD
:10C01C000D6AD8900C328DEC5FF0000901E00C8EAB
:10C02C000D2A070E0D64F5D70C50120003AEFED787
:10C03C00F29E0AC0D9FF0BC0DAFF06C0DFFF039ED9
:10C04C00F28E8982055012000B6E0C6A0B50010B9C
:10C05C00CFEC5DF0D8900B320C2A070E0C64F6D79F
:10C06C00070C020E586E400E02011B6F7E0E000173
:10C07C009D6FFA0E9E6F4FEF60F0B9EC60F09BEC89
:10C08C0060F079EC5EF0000901E0010CA8EC60F0C6
:10C09C00000C9F0E1E6E176A186A9DC019F09EC088
:10C0AC001AF01E0E1B6E85EF14F00B50030B7F6EF7
:10C0BC000AC07EFF3F0E8116818000000000805078
:10C0CC00120088888DA803D0010E0A6E01D00A6A6E
:10C0DC000A5012000A6E01D004000E01CDA9FCD743
:10C0EC000AC09AFF12000A6E0AC092FF0E01CDA17F
:10C0FC00FDD7CD91925012000A6E01D004000E01B2
:10C10C00CDA9FCD70AC09AFF120003AE8982010E9A
:10C11C0003AE000E0A6E0B6A12000A6E02D0838CFC
:10C12C00839C0A060A28FBE1120092680E01CDA13D
:10C13C00FDD7CD91925012000A6E0A5001E0010C0D
:10C14C005C501200B7EC60F09BEF60F08390536B87
:10C15C001200839888981200839888881200039E96
:0BC16C00120085801200859012000177
:10F85E0000819FE0FC407E80FC000020004F4B00AA
:10F86E004449534B5F455252004E4F545F524541EF
:10F87E004459004E4F5F46494C45004E4F545F4F22
:10F88E0050454E4544004E4F545F454E41424C4507
:10F89E0044004E4F5F46494C455F53595354454DB6
:10F8AE0000000D0A202532582025325820253273AB
:10F8BE002025327320253273202532732025327392
:10F8CE002025327320253273202532732025347380
:10F8DE00202534732025347320253473202534736A
:10F8EE0020253473202534732025347320000D0A0F
:10F8FE0048504469736B204D6B204949202831389C
:10F90E004634364B34302920257320257320257339
:10F91E00205374617274696E672E2E2E0D0A000DBF
:10F92E000A4461746120706F7274206973202558C7
:10F93E00202D2053686F756C64206265203C3E203C
:10F94E0030784646000D0A5365656B20657272204D
:10F95E002564203E2025642C202564203E2025642D
:10F96E002C202564203E202564000D0A53746174FA
:10F97E00757320706F7274206973202558202D20A6
:10F98E0053686F756C642062652030784646000DB2
:10F99E000A4461746120706F727420697320255857
:10F9AE00202D2053686F756C642062652030784678
:10F9BE0046000D0A526420752025642072746E2054
:10F9CE0025642C202564206279746573207265612C
:10F9DE00640D0A000D0A2530345820535338307800
:10F9EE003A5374617475732C20756E697420256496
:10F9FE003A20256420000D0A4D6178205665637407
:10FA0E006F72206469736B20256420256C64202836
:10FA1E00256C582920000D0A44736B73656C2069A0
:10FA2E00732025642C206E756D62657220697320BB
:10FA3E00256420000D0A4469736B206368616E674C
:10FA4E00656420746F2025642025303258253032AD
:10FA5E0058000D0A426C6F636B73697A6520666F8E
:10FA6E0072206469736B20256420697320256400FD
:10FA7E000D0A5374617475732073657420746F204E
:10FA8E00706F776572206661696C000D0A253032E1
:10FA9E0058253032582053533830783A466D7420FA
:10FAAE006F70747300466F756E6420616E205254D1
:10FABE00432066696C652061742025580D0A004C40
:10FACE006F6F6B696E6720666F7220616E20525485
:10FADE00432066696C650D0A000D0A5573696E67E1
:10FAEE00206469736B2067656F6D6574727920256C
:10FAFE0073200046696E6446696C65206661696CA8
:10FB0E006564207365617263680D0A000D0A537493
:10FB1E006174757320706F7274206973202558207C
:10FB2E002D204F4B000D0A5365656B20746F2025F9
:10FB3E006C64206661696C6564202564000D0A574B
:10FB4E00726974655F736563746F72732066616941
:10FB5E006C202564000D0A454550524F4D206469B6
:10FB6E00736B206E756D626572202564000D0A44FC
:10FB7E0069736B2073656C656374206E756D626559
:10FB8E0072202564005365656B696E6720746F2063
:10FB9E00736563746F722025580D0A0046696E6492
:10FBAE0046696C65206661696C6564207265616486
:10FBBE000D0A000D0A4F70656E696E6720657869D3
:10FBCE007374696E6720257320000D0A4461746199
:10FBDE0020706F7274206973202558202D204F4B92
:10FBEE00000D0A476F7420256C7520202D2072653C
:10FBFE0073657474696E670020255820255820257A
:10FC0E005820255820256C752020200A000D0A57F3
:10FC1E00726F7465206469736B6E6F3A2025642071
:10FC2E00000D0A57616974696E6720666F722063F2
:10FC3E0061726420000D0A54726967706F696E7488
:10FC4E0020697320256420000D0A46696C65202505
:10FC5E0073206973206F70656E20000D0A727463D5
:10FC6E005F726561642825642C25582900416464FF
:10FC7E007265737320256420202020202020000D23
:10FC8E000A253032582530325820457869742000C4
:10FC9E0020436F6C642025582C2025582C20255885
:10FCAE00004E6F742061204C4946206469736B0DC1
:10FCBE000A000D0A5265616420646573637269629D
:10FCCE006520000D0A46696C652025582069732051
:10FCDE00257320000D0A4469736B20255820697323
:10FCEE0020257320000D0A416464726573732069C8
:10FCFE00733A202564000D0A487374206279746586
:10FD0E007332202564000D0A204F7074696F6E7374
:10FD1E002025640D0A000D0A57726974652066610C
:10FD2E00696C202564000D0A52656164696E672056
:10FD3E005254430D0A000D0A416D69676F20393127
:10FD4E003231440D0A000D0A53532F383020393109
:10FD5E003232440D0A000D0A44736B73656C2069D0
:10FD6E007320256420000D0A5265616420256420ED
:10FD7E00627974657300566563746F7220697320BF
:10FD8E0025580D0A000D0A5353383078202564206B
:10FD9E0025642000222A2B2C3A3B3C3D3E3F5B5DE6
:10FDAE007C7F000D0A4F70656E696E67202573208B
:10FDBE0020000D0A44656275672069732025642052
:10FDCE00000D0A436C6F636B20697320256420005D
:10FDDE000D0A50726F746F20697320256420000D18
:10FDEE000A5265616420636F6E66696720000D0AB2
:10FDFE0046696C656E616D6520257320000D0A469F
:10FE0E006F726D617474696E67200072633D257543
:10FE1E002046525F25730D0A002A2A204E4F204499
:10FE2E0049534B202A2A002A2A2056657269667980
:10FE3E00202A2A000D0A73627974657331202564B5
:10FE4E00000D0A41737365727420454F49000D0A07
:10FE5E004173736572742041544E000D0A4E6F202B
:10FE6E006361726420256400646573637269626500
:10FE7E002E636667002F6C6966646174612E626919
:10FE8E006E000D0A456E61626C6520505000EB7677
:10FE9E00904558464154202020000D0A4D6F756E36
:10FEAE0074696E6720004A616E2033312032303221
:10FEBE0034000D0A41737365727420505000202572
:10FECE005820772041544E20000D0A476F74204170
:10FEDE00544E31000D0A476F742041544E32000DBE
:10FEEE000A476F742041544E33004C6F6164696E43
:10FEFE00672E2E2E002049442025582530325800DA
:10FF0E002A2A20525141202A2A00466D74206578F3
:10FF1E00697420000D0A476F74204946430020255E
:10FF2E00643A20253032580020476F742041544ED9
:10FF3E000031393A31343A3135005B2532582025BB
:10FF4E00645D004572726F722025640048504469EA
:10FF5E00736B20003C6964656E743E004E6F2063C7
:10FF6E006172640072633D2564200044534B534517
:10FF7E004C004E414D452558004449534B255800E1
:10FF8E0046415433320044454255470050524F5477
:10FF9E004F00526561647900302E3237004144447F
:10FFAE0052004946432000454F49200052454E20FD
:10FFBE0000535251200044415620004E444143000C
:10FFCE004E52464400464154005254430054524748
:10FFDE0000434C4B0025325800443000443100445D
:10FFEE003200443300443400443500443600443774
:02FFFE00000001
:020000040020DA
:10000000FFFFFFFFFFFFFFFFFFFFFFFFFFFFFFFF00
:020000040030CA
:0C0000008CFFFFFC8EFFFFFFFFFFFFFFE7
:00000001FF
